:10000000584C00203DEA00001B6D0000A5E30000F5
:100010003B6D0000EF6D0000DB7000000000000091
:10002000000000000000000000000000FB70000065
:100030002F7100000000000027740000EF84000012
:10004000197400000785000045BB0000A5CC000026
:100050003F8600006F8600008FB90000AB8700006C
:10006000E78700000B880000EF880000378B000056
:100070007B8B00009F8F0000A38F00009BB50000CA
:10008000DBE30000BDA5000091E6000057E700009B
:1000900063E7000089EB00008BEB00008DEB0000B4
:1000A0008FEB000091EB000093EB000095EB00005C
:1000B00097EB000099EB000000000000000000003A
:1000C0009BEB00009DEB00009FEB0000A1EB00000C
:1000D000A3EB0000A5EB0000A7EB0000110E000051
:1000E000A9EB000039C60000ABEB000000000000E7
:1000F00000000000ADEB000000000000AFEB0000CE
:1001000000000000000000000000000000000000EF
:1001100000000000000000000000000000000000DF
:1001200000000000000000000000000000000000CF
:1001300000000000000000000000000000000000BF
:1001400000000000000000000000000000000000AF
:10015000000000000000000000000000000000009F
:10016000000000000000000000000000000000008F
:10017000000000000000000000000000000000007F
:10018000000000000000000000000000000000006F
:10019000000000000000000000000000000000005F
:1001A000000000000000000000000000000000004F
:1001B000000000000000000000000000000000003F
:1001C000000000000000000000000000000000002F
:1001D000000000000000000000000000000000001F
:1001E000000000000000000000000000000000000F
:1001F00000000000000000000000000000000000FF
:100200000146001101EBD062DFF8E03B521153F8D8
:100210002200A1EB4211C84033E2DFF8D41B0844AE
:10022000704780B5FFF7F9FF012103E080B5FFF7C4
:10023000F4FF0021016001F08CFA01BDDFF8B01B72
:10024000085801F044B838B50446FFF7F7FF050039
:100250001CBF2046FFF7EAFF284632BDDFF8940BAB
:1002600000687047DFF88C1B086001F003B9DFF805
:10027000880B0068C0B2704710B50446210604F030
:100280000F0002D5092808DB01E0092805DBDFF8AB
:100290006C1B40F2B74001F037FBDFF8640B22061D
:1002A00004F00F014CBF00684068C84000F0010036
:1002B00010BD01F009B8DFF84C0B0168082901D125
:1002C000012070470020704780B5FFF7F4FF002839
:1002D0001FBFDFF8340B006800280120C0B202BD48
:1002E00080B5FFF7E8FF20B1FFF7EEFF401E804129
:1002F000C00F02BD80B50DE080B5FFF7E5FF30B956
:10030000DFF8000B01680D2901D0002002BD01209B
:1003100002BD80B5FFF7CFFF00B1012002BD000094
:1003200038B500F060F902D5092D0ADB01E0092D8E
:100330000ADBDFF8481C40F27B1001F0E5FA2006EA
:1003400002D500BF02A000E006A030F9150032BDC2
:1003500008010C011001140118011C0120012401E5
:100360002C0100003001340138013C0140014401FE
:1003700048014C015001000038B500F034F902D5B5
:10038000092D0ADB01E0092D0ADBDFF8F01B4FF431
:10039000D27001F0B9FA200602D500BF03A100E037
:1003A00005A1495D0120884032BD0000020304051B
:1003B000060708090B0000000C0D0E0F1011121398
:1003C000140000002DE9F04114461D46AC420646DB
:1003D0000F46DFF8288A05D208F1780140F2DB10D9
:1003E00001F092FA386800281CBF00F06040B0F1BC
:1003F000005F05D008F1780140F2DD1001F084FAC9
:100400007868A84204D2002171603A68326007E03F
:100410007560401B3968316078603A68AA183A60A4
:10042000AC4202D110B1012000E00020C0B2BDE812
:10043000F08170B50D460446286800F06040B0F1C8
:10044000005F164605D0DFF8341B40F2022001F0B1
:100450005BFA6868864288BF064628682060666046
:100460006968891B6960286836182E60686800B161
:100470000120C0B270BD70B50E460546306800F070
:1004800082F805D0DFF8F41A40F2232001F03CFA9C
:100490007068844288BF0446002C0CBF002030687E
:1004A00028606C607068001B706031686118200003
:1004B00018BF01203160C0B270BDF8B50C460646C9
:1004C0002068DFF8387900F06040B0F1005F154631
:1004D00005D107F1780140F2412001F015FA60687A
:1004E000854288BF0546412D05D307F1780140F2CA
:1004F0004B2001F009FADFF86C7C21682A46384667
:1005000001F02AFA376075606068401B60602168FE
:100510006D182560606800B10120C0B2F2BDF8B569
:100520000D4606462868DFF8D47800F02CF805D18F
:1005300007F178014FF4197001F0E6F96868844218
:1005400088BF0446412C06D307F1780140F26E20A3
:1005500001F0DAF900E044B1DFF8087C29682246AE
:10056000384601F0F9F9376001E00020306074602E
:100570006868001B6860296861182000296018BF3E
:100580000120C0B2F2BD00F06040B0F1005F14463F
:10059000704710B50446210604F00F0002D5092863
:1005A00008DB01E0092805DBDFF8D01940F28E20D6
:1005B00001F0AAF9204610BD70B500F014F8DFF87C
:1005C000A86B02D5092D0ADB01E0092D08DBDFF855
:1005D000AC1940F2AB2001F097F9200600D5903617
:1005E00006EB051070BD0446200604F00F057047A9
:1005F00038B50446210604F00F0502D5092D0ADBA3
:1006000001E0092D09DBDFF8741940F2BE2001F08A
:100610007BF9200601D5002000E010202D18E8B25B
:1006200032BD1028ACBF103840F08000C0B2704717
:1006300080B5FFF76EFE18B1DFF8801B0020086060
:100640000022DFF8000CC27001BD38B50446210657
:1006500004F00F0502D5092D0ADB01E0092D09DBA5
:10066000DFF8181940F29B2001F04EF9200601D561
:10067000042000E0282000EB8500BDE83240C0B235
:10068000CFE500F00100704700000000F8B5044617
:1006900000F06DFF2046FFF78FFF0546012620067C
:1006A000DFF8A07B18D400F02BF9F968C943C140EA
:1006B000C80703D5204601F093F80AE0002028601F
:1006C00000F01EF900F016F9B968864021EA060626
:1006D000BE600320A87338E004F00F00082817DA82
:1006E000802CDFF8101C08D0400000F2B4700860C5
:1006F00048684A6840F0020006E040F2B4720A60BE
:1007000048684A6840F00400C0B210434860486836
:1007100000F0F6F8FA68B96862EA0102C240D00750
:1007200013D500F0EDF800F0E5F8B96886400E4307
:10073000BE6000202860032205A1AA7368460B68EA
:10074000796800938DF80240884700F003F8F1BD06
:1007500006000003002001F021B997E770B5DFF82B
:10076000E45AA868EC68000C54EA004413E094FAD8
:10077000A4F0B0FA80F6F0B2FFF753FF00F00F00DC
:10078000082804DAF0B2FFF74CFFFFF77FFF0120E3
:1007900000FA06F6B443EAD140F2FF10A86070BD3B
:1007A0001CB5DFF8A01A00BF04A3002048708870B1
:1007B00068461C6849680094884713BD0100000022
:1007C000704738B5FFF734FF8020FFF7F5FE00F0E3
:1007D000C5F81CBF006800280AD18020FFF708FF79
:1007E0008540E94304F10C00BDE8344001F00EB946
:1007F00031BD70B504462206DFF8005605D405F178
:10080000780140F2BF3001F07FF804F00F010829B1
:1008100005DB05F178014FF4707001F075F814F004
:100820000F0F05D105F1780140F2C13001F06CF8ED
:10083000FFF7FEFE2046FFF7BFFE00F055F81CBF95
:100840000068002809D100F05BF88640F14305F10B
:100850000C00BDE8704001F0D9B870BD7CB504460D
:100860002206DFF8985505D505F1780140F21D40C4
:1008700001F04AF804F00F01082905DB05F17801C1
:1008800040F21E4001F040F814F00F0F05D105F1C1
:10089000780140F21F4001F037F8FFF7C9FE20460B
:1008A000FFF78AFE00F020F804D100F029F800F0EC
:1008B00015F80DE0006858B900F022F800F00EF8C5
:1008C00005A10A68696800928DF802406846884769
:1008D00000F0B3F973BD0000060000008640F1434C
:1008E00005F10C0001F092B80126817BDFF8545924
:1008F00003297047F96806FA00F021EA0000F86061
:10090000204675E65DE7812073E7822071E783204A
:100910006FE784206DE785206BE7862069E78720F5
:1009200067E7000038B5FFF783FE8820FFF744FE35
:1009300000F014F801D188203BE0006850B988200D
:10094000FFF756FE00F03AF803A10A6800928823E8
:1009500000F02AF831BD0000060000000125817B6F
:10096000DFF8E0480329704738B5FFF761FEDFF88C
:10097000F807DFF8D048817B0125032901D1002049
:1009800017E0006858B9FFF733FE00F017F800BF12
:1009900004A10A680092002300F006F831BD00F0BF
:1009A000F9FE31BD060000008DF80230684661682E
:1009B0000847FFF71DFE00F001F831BD8540E9430F
:1009C00004F10C0001F022B8012047E7022045E7BE
:1009D000032043E7042041E705203FE706203DE7E9
:1009E00007203BE71CB5FFF723FEDFF8940A817B65
:1009F000032915D0006898B90820FFF7F9FD0121F7
:100A000001FA00F0DFF83C48C14304F10C0000F0AB
:100A1000FDFF00BF03A10A6800920823FFF7C4FF8F
:100A200013BD0000060000007CB500BF11A0DFF878
:100A3000546A016800910124306EADF802008820EC
:100A4000FFF7D6FD04FA00F5306848B1C10302D4BF
:100A500010F1010F04D00820FFF7CAFD84402543A0
:100A6000DFF8E017886805438D6068464968884765
:100A700073BD0000000000007CB5DFF8C8570446D5
:100A80000E46A8680121B1400843A860200613D58E
:100A90002046FFF745FCFFF7D6FB38B120468028FB
:100AA00002D0FFF7A6FE01E0FFF78BFEE868F040FA
:100AB000C1070DD407A204E0E868F040C10707D4DD
:100AC00005A21368696800938DF80240684688475C
:100AD00073BD0000060000000600000110B5DFF83D
:100AE0006447A078FFF784FD0146A078BDE8104078
:100AF000C2E700007CB5FFF7BAFBDFF848470546C0
:100B0000A078FFF775FDA268E168D24392B2114365
:100B1000C140C80744BFA078FFF7B8FD280654BFFE
:100B200000208020A07001260020FFF761FD05460F
:100B30008020FFF75DFD06FA05F506FA00F0054393
:100B4000FFF73DFF8020FFF753FDA16886400E436D
:100B500003A06168A660026800F041F873BD000060
:100B60000500000038B5FFF779FB0546FFF77AFB73
:100B700000F0EFFDE805DFF8CC4604D5012100BF09
:100B800012A000F029F8A80503D5002110A000F05C
:100B900023F86A0519D56078B8B1FFF78AFB28B148
:100BA000DFF8D81340F2FE4000F0AEFE0020DFF880
:100BB000E02B6070012111605820FFF732FB00BF6D
:100BC00004A001680091FFF7F1FE31BD02000000B2
:100BD0000300000004000000617002686168009278
:100BE0006846084738B5DFF8B00A046800F0B0FD81
:100BF000FFF776FBB0B1DFF84C160A6922F001105E
:100C000002F0011204430A610CE094FAA4F0B0FA75
:100C100080F5E8B2FFF705FD0121A9408C43E9B258
:100C2000FFF72AFF002CF0D1BDE8314005E090FA33
:100C3000A0F0B0FA80F0C0B270472DE9FF47DFF8AE
:100C40000446E078002840F0CF80DFF8B08121E052
:100C5000384600F0E0FC8246AA896968D5F800C0F1
:100C600053466846E047814600980199002839D0EC
:100C700051453DD20221A97304F10C00314600F028
:100C8000C5FE0FF288110A68616802928DF80A7039
:100C900002A88847E068A168084000F0A58010F02D
:100CA000012F18BF00F00120FFF7C1FF0646FFF734
:100CB000B8FC0746FFF780FC0546286828B908F10C
:100CC000780140F2715000F01FFE012000FA06F694
:100CD000F6433906BCD5AA8969682B6868469847E7
:100CE00090B910E059B108F1780140F28D5004E05C
:100CF00005D008F1780140F29C5000F005FEB9F1F2
:100D0000000F01D100202860FFF703FB18B1DFF8C6
:100D1000AC14822008600122A068E2700640A66040
:100D2000A96801984118A9603806019C009D07F048
:100D30000F060FD5082EA8BFDFF8940A0EDA04D3E9
:100D4000414640F2345000F0DFFD14204643DFF806
:100D5000840A10E0082E04DBDFF87C0A056044609A
:100D60000CE004D3414640F2435000F0CDFD142086
:100D70004643DFF8680A8551011D8C51FFF7B0FA30
:100D800018B34FF48270FFF751FA3846FFF75DFC55
:100D9000022000F059FE4FF48270FFF74FFA00284E
:100DA000EFD01E2000E0022000F04EFEDFF8C40A63
:100DB00001688A06F7D5012000F046FE3846FFF7A5
:100DC000AFFAFFF73BFA78B9DBE73846FFF73DFCAF
:100DD0003846FFF7A5FAFFF731FA28B94FF48070CB
:100DE000FFF72CFA0028F3D0BDE8FF8700E100E010
:100DF00000700240007402408074024068D200001B
:100E0000107502403001001034010010060000028D
:100E10002DE9F843DFF8600A07683C4600260DE03C
:100E200094FAA4F0B0FA80F0C0B28540800000F5DA
:100E30008070FFF708FA00B12E43AC430125002C67
:100E4000EED1FFF74DFA0028344679D0DFF8F4638D
:100E5000F078002874D1A00272D5DFF898C440F26F
:100E6000A979CCF80090DCF80420D0B218B1DCF8F5
:100E70000400C0B2024040F2AA7ECCF800E0DCF8E8
:100E80000400C1B219B1DCF80410C9B2084040F244
:100E9000AB78CCF80080DCF80410CBB21BB1DCF8E6
:100EA0000430DBB2194040F2AC73CCF80030DCF80F
:100EB00004301A40D2B242B1336913433361CCF8E3
:100EC0000090CCF80420DCF8042040F2AD73CCF89C
:100ED0000030DCF804201040C0B248B1326942EA68
:100EE00000423261CCF800E0CCF80400DCF80400E9
:100EF00040F2AE72CCF80020DCF804000140C9B228
:100F000069B1C807CCF8008048BF44F40004CCF8AD
:100F10000410C806DCF8040048BF44F0010432693C
:100F200032F001101CBF07F080710C4312F0011F5A
:100F300006D0780504D522F00112326144F48064B1
:100F4000E60D06F0010634F40004DFF830790BE01A
:100F500094FAA4F0B0FA80F85FFA88F857F82800FD
:100F6000804705FA08F08443F2D1FFF766FE16B118
:100F7000BDE8F143BEE5BDE8F1830000E0D200002A
:100F800070B5040005D1DFF8E81640F29B6000F070
:100F9000BBFCDFF8EC18087808B1082070BD4C6085
:100FA0000120087000254FF4007445F0800606F01B
:100FB0000F000828ACBF21464021F0B200F09CF998
:100FC000F0B2FFF7F9FA00F013F8EEDD002505F0B6
:100FD0000F000828ACBF21464021E8B200F08CF990
:100FE000E8B2FFF7E9FA00F003F8F0DD002070BD89
:100FF00000218173016081606D1CE8B20828704790
:1010000010B5904C2078012805D0DFF864164FF415
:10101000D86000F079FC00216160217010BD2DE9DD
:10102000F041884F3878012805D0DFF8441640F2A7
:10103000C96000F069FC4FF40060FFF713F9FFF797
:101040005BF9DFF84048DFF8406849F2753560B178
:1010500000F08DFA306820B93560032121603560D9
:1010600001E003202060FFF775FBFFF743F960B153
:1010700000F07DFA306820B93560C02171613560BB
:1010800001E0C0207061FFF765FBDFF800880120F8
:10109000C8F8000000F05DFBDFF8F41708680005F1
:1010A000FCD54FF40060FFF7DDF8FFF723F960B1DE
:1010B00000F05DFA306820B935600021716135605B
:1010C00001E00020706100F069FCDFF8C8070168EA
:1010D000082908D1DFF8C00740F2E371016040221F
:1010E000426000F036FB8020C8F81C000021C8F8E0
:1010F000301040F2FF10B860F960FFF799FA002055
:101100000221B8703970FFF7F7F870B100F02FFACC
:10111000306820B9356000212160356001E0002091
:101120002060BDE8F04100F039BCBDE8F08110B5A9
:10113000444C207828B9DFF8381540F2357000F0BB
:10114000E3FB00F03DF8DFF8300701684160002064
:10115000DFF83817086000F0FCFAFFF769FA0120A1
:10116000207010BDC02A00207424002038B5354DF1
:1011700004462878022805D0DFF8F41440F24370C2
:1011800000F0C2FB00216970DFF8105714B9FFF7B7
:10119000A7F808B1DFF80857DFF8DC06DFF8042706
:1011A0000560C021DFF8000711708023DFF8FC26FE
:1011B00003600121116000F0CCFA31BD1C7C0240BB
:1011C00080B520480178022905D0DFF8A41440F248
:1011D000627000F099FBDFF8D806802101602720BB
:1011E000FFF70EF880B1FFF7B9FADFF8C01600205C
:1011F000086000F0AEFA8022DFF8B806DFF8B836F3
:1012000002604FF0FF31196001BDDFF8740600780D
:1012100000B101207047DFF868060178022901DB80
:10122000012070470020704780B5DFF85406017830
:10123000022905DB2720FEF7E3FF10B1012002BDE4
:10124000002002BD94250020002010B500F097FB7F
:10125000DFF82C164878002478B1FFF77FFADFF822
:1012600030060168890508D4DFF8501601220A60AB
:10127000006880054CBF0C60012420E0002010B500
:1012800000F07DFBDFF8F8154878002400281EBF29
:10129000DFF828160868002811D00C60FFF72AF83C
:1012A000012460B1DFF8E015086830B949F2753003
:1012B0000860C0224A61086001E0C0204861FFF771
:1012C00049FA204610BD0000DFF8F005006800B1C3
:1012D0000120C0B27047DFF8E01501E0DFF8981593
:1012E000DFF8DC0508607047DFF8941500204870CF
:1012F000704700000078024070B50D46EA070646C8
:10130000DFF8C04505D504F1780140F2DB7000F04C
:10131000FBFA290006F00F0014D1082812DA04F1B4
:10132000780140F2DD7000F0EFFA412D05DB04F1A9
:1013300078014FF4FC6000F0E7FA3046FFF73CF923
:10134000858170BD0828F0DBDFF87C050068C0B23D
:1013500080280CBF4FF400704FF48060A842ECD29C
:10136000E5E780B5FFF728F9808902BD80B5FFF772
:1013700010F9BDE80240FEF77FBF70B50446FEF7E6
:10138000FBFFDFF8F41408602046FEF775FF002825
:101390003ED12046FFF7FDF80646310606F00F0065
:1013A00002D5082808DD01E0082805DDDFF814155E
:1013B00040F2C64000F0A8FA06F00F000125320600
:1013C00005FA00F0DFF8041503D50B681843086030
:1013D00002E04A681043486000F0BBF914F00F00C7
:1013E00016D0210614D4082812DA00F0C0F82046DE
:1013F00000F0F6F9FFF784FADFF88414CA68854034
:1014000022EA0505CD600020BDE8704000F0C6BAB4
:1014100070BD38B50446FFF739F92046FFF7B9F833
:101420000546290605F00F0002D5092808DB01E072
:10143000092805DBDFF88C1440F2D74000F064FA8D
:1014400005F00F00012101FA00F0C0432A06DFF881
:101450007C1403D50B681840086002E04A6810400D
:10146000486000F076F92046FEF786FFDFF8481462
:10147000086031BDBFF36F8FBFF34F8F704700001F
:10148000F4240020C07402402DE9F84381460C4644
:10149000FFF7AEF80546DFF82C842CB908F1780187
:1014A00040F62A0000F030FA00F061F819F00F0F52
:1014B000DFF8CC6304D1B178894518BF102451D12D
:1014C00000F08DF848BF11244CD44846FFF774F85B
:1014D000074609F00F010C20414370185FEA0962CA
:1014E00019D5216800F1140901F06041A068B1F13B
:1014F000005F04D1C00709D4DFF8D41309E0C007A6
:1015000054BFDFF8D013DFF8D01302E0DFF8CC03CC
:1015100013E0396012E000F18009206800281CBF48
:1015200000F06041B1F1005F05D008F1780140F6AC
:10153000840000F0E9F9DFF8A803386094E80700B8
:1015400089E807000021B960B973C7F80490012049
:10155000F16800FA05F50D43DFF88803F560802196
:1015600000240160FFF7F6F82046BDE8F283002072
:1015700000F005BAF8B507460C46FFF739F80546FE
:1015800024B93B4940F69A0000F0BEF9FFF7EFFF9F
:1015900017F00F0FBA4E04D1B1788F4218BF102444
:1015A00019D100F01CF848BF112414D43846FFF7B5
:1015B00003F80021816022680260002261684160B6
:1015C00082730121F06801FA05F50543C549F5600C
:1015D000802000240860FFF7BDF82046F2BDB16806
:1015E000F068C94389B20843E840C0077047BE4865
:1015F000704738B50C46FEF7DFFF0546FFF7B7FF2B
:10160000A9682160286800280CBFAC7B0424FFF780
:10161000A1F8204632BDD0B5FEF7BBFF0446200638
:1016200004F00F06A74F02D5082E09DD01E0082EB1
:101630000BDD394640F25F4000F066F9200604D524
:1016400039464FF48C6000F05FF9082E05DBA7489F
:101650000068C1030AD50020D0BD04D3394640F24A
:101660006B4000F051F9A24850F82600D0BD0000B0
:10167000E0D2000010B5FEF78CFF044604F00F0026
:10168000082804DB8F494FF49E6000F03DF999482B
:1016900044F480741BE000006C74024010B50446F2
:1016A000200606D4204600F015F810B1204600F0C0
:1016B00097F82046FEF76DFF044604F00F00082857
:1016C00004DB80494FF49F6000F01EF9894800F068
:1016D0003FF810BD10B5FEF75CFF00F00F04082CBA
:1016E00015DA0006774907D5082C24BF4FF481602E
:1016F00000F00AF9804806E0082C24BF40F20D40B3
:1017000000F002F97D4850F82400012800D00020A4
:1017100010BD70B5FEF767FF6A4E02D5082D07DDD4
:1017200001E0082D04DD314640F2A34000F0ECF862
:10173000082D04DB314640F2A44000F0E5F8704883
:101740000460BFF34F8F44F4807400F001F870BD63
:101750000460BFF36F8FBFF34F8F704710B504461F
:10176000082100F099F967480168217041686170AB
:101770008168C26841EA022161800169426941EAE7
:101780000221A1808169C06941EA0021E18010BD88
:101790000875024010B5FEF7A3FD58B1EFF31084B1
:1017A00072B64C20FEF73DFD4C20FEF73AFD84F367
:1017B000108810BDBDE810404C20FEF732BD50200F
:1017C000FEF72FBD5420FEF72CBD2D4880787047C2
:1017D000A076024000760240A077024000770240E7
:1017E0002DE9F04204462206DFF8D89005D509F12C
:1017F000780140F6291000F087F82648204D01684E
:101800000127082904F00F0614D1FEF75DFD88B901
:1018100000F0B5F8FFF774F8A968874021EA0707D8
:101820001D48AF60740004F2C5740460002141607B
:10183000406819E0FFF79BFEFFF762F8A968874050
:1018400021EA0707082EAF600EDA200601D4082E21
:1018500004D3494640F2834000F056F82449002062
:1018600041F82600FFF775FF0020BDE8F04200F0C8
:1018700095B80000747402400473024080D80000E0
:101880009425002014ED064000EC0640007502404F
:101890000074024030010010007802400714C001BB
:1018A0000714E00127E400E004E100E004750240D1
:1018B00084E200E084E100E0087302402C750240FD
:1018C0000414800168D200001C75024010750240AB
:1018D00033040000BB0400001F0500007704000073
:1018E000C503000004E200E0C02A0020C0740240EA
:1018F000A0740240187502402074024044740240F3
:101900000C75024080740240E0B5ADF80000019112
:101910006A46002144F2020000F0D0F807BD30B45E
:10192000002513E050F8042BD30744BFA9F10103AD
:101930009A18091F042942F8045BFAD213468C074F
:1019400044BF15809B1CC90748BF1D7050F8041B7D
:101950000029E7D130BC70474AB1000011F8013BC3
:10196000521E00F8013B1CBF11F8013BF8E770471D
:1019700022490868401E086000D162B6704780B5F1
:1019800000F018F8012803D01D494320FFF7BCFFE1
:1019900072B61A480168491C016001BD80B500F0AB
:1019A00009F8012803D016495120FFF7ADFFBDE823
:1019B0000140DDE7EFF30580C00506D1EFF31480A9
:1019C00000F0010080F00100704701207047EFF344
:1019D0000580C0F3080000280ED0103841B200295D
:1019E00006D5084900F00F00084410F8040C01E087
:1019F0000548405C400970470F207047442C002088
:101A00003CDD000018ED00E000E400E010B5024607
:101A100052E8000F00EA010442E8004393F0000F8F
:101A2000F6D110BD10B50446B4F5000F03D3174925
:101A30009020FFF769FF1348016802688A1A22F0B4
:101A40007F42A242F9D310BD38B50F4D00F010F817
:101A50002868B0FBF2F2B3FBF2F3A34203D20B49C6
:101A60009B20FFF751FF29680948B1FBF0F003E024
:101A7000074A084B044670476043BDE83240D1E74F
:101A80000000000018E000E08C070020F0E20000F9
:101A900040420F00FFFF7F00002200F061B8B1F567
:101AA000807F02D34FF0FF307047017001207047F4
:101AB0000078401E8041C043C00F7047FEB5054608
:101AC0000E46174672B600F043FB00F00DFA0028F0
:101AD000FBD11C481C4C041BE40844F20101240403
:101AE000681A44F0010408D0401E19D13B887A6876
:101AF0001649204600F0C6F917E0B86800F060FB10
:101B00000346029638680190204679680091BA68C9
:101B10000F4900F0D6F90F49204600F0AAF904E079
:101B200032460D49204600F0A7F90C480168CA0763
:101B300000D500BE3A463146284603B0BDE8F04025
:101B400000F06CBB90D4000058D4000064DC0000AE
:101B5000D4E4000080DC000094DC0000F0ED00E044
:101B60004018491C1CBFB1F1010100F8012DF9D149
:101B700070478268521C8260426832B10268531C0E
:101B8000036011704168491E4160704738B5040018
:101B900001D1072032BDDFF8DC05FF22002300F26F
:101BA0000C45826003604360EB60AB602B750846B8
:101BB00000F077FC2C60DFF8C00500F0B9FC20B91C
:101BC0000FF2F05000F080FD002032BDDFF8AC05D0
:101BD000DFF8AC15401AC008704738B5044689B123
:101BE000FFF7F4FF2568DFF89C25002100E0491C81
:101BF000814205D232F82130AB42F8D1216001E0B8
:101C0000052032BD002032BD01B56846FFF7E5FF73
:101C100028B9DFF87405009950F8310002BD0020A2
:101C200002BD0000491EDFF86025032902EBC00059
:101C30000BD8DFE801F002040608022070470420F8
:101C4000704700797047407970470020704703461D
:101C500000201A68C2F38002A2B1186800F00302E3
:101C6000012A02D0022A07D00BE00B68C0F38310D0
:101C7000C01CC3180B6004E00A68800DC01C8018EB
:101C800008600120704780B50021DFF8000500F0F2
:101C900025FD80F3100002BD2DE9F04F85B00D4603
:101CA0009346DFF8D074DFF8E89404460020FFF78D
:101CB00066FE38682860E61CBA6839687868521C85
:101CC000511A07F214424118049207F21C481DE011
:101CD00049464FF4BF70FFF717FE07E001998246AF
:101CE0000098890DC91C00EB91000090049800F049
:101CF00041FD08B1009878605146404600F012FD61
:101D0000B8683968401C411A78684118B14234D229
:101D10000121404600F006FD07F5836000F028FD34
:101D2000049800F025FD786800904FF0000ABD6827
:101D3000009907F10C00294000EB81006946FFF78C
:101D400086FF0028F4D101AB009A07F10C012A406C
:101D500000F0C6F9F8D30199BDF80A0001F00301BB
:101D6000012902D00229B9D0B2E782460198009930
:101D7000C0F3831041180091B8E7BBF1000F05D004
:101D8000A40104F4707444F0050402E0A40544F0D6
:101D900006043A68B86807F10C01024041F8224095
:101DA0000020396876183E60FFF7F8FD012005B085
:101DB000BDE8F08F2DE9FE4FDFF8B8B30646884640
:101DC00017469A46DBF80840012201A95046FFF762
:101DD00063FF0028DFF8BC5343D00198C01C0021EA
:101DE0000BF10C0207E057F821C004EA000342F8A7
:101DF00023C0401C491C5145F5D3300C019F009075
:101E0000FFF741FF8146FFF7E1FE0099814205D3CC
:101E1000DFF87C1340F2A310FFF776FD009A0BF178
:101E20000C00791C214042EA094240F82120B81CEC
:101E3000204000900BF10C0929688847009949F867
:101E40002100F60006F0380646EA8A16C6F30906AF
:101E50000BF10C0046EA88263C4046F0010640F8AB
:101E60002460287D18B100F03FF80028FBD1BDE8C0
:101E7000F78F002300229DE780B50092012300F038
:101E800012F801BDE0B5009201936A460223FFF704
:101E900091FF07BD1FB5069C009201930294032396
:101EA00000F001F81FBD6A4684E77FB5089D099ED2
:101EB00000920193029503960423FFF7F4FF05B007
:101EC00060BD78B585B00A9C0B9D0C9E00F005F8AE
:101ED0000523FFF7E8FF06B070BD0092019302945E
:101EE00003950496704700002DE9FF47A14E7068E6
:101EF0003168884220D006F582670020B860BFF3C1
:101F00004F8F7068B468009006F10C000099214072
:101F100000EB810005E006F10C0004EA010200EB91
:101F200082006946FFF793FE38B1B86828B9306877
:101F300000998142EFD37060CCE0002001AB009AA1
:101F400006F10C01224000F0CBF8F8D301998A4841
:101F500001F00301022945D1019D0199AD0DA9466A
:101F6000502DA8BF502565F39F51019105F10C013B
:101F700000F0E0FA5FEA000A51D000F023FB00F025
:101F8000B9F800982040641C241AA40006F10C0142
:101F9000AC4201EB800119D234B9284606F10C019C
:101FA0004FF00008002503E0204606F10C082D1B29
:101FB000C4B20C232246504600F065FBB8F1000F76
:101FC00009D004F10C03EAB2414601E00C232A4691
:101FD000504600F058FB009809F1030100EB910016
:101FE00000903CE0019901F00301012959D10199C8
:101FF000019AC1F383110529DABF019901F47071C7
:102000004FF4C07122F47072114301910199C1F330
:102010008311C91C890000F08DFA5FEA000A40D0E4
:1020200000F0D0FA00F066F84FF00C094FF000080D
:1020300010E00098411C009106F10C05204005EBD2
:1020400080014B460422504600F01DFB09F10409B3
:1020500008F101080198C0F383108045E9D33C687A
:10206000B86870B1504600F0B1FA2FE0E0684179ED
:10207000012904D122681368514620469847E06838
:102080000468002CF2D1504600F0A0FA0020FFF7BF
:1020900076FCB86808B9009870600020FFF77EFCF5
:1020A00014E03C6805E021688A6820469047E068B3
:1020B0000468002CF7D13848DFF8C42038A1801A12
:1020C000C008000440F00200FFF7D3FE70683168DA
:1020D000884201D1002000E0012004B0BDE8F08773
:1020E00051F8221043F82010401C0099491C032885
:1020F0000091704700230C2201A9504600F0C3BA9A
:1021000030B5024600201B4BD3F8101400E00968DC
:1021100049B1C9680C798442F9D1401C0A28F3DB23
:102120004FF0FF3030BD10F1010F10D0D1680871B1
:10213000D468D3F8101419B9C3F81024216030BD45
:10214000CD6829682160D3F81034D9680A6030BDA1
:1021500010B5124804680121017408E0E168012209
:102160004A712046226851688847E0680468002C5C
:10217000F4D110BD50200020D8E90000D8D40000D0
:1021800058D400000000000058D400006C24002047
:1021900084DD00005C24002090D400006024002036
:1021A0004261636B656E647320666C757368656409
:1021B00000000000D02800207F000000902B0020AD
:1021C00080B500F003F800B90FA002BD10B50D49AD
:1021D00001F58C7200E01A46914210D2531ADB10BE
:1021E00003EBD3735B1001EBC3031C68A042F2D373
:1021F000844238BF03F10801EED3586810BD0020B7
:1022000010BD00001CCB0000556E6B6E6F776E200A
:102210006572726F7220636F6465000018B589B0D3
:102220000B4601218DF800109DF80040144908600C
:102230004B608A6044F20103C01A09D0401E11D1DC
:10224000CA60C86802888A61C8684268CA6109E0D1
:102250000A61086982684A61086902688A610869D6
:102260004368CB6101A82022FFF776FB72B69DF888
:1022700000000028FBD162B60AB010BD00000000CB
:10228000702B0020FEB504460D46E3884BB100BF1D
:102290000FF244260FF248229AA10096284600F039
:1022A0007BFA217A052946D0607A894E48B1A08808
:1022B000FFF7B8FC06EB80007FA14269284600F0DA
:1022C0006BFA2068F16BB0FBF1F0B16BB0FBF1F78A
:1022D00001FB17004FF46162B7FBF2F24FF4616C3F
:1022E0000CFB127C4FF47A777843B0FBF1FE01FBD4
:1022F0001E003C237843BCFBF3F3B0FBF1F13C2020
:10230000029100FB13CCCDF804E0CDF800C02846C4
:1023100075A100F041FAA0880021FFF775FC034683
:10232000207A56F8202028460DF10C0DBDE8F0402B
:102330007AA100F031BAF7BD38B50C46017A05290B
:102340005EA507D0407A30B163A25BA1204600F0C1
:1023500023FA00E01AB12946204600F01DFA204673
:10236000BDE8324000F008BA2DE9F84384B01746C2
:102370000C9D2E7B002281460C4698462A732946E6
:102380004046FFF77FFF062F2CD8DFE807F004094F
:102390000F1A21161D004946284600F0FDF921E0DC
:1023A00022684946284600F0F7F91BE06368226876
:1023B0004946284600F0F0F914E020690290E168EF
:1023C0000191A068009007E0606903902169029183
:1023D000E0680190A1680091636822684946284638
:1023E00000F0DAF9002229464046FFF7A5FF2E73D8
:1023F00005B0BDE8F08300002DE9F84F8A46BAF138
:10240000080F814698464AD80092002298F80CB0EE
:1024100045A588F80C2041460098FFF733FF0027B8
:1024200027A4574506D219F807202946404600F050
:10243000B3F903E02146404600F0AEF97F1C082FB7
:10244000EFD320A1404600F0A7F900261EA71FA445
:10245000564516D219F806507F2D0BDAA5F120004B
:102460005F2808D3284600F0C7F920B9284600F0B5
:10247000CDF900B92E252A462146404600F08CF9B8
:1024800003E03946404600F087F9761C082EDFD37A
:10249000009801224146FFF74FFF88F80CB0BDE8D5
:1024A000F18F01210B4A01E0400849009042FBD224
:1024B000074A9063D1637047257300000D0A00003E
:1024C000202020007C000000200000002563000088
:1024D0004C07002041420F001B5B306D00000000E4
:1024E0001B5B313B33316D005B253032643A253064
:1024F00032643A253032642E253033642C25303353
:10250000645D200025734C6F67732064726F707078
:102510006564202825642925730D0A003C25733E37
:102520002025733A2000000020253032780000007A
:1025300000F076B92DE9F04105460F462E8A00F0ED
:10254000AAF9361F040002D10020BDE8F081F71976
:1025500000200121FF1C20716171A046B7FBF6F736
:10256000E680FFB27F1EC8F80050002607E06179C0
:10257000491C6171C8F8000005608046761CBE42A7
:1025800008D2284600F087F90028F0D1204600F054
:1025900003F8D9E72046D8E7F8B501460D464C794F
:1025A000601E002200E0521C2D688242FBD30026F0
:1025B00005E00F68284600F09BF93946761CA642D4
:1025C000F7D3F1BD0121001D00F0ACB81CB50446E5
:1025D0000121201D00F0B2F800909DF8000018B90C
:1025E0002046BDE81640D7E713BD2DE9F0470400AB
:1025F000894690461E46DFF8C4A003D15146B62056
:10260000FFF782F9E588607945432D1FAE422746E2
:1026100003D35146C420FFF777F94246B4F8068049
:1026200014683319311D9D42B1FBF8F038BFAC1B63
:1026300008FB10111460002801E03F68401EFCD127
:102640000025A8EB0100A246844288BF8246089E6E
:10265000084614E03844001D09EB050331005246DA
:102660000EBF194601461846FFF776F90020A4EB85
:102670000A0455443F68A246444588BFC246002C20
:10268000E8D1BDE8F0873EB51446002500F018F803
:102690000198A04203D00949F620FFF735F937BD6C
:1026A0003EB51446012500F00BF80198A04204D075
:1026B00002494FF48070FFF727F937BDACDF000007
:1026C0000194009501AA90E7806800218160016172
:1026D0004161C1604160016070472E0010B5024643
:1026E00052E8000F0C4642E8004393F0000FF7D188
:1026F00010BD000010B5024652E8004F44EA010048
:1027000042E8000393F0000FF6D110BD10B5024669
:1027100052E8000F00EA010442E8004393F0000F82
:10272000F6D110BD10B5024652E8004F04EB01008F
:1027300042E8000393F0000FF6D110BD10B5024639
:1027400052E8004FA4EB010042E8000393F0000FB1
:10275000F6D110BD10B5024652E8004F8C422CBF96
:10276000601A204642E8000393F0000FF4D110BD38
:102770000121BFE70021C9E710B5040003D11C49BE
:102780003120FFF7C1F8A2682AB121682069636986
:1027900098470020A06010BD0CB47CB504000D4625
:1027A000134E03D131464220FFF7AEF8606918B9E5
:1027B00031464320FFF7A8F8206818B93146442075
:1027C000FFF7A2F8606818B931464520FFF79CF87A
:1027D00055B100BF07A10A68009206AB00936A4694
:1027E0002946204600F015F973BC5DF80CFB00008B
:1027F0006CE300000000000010B5044600F075FA1C
:10280000014620460969BDE81040084710B5044656
:1028100000F06BFA01462046C969BDE81040084740
:1028200038B5040001D10E2032BD2068444D18B9DE
:102830002946FF20FFF768F8606820B929464FF461
:102840008070FFF761F8A06820B9294640F20110B6
:10285000FFF75AF8E06820B929464FF48170FFF776
:1028600053F8208A20B9294640F20310FFF74CF8AC
:1028700022686168A0681160401A03E00A68531C6E
:102880000B6010700246501ED2B22168002AF5D1AA
:102890000020087132BD70B50400294E04D13146C4
:1028A0004FF49270FFF730F80020FFF768F82068C7
:1028B0006268016800258A4215D2491E01600D78C0
:1028C0001CB93146E820FFF71FF8208AE168A268AA
:1028D0004543206803790D440168511AC9B29942F1
:1028E00038BF194601710020FFF758F8284670BD1F
:1028F000F8B504000D46124F04D1394640F2471096
:10290000FFF702F825B939464FF4A470FEF7FCFF33
:102910000020FFF734F820680668711C01601CB9BC
:102920003946F520FEF7F0FFE068218A2D1AB5FB45
:10293000F1F131700020BDE8F240FFF72FB8000040
:1029400068DF000038B50D4604460A2D04BF0D218E
:10295000FFF7F8FFA068411CA16022681554606869
:10296000814204D32046BDE83240FFF705BF31BDA8
:102970002DE9F84F8B460124154602E0B1FBF5F135
:10298000641CA942FAD29A460B9FD146A24538BF91
:10299000A14680460A9CF8070CD45CB1B8070CD459
:1029A0002026A14506D231464046FFF7CBFF641EE4
:1029B000002CF6D12E46012507E0BAF1000FEFD129
:1029C0003026EEE7AAF1010A7543BAF1010FF9D8F2
:1029D000BBFBF5F0B04228BF7543F9D2AFA1BBFBFA
:1029E000F5F005FB10BB095C4046FFF7ABFFB5FBFC
:1029F000F6F5002DF2D1F80709D544B1A14506D26C
:102A000020214046FFF79EFF641E002CF6D1BDE852
:102A1000F18F2DE9FE4F5FEA00090F461646984CEC
:102A200004D1214640F25220FEF76EFFD9F814007F
:102A300020B921464FF41570FEF766FFD9F8000063
:102A400020B9214640F25520FEF75EFFD9F8040078
:102A500020B9214640F25620FEF756FF002F00F025
:102A60000C8117F8010B002800F0FF80252840F0AA
:102A7000F580002502E045F001057F1C39782B29FF
:102A800007D02D29F7D0302908BF45F00205F4D032
:102A900002E045F00405F0E700240A2007E0397859
:102AA000A1F130020A2A0AD27F1C00FB04242A2941
:102AB000F5D1316851F8042B316014197F1C397835
:102AC0002E294FF000080BD17F1C04E0303900FBA9
:102AD00008117F1C88463978A1F130020A2AF5D303
:102AE000397801E017F8011F6C2918BF6829F9D05F
:102AF000252905F0010016D0582964D063290DD08E
:102B0000642918BF69290FD0702900F08E807329BD
:102B10005DD0752953D0782955D09DE0306850F8A4
:102B2000041B3060C9B295E0316851F804AB3160E4
:102B30005146002948BF494201220A2302E091FB85
:102B4000F3F1521C0A29FADAC346904538BF93467E
:102B50002CB1BAF1000F01D4690700D5641EA90792
:102B600002D5B8F1000F08D038B934B1A34504D26A
:102B700000F090F8641E002CF8D1BAF1000F03D5D4
:102B8000CAF1000A2D2102E0680702D52B2100F0CE
:102B900082F805F00300022808BFB8F1000F08D141
:102BA0003CB1A34505D2302100F075F8641E002C1D
:102BB000F7D10195009443460A22514646E000F0C1
:102BC00061F80A2242E000F05DF810223EE0316830
:102BD00051F8048B3160002140B9B8F1000F03D0E7
:102BE000404600F0C1F801460D4613E08B4603E075
:102BF00000F051F80BF1010B18F8011B0800F7D198
:102C0000A34529D244B300F045F8641EF8E700F06C
:102C100041F8641EA54201D2002CF8D118F8011B1E
:102C2000080019D000F037F8F8E7306850F8044B86
:102C30003060302100F02FF8782100F02CF80821C6
:102C40000091002001900823102221464846FFF7FA
:102C50008FFE01E000F01FF87F1C02E0014600F04B
:102C60001AF8387800287FF4FCAE99F80C0020B1EF
:102C70004846BDE8FE4FFFF77FBDBDE8F78F000077
:102C8000B0E10000306850F8041B306001950094FA
:102C9000434670472021484654E600003031323325
:102CA000343536373839414243444546613807E0C8
:102CB00005E0A0F161011A2901D2012070474138D5
:102CC0001A288041C00F7047A0F121010F290AD3B3
:102CD000A0F13A02062A06D9A0F15B01062902D327
:102CE0007B380428EDE7012070471D48704770B419
:102CF0005368D41801E05B1C491E042B08DA002934
:102D00001FBF057804F8015B10F8016B002EF2D1AB
:102D1000536070BC704738B514461D4661B1FFF76B
:102D2000E6FF61686A6B204690476FF00102811AE6
:102D300002D0491E01D001E003E005E000216160FE
:102D400032BD6FF0010032BD4FF0FF3032BDDA6BA3
:102D50001047034BDFE7024BF9E7024870470000DA
:102D6000D00700209807002000F1010310F8011B94
:102D700011B110F8011BFBE7C01A704741780078C9
:102D800007E0C178827842EA01224178007841EA7E
:102D9000022140EA012070470170090A4170704722
:102DA0000170090A4170090A8170090AC1707047EF
:102DB0002AB111F8013B00F8013B521EF9D17047CE
:102DC000521E00F8011BFBD17047F8B505460024E0
:102DD000E878A0B1EE6A00F014F808B101240EE022
:102DE000E870296AA869711A814208D2AF7804E0B4
:102DF000A869861900F005F87F1E012FF8D8204633
:102E0000F2BD68780123324605F1300101F001BCC2
:102E100070B504460D46E06A0026854210D0204673
:102E2000FFF7D3FF06000BD1607801232A4604F197
:102E3000300101F0A8FB10B14FF0FF350126E5622B
:102E4000304670BD38B50446FFF7BFFF05003AD1E4
:102E50002078032804BF207901282DD14FF4007277
:102E6000002104F13000FFF7ABFF4AF6552104F2D0
:102E70002E20FFF791FFDFF8301B04F13000FFF741
:102E80008FFFDFF8281B04F50570FFF789FF216924
:102E900004F50670FFF784FFE16804F50770FFF79B
:102EA0007FFFE2696078521CE262012304F1300185
:102EB00001F0AFFB0020207100226078002101F0BA
:102EC0000BFC00B10125284632BD4269891E921EC5
:102ED000914201D3002070474289806A02FB0101C0
:102EE000084670472DE9F0410C460568022C47D38F
:102EF0006869844244D2297801294FF0FF3604D012
:102F00003ED303292CD01CD33AE0296A04EB5407A2
:102F100000F081FA002834D100F0AAF810F80180FE
:102F2000296A00F078FA60BB05F13000C7F30807A2
:102F3000C15D48EA0126E00754BFC6F30B06360917
:102F40001FE0296A01EB142100F067FAC8B905F106
:102F50003000240600EBD450FFF710FF064610E0C7
:102F6000296A01EBD41100F058FA50B905F130008C
:102F7000640600EBD450FFF704FF20F0704600E039
:102F800001263046BDE8F0812DE9F0410E46022EC3
:102F9000054614464FF0020867D36869864264D23A
:102FA0002978012904D060D3032943D031D35CE0D0
:102FB000296A06EB560700F02EFA5FEA000854D1A2
:102FC00000F056F80844F20743BF017801F00F0102
:102FD00041EA0411214601700120E8702846296A5F
:102FE00001EB5721FFF714FF5FEA00083DD105F11F
:102FF0003000C7F30807C019F10748BF240906D4F9
:103000000178240A01F0F00104F00F040C4304706D
:1030100029E0296A01EB162100F0FFF95FEA0008B8
:1030200023D105F130003606A1B200EBD650FFF7F0
:10303000B3FE18E0296A01EBD61100F0EEF95FEA61
:10304000000812D105F13000760600EBD656304666
:10305000FFF797FE24F0704400F0704040EA04014E
:103060003046FFF79DFE0120E8704046BDE8F08144
:1030700005F13000C7F308017F1C7047F8B505461D
:103080000F462E68012F114629D97069874226D232
:1030900029B14FF0FF3200F078F801001ED1394617
:1030A0002846FFF71FFF040017D0012C17D014F19A
:1030B000010F16D0002200F067F801000ED17069F0
:1030C0003169821E914205D2491C3161317941F04A
:1030D0000101317127468742E1D30020F2BD022071
:1030E000F2BD0120F2BD2DE9F04180460C00D8F878
:1030F000006006D1F56815B1706985420ED30125CF
:103100000CE0FFF7EFFE012898BF01203AD910F13B
:10311000010F37D07169884234D325462F46706934
:103120007F1C874202D30227012D0BD93946404626
:10313000FFF7D8FE40B1012818BF10F1010F21D0D0
:10314000AF42ECD100201DE04FF0FF3200F01CF840
:1031500090B924B13A46214600F017F860B9F760FB
:1031600071693069891E88423CBF401E30613079E8
:1031700040F00100307104E001280CBF4FF0FF3730
:1031800001273846BDE8F08139463046FCE62DE996
:10319000F04105460E462F68B6F5001F2DD216F0F9
:1031A0001F0F2AD1AC682E6154B93878032801DB8F
:1031B0007C6A2CB93989700988421ED2786A18E075
:1031C000B7F80A8006E0022C17D37869844214D23B
:1031D000A6EB4826B6EB482F214608D32846FFF732
:1031E00081FE044614F1010FEDD1012011E000F041
:1031F00083F8A8616C61A86908B9022009E000EBB6
:103200005620A861C6F30806B81900F13001E9613B
:103210000020BDE8F0812DE9F04106460C463569F5
:103220003768B069203510B3B5F5001F1FD2E90526
:1032300057D1401C7169B06121B939896809884248
:103240004FD312E07889401E10EA552F49D13046FD
:10325000FFF748FE8046B8F1010F16D918F1010FAB
:1032600035D07869804537D31CB90020B06104207F
:103270003FE071693046FFF736FF5FEA000808BF9C
:10328000072036D0B8F1010F01D1022031E018F14A
:10329000010F1CD03846FFF798FDC0B94FF40072FB
:1032A000002107F13000FFF78BFD00F024F8002427
:1032B00002E0F86A641C401CF8627889844208D2F3
:1032C0000121F9703846FFF780FD0028F1D0012078
:1032D0000FE0F86A041BFC62C6F8148000F00BF8DB
:1032E000B061356107F13000C5F308054119F1619E
:1032F0000020BDE8F08141463846E6E570B5044659
:103300000D4605F11A00FFF739FD2178032906461D
:1033100005D105F11400FFF731FD46EA00463046BD
:1033200070BD70B504460D461646B1B205F11A00DF
:10333000FFF732FD2178032905D1310C05F1140086
:10334000BDE8704028E570BD70B504460D4626689E
:103350000422A169F1B13046FFF75AFD020019D1EC
:10336000E1690878D8B1C97AE52801F03F011CBFAE
:103370002E280F29A17107D021F02001082914BFA0
:1033800000200120A8420CD000212046FFF743FF77
:103390000200DED0100004D00020A06101E0042271
:1033A000FAE7104670BDF8B5054600212C68FFF716
:1033B000EEFE070015D10026A9692046FFF728FD7B
:1033C00007000ED1E8690078E5281CBF0028002618
:1033D00002D1761C012E07D0012100F028F9070048
:1033E000EAD0042F08BF0727380012D1A969204668
:1033F000FFF70EFD07000CD1E86920220021FFF73E
:10340000DFFCE8690B2205F12001FFF7D1FC012068
:10341000E0703846F2BD01EB57212846F8E470B55C
:103420000C46054600216172A86948B3002004F1EA
:103430000906EA69525C491C202A0BD0052A08BFFC
:10344000E522092902D12E233354401C04F109033B
:103450001A54401C0B29ECD304F109020021115429
:10346000E869C17A2172EA6902F11C00FFF789FC60
:103470002060E8691630FFF784FCE080000CA08033
:1034800070BD2DE9F04105460C46D5F8008000E0FE
:10349000641C20782F2818BF5C28F9D00020A86071
:1034A0002178202930D2802285F82B2000F0C8FC1A
:1034B0000246AFE095F82000E52804BF052185F815
:1034C0002010202FCCBF0020042085F82B000021E5
:1034D0002E6800F0B6FC020000F08B8095F82B00FF
:1034E000110040F092804007E3D4A979C80640F16A
:1034F00090802969C1F3080108EB010000F1300157
:103500004046FFF7FBFEA8600B22202105F12000BA
:10351000FFF756FC0021002208230FF2001C10E0E8
:10352000761C3078002818BFB842F9D1002844D161
:10353000A7F161061A2E05F1200038BF203F47543D
:103540007146A75C521C202F33DD2F2F18BF5C2F34
:103550002AD02E2F22D099422FD2A7F181001F28E6
:1035600022BFA7F1E0061D2E664601F1010ED8D25A
:10357000A05C521CA0F140063F2E27BFA0F18006A0
:103580007D2E5E1EB14218D205F12006775405F15A
:1035900020070EF1010107F80E00D2E70B2B0CD02B
:1035A00008210B23CDE7521CA05C2F2818BF5C28F4
:1035B000F9D0002914447FF47DAF06222AE0C87AAE
:1035C000EB6900F03F00A871D87A01070DD405F12E
:1035D000200C0B2113F8017B1CF8010B381A491E33
:1035E00001D00028F6D000280ED000F01FF802000D
:1035F0000AD1A9693046FFF70BFC020004D1E96942
:1036000008780028DBD1042268E7042A02D14007A9
:1036100000D405221046BDE8F0810000222A2B2CA0
:103620003A3B3C3D3E3F5B5D7C7F000000212846ED
:10363000F1E503464FF0FF301A68002A00D17047C9
:1036400010B5144600E0641C2178212901D33A29E1
:10365000F9D13A290CD112F8011B30390A2908D2C4
:10366000A24208BF002904D1611C0020196010BDCE
:10367000002010BD10B5044600224FF0FF33E27069
:10368000E362FFF7C5FB08B1042010BD04F22E2051
:10369000FFF774FB4AF65521884201D0032010BD84
:1036A00004F130000178E92904D0EB2904BF8078C7
:1036B000902813D104F16600FFF763FB20F07F40F0
:1036C000DFF89C16884207D004F18200FFF759FB0F
:1036D000DFF89016884201D1002010BD022010BDF5
:1036E0002DE9FF410E46002131601446FFF7A1FF8E
:1036F000070048BF0B2007D4DFF86C8608F10400F0
:1037000050F827500DB90C2008E1356004F0FE0494
:10371000287848B1687800F022FFC10704D4002C53
:1037200001D040070DD4F8E0002028706F70687851
:1037300000F082FEC10748BF032003D41CB140073C
:1037400001D50A20EAE000212846FFF793FF002672
:1037500002281ED1002405EB041101F5F771087948
:1037600018B101F10800FFF70CFB4DF82400641CB0
:10377000042CF0D35DF8264024B121462846FFF7FB
:1037800079FF00E00320022802DB761C042EF1D32F
:103790002646042808BF0120D4D0022880F2818068
:1037A00005F13B00FFF7EAFAB0F5007F79D105F1AA
:1037B0004600FFF7E3FA040004D105F15400FFF7D7
:1037C000E0FA044605F13D00AC61C178A970012919
:1037D00018BF022965D14C4300786881010060D090
:1037E000421E10425DD105F14100FFF7C7FA10F00B
:1037F0000F0F288155D105F14300FFF7BFFA0700ED
:1038000004D105F15000FFF7BCFA074605F13E0070
:10381000FFF7B4FA002844D02989231803EB1113C9
:103820009F423ED36A89FF1AB7FBF2F2002A38D0D2
:1038300003274FF6F67C624538BF022740F6F67C38
:10384000624538BF0127921C6A61EE6180199B199D
:10385000032F2862AB6210D105F15A00FFF78EFAF0
:10386000002804BF288900281BD105F15C00FFF760
:1038700088FA6862686980000DE091B1286A2418AE
:1038800068696C62022F0FBF400000EB400100F03E
:10389000010000EB5100A96900F2FF10B1EB502FBD
:1038A00001D20D203AE04FF0FF302861E86080201F
:1038B000032F28712AD105F16000FFF75FFA012874
:1038C00024D1711CFFF7A9FD00BB287105F22E2041
:1038D000FFF754FA4AF65521884217D105F1300016
:1038E000FFF74FFA3049884210D105F50570FFF710
:1038F00048FA2E49884209D105F50670FFF741FACA
:10390000286105F50770FFF73CFAE8602F70B8F8FA
:103910000000401CA8F80000E880002004B0BDE8CA
:10392000F08138B504000D461CBF216800290AD07B
:10393000087840B1C888A288904204D1487800F045
:103940000EFEC00702D50021092001E021680020F9
:10395000296032BD13B582B0144600916846FFF766
:1039600068FE002848BF0B201CD4DFF8FC1301EBD5
:103970008001486808B100220270029810B9002244
:103980004A6008E0029A00201070029B4B60029887
:1039900008B1012C01D0002004E0002202A903A8F4
:1039A000FFF79EFE04B010BD525261417272416138
:1039B0002DE9F34104008CB008BF092000F0D3804A
:1039C00002F03F073A4669460DA8FFF789FE060058
:1039D00053D100980D99019001A8FFF752FD060000
:1039E00004D19DF82F00010648BF062617F01C0FD2
:1039F00000F09380300000F08680042E3DD101A8B5
:103A0000FFF7D1FC0646300047F0080734D13807ED
:103A100038D50898DFF8405429460E30FFF7C0F932
:103A2000089829461630FFF7BBF908992020C8727C
:103A3000DDF8208000984146FFF760FC05460098BD
:103A400000224146FFF76DFC089800211C30FFF76B
:103A5000A7F900990120C87085B10098D0F82C8092
:103A600000F0FCF9060007D100984146FFF7D0F9B5
:103A7000064600986D1EC560300071D1380748BFFA
:103A800047F040070098C16A216208986062089D6B
:103A900000982946FFF732FCA06005F11C00FFF7F3
:103AA00070F9E0604FF40072009820600099C888B7
:103AB000A08000216174E1616161277404F1280034
:103AC000FFF77EF9B8064DD5E568002D4AD065614F
:103AD00000984789A1687F02AF420CD22046FFF7C9
:103AE00001FA0146022926D311F1010F26D0ED1B60
:103AF0003000F1D020E0E805A16133D000F0EEF80D
:103B000008BB02262CE09DF80A0010F0110F10D11E
:103B100078077FF57CAF082622E03000ACD19DF815
:103B20000A00C10648BF04261AD4B907A6D5C007A3
:103B3000A4D5072614E00226A16111E04FF0FF3062
:103B40000126A0610CE000EB5520E06102460098E0
:103B50004078012304F1280100F015FD10B1012681
:103B60000020206030460EB0BDE8F0812DE9FC4712
:103B7000144600F0A9F800F0ADF8010001D1787CFE
:103B8000010040F09F80387C810758BF072040F13A
:103B9000998078692118814235D24FF0FF32141A8A
:103BA00031E0660A05EB00085DD000984089711984
:103BB000884238BF461B00984078334642465146FB
:103BC00000F027FD002875D1F869A0EB0800B0428D
:103BD00009D20AEB40214FF4007207F12800FFF7E9
:103BE000E7F800F0D2F87602B244786930187861CC
:103BF000F968884238BF0846F860A41BD9F800006D
:103C00003018C9F80000002C57D07869C1053CD1A4
:103C100000994D896D1E15EA502513D118B9B86861
:103C200028B9002100E0B9693846FFF75CFA00289E
:103C300043D0012815D010F1010F3BD0B861B9680D
:103C400001B9B860387C010606D50098FA6900F021
:103C5000A1F878BB00F099F8B96900F03FF80100CD
:103C60009FD1022027E0F86940450CD07969F868B7
:103C7000814208D2009840780123424607F128018A
:103C800000F081FCB0B9C7F81C807B69C3F308035E
:103C9000C3F500702646844288BF064607F1280017
:103CA000324651461844FFF783F8387C40F08000D4
:103CB000387499E70120787404E0387C40F04000C3
:103CC00038740020BDE8F687994600228A46C9F874
:103CD000002070470746694623E601460098FFF733
:103CE000F4B838B500F08CF8010037D1217C4A06D1
:103CF00034D5080608D500F0A7F808B1012032BD78
:103D0000207C00F07F002074216A0098FFF780F883
:103D1000010023D1656AE87A40F02000E872294664
:103D2000A2682068FFF7FDFAE16805F11C00FFF7C3
:103D300037F8DFF8DC1505F11600FFF731F8002140
:103D400005F11200FFF728F800990120C8700098CB
:103D5000FFF778F8217C01F0BF01217432BD00002B
:103D60004641540046415433202C00201CB50446E3
:103D7000FFF7B7FF010007D169462046FFF7D1FDE5
:103D8000010004BF0021216016BD387C00F07F00D7
:103D9000387470474078012307F1280100F039BCDE
:103DA00013B5040001D1092016BD0022694601A8FF
:103DB000FFF796FC01001ED1009820602046019973
:103DC000FFF75FFB010012D194F82B00010607D426
:103DD000A079C1060DD5E1690098FFF78FFAA060C0
:103DE0000098C188A18020460021FFF7D0F904285F
:103DF00001D1052001E0010001D00021216016BDA4
:103E0000044669468DE538B50C460546FFF763FF65
:103E1000010014D114B900F013F832BD0021284676
:103E2000FFF792FA042801D0010008D12146284664
:103E3000FFF7F5FAFFF7FAFB042808BF002032BDB0
:103E400000212846FFF7A3B90098E26940780123D2
:103E500004F1280100F0DDBB0000214800222946C2
:103E600001A8FFF70BB900002DE9F94F87B00D4607
:103E7000144607A8FFF7DDFB010048BF0B2062D402
:103E8000DFF8900450F8210008B1002202708DF88C
:103E900000109DF8000000F0CFFAC10748BF0320D2
:103EA00051D4400748BF0A204DD49DF8000002AA13
:103EB000032100F011FC40B9029830B148F2010131
:103EC000884202D2411E084201D0012002902CB14A
:103ED000A4F50070DFF84014884233D2621E144209
:103EE00030D11298400A0390640A4002059050D0E5
:103EF0009DF8000001AA012100F0EEFB002840F02F
:103F00000382290701988DF801504CBF4FF000093A
:103F10004FF03F09484522BFA0EB090101918029DC
:103F200037D3802C0ED815F0020040F6F67207D079
:103F300005F00701022900F08680EB0740F183803D
:103F4000EB0701D41320E0E1022625002AD1019BD2
:103F50000FF244471B0B4FF0000801251DE008F14C
:103F600001086D0037F8181009B18B42F7D201999A
:103F7000B1FBF5F39F00DFF8A41307F20727CB1876
:103F80007F0ADFF89C138B424FF0200A4FF00008A5
:103F90001DD36EE008F101086D0037F8181009B163
:103FA0008B42F7D20199B1FBF5F7974202D37F001C
:103FB0003F1D05E007EB47077F1C7F080126FF1C1C
:103FC00007F2FF177F0A4FF0010A4FF020080AEBB3
:103FD000090104917918DDF808C0029B41448C4422
:103FE000ACF1010C5B1E2CEA03035B1A032E05D116
:103FF000DDF810E09A447344049300E0DF19019B5C
:1040000001EB0511A1EB09018B4232D3A3EB0A01AD
:10401000C91BA1EB0801B1FBF5FB032E4FF6F671AE
:1040200006D18B4527D224BB6C0822D025469EE7BB
:10403000022E1AD16B008B4510D31CB9412B38BF0F
:104040001C4682D360B10326250090D1019B0FF25C
:1040500058375B0C4FF00008012583E793450AD2DF
:104060003CB91C46802C04D86FE7012E03D1934540
:1040700001D30E2049E1089C00F06AF95FF00B02C1
:10408000B8A12046FEF794FE4FF4007104F10B0036
:10409000FEF782FE65731FFA8AF104F10E00FEF747
:1040A0007BFE01202074032E0CBF00214FF4007111
:1040B00004F11100FEF770FE0198B0F5803F014653
:1040C00005D289B204F11300FEF766FE03E004F1A5
:1040D0002000FEF765FEF82060753F2104F118000E
:1040E000FEF75AFEFF2104F11A00FEF755FE49467D
:1040F00004F11C00FEF754FE032E04F1240A844947
:1041000022D104F14300FEF74BFE39465046FEF73C
:1041100047FE022104F12C00FEF742FE012104F1CA
:104120003000FEF739FE062104F13200FEF734FEBE
:10413000802029218AF81C008AF81E105FF01302E3
:104140008BA104F1470012E004F12700FEF728FEDE
:10415000B9B204F11600FEF71FFE802029218AF86B
:1041600000008AF80210132286A104F12B00FEF74A
:104170001FFE00F0E1F800F0DBF84A4600F0EEF830
:10418000002859D1032E29D100F0D2F809F10602F6
:1041900000F0E4F800F0DCF862492046FEF700FE8B
:1041A000614904F5F270FEF7FBFDABF1010104F586
:1041B000F470FEF7F5FD022104F5F670FEF7F0FD50
:1041C00000F0BAF800F0B4F809F1070200F0C6F800
:1041D00000F0AEF809F1010200F0C0F8059A0021E4
:1041E0002046FEF7EDFDDDF810A0032E6FF007016D
:1041F0000CD12046FEF7D4FD4FF0FF31201DFEF715
:10420000CFFD6FF0704104F1080003E0012E08BFFC
:1042100046492046FEF7C4FD384627460446DDF8E9
:104220000CB09DF80000A34588BFA3465B465246EC
:10423000394600F0EEF9002866D100F083F8B4EBBF
:104240000B00DA440446EAD19DF800400398032E9F
:1042500015D18046C346A84588BFAB465B4652464B
:104260003946204600F0D5F900284DD1B5EB0B00BA
:10427000DA440546EED1032E03D10C250BE045466A
:10428000E7E70198B0F5803F28BF062503D2022E4C
:104290000CBF042501259DF8010001072ED400F074
:1042A00051F84AF6552107F5FF70FEF775FD07F541
:1042B000DF71002008700122C8704A708A700D7189
:1042C00043F6C16201984844B0FBF2F08508FE2332
:1042D00045F03F054B718D71C871494607F5E37094
:1042E000FEF75EFD019907F5E570FEF759FD012324
:1042F00000223946204600F08CF928B9002200211E
:10430000204600F0E9F900B1012009B0BDE8F08FC6
:1043100000002148242C002001FEFF000A00FFFFBE
:104320000000FF0F5252614172724161F8FFFF00BD
:104330009DF80000012370474AF6552104F5FF70EF
:10434000FEF72ABD4FF4007200213846FEF738BD53
:104350004FF4007200212046FEF732BD214600F0E6
:1043600058B90000EBFE904D53444F53352E3000AA
:104370004E4F204E414D452020202046415433329F
:10438000202020004E4F204E414D45202020204629
:104390004154202020202000010004001000400093
:1043A00000010002000000000100020004000800FB
:1043B000100020000000000070B504460D46216882
:1043C0000869164628B9DFF8A8134FF4A370FDF763
:1043D0009BFA236820461C6932462946A04770BDD7
:1043E00010B504462168486928B9DFF884134FF4F2
:1043F000AA70FDF789FA21684A692046BDE8104095
:10440000104770B50C46DFF86C63257A307885422A
:1044100004DBDFF864133F20FDF776FA21780329E7
:1044200007D8736861780C2045435819002201723F
:10443000827270BD20BF70472DE9F041DFF8344330
:10444000DFF82C638046606820B906F18C015920A2
:10445000FDF75AFA2278904506D245460C214D4385
:1044600061684A19106808B9032031E001F10900B8
:10447000435DD90758BF405D2AD5506810B9DFF8B1
:10448000FC1251600120907217683968086818B9E9
:104490003146F020FDF738FA3B68B9491E684246BC
:1044A0003846B04780B901E04868804762685119D2
:1044B000887A0028F8D1087A30B902F10901093266
:1044C000485D00F0FE005055606800F10901485D4C
:1044D000BDE8F081F8B5A74DA54E0446686820B93F
:1044E00006F18C018620FDF70FFA29788C4204D260
:1044F0000C2069684443085908B90320F2BD01F152
:104500000902135DDF0703D501F10900005DF2BD6B
:1045100000220021FFF750FF686807593968486892
:1045200018B93146FD20FDF7EFF939684A68384679
:1045300090471128F0D040B902E0081D0159884782
:1045400069680A19907A0028F7D169682144087AC5
:1045500018B9487A40F001004872487AF2BD38B57F
:10456000844D0446686818B98349B320FDF7CCF937
:1045700029788C4201D3012032BD69680C20444364
:104580000819407A32BD2DE9FE4300F096F820B9B3
:1045900008F18C01BE20FDF7B7F929788E4200D2D0
:1045A0000CB9042027E000F091F810B1487AC20756
:1045B00001D503201FE000F077F8886820B9414654
:1045C0004FF48970FDF7A0F92168486920B9414688
:1045D00040F21310FDF798F921684A692046904788
:1045E00000990068814205D2226893686946204696
:1045F000984728B10120BDE8FE83081D81598847EE
:1046000069688A19907A0028F7D1107A0028F1D1C8
:10461000F1E72DE9FE4300F050F820B908F18C01D4
:10462000E520FDF771F929788E4200D20CB90420FB
:104630002CE000F04BF810B1487AC20701D50320F6
:1046400024E0487A420748BF02201FD400F02CF82B
:10465000C86820B941464FF49770FDF755F92168B5
:10466000486920B9414640F22F10FDF74DF9216805
:104670004A692046904700990068814205D2226825
:10468000D36869462046984728B10120BDE8FE83DB
:10469000081D8159884769688A19907A0028F7D1DE
:1046A000107A0028F1D1F1E7CDF80090019402973B
:1046B00001228A720C68216870472E4DDFF8B080A5
:1046C000064668680F4691461C4670470C216A688A
:1046D0004E43911908687047F8B5264E0546706834
:1046E0000F46144620B924494FF48870FDF70CF9A1
:1046F00031788D4201D30420F2BD0C20454370680F
:104700001FB1022F1AD012D322E001208DF8000031
:10471000706840596A460021FFF74EFE002818BF16
:10472000112813D19DF800000028F1D10EE0405966
:1047300030B1FFF755FE0068206007E0405908B926
:104740000320F2BDFFF74CFE406820800020F2BD40
:104750000120F2BD38B504000D4604D106494FF4DE
:10476000A470FDF7D1F803484460057031BD000026
:10477000C0CE0000182C00204CCF000035440000B3
:10478000034400000178407840EA01207047014668
:1047900008784A788B78C97840EA022040EA0340DA
:1047A00040EA01607047014648780A78000440EA10
:1047B00002608A78C97840EA02200843704700BA4C
:1047C000086004207047C0F341107047007A7047BA
:1047D00038B504000D4605D1DFF864164FF4887033
:1047E000FDF792F82046FFF7F1FF854201D3002044
:1047F00032BD05EB45056019093032BD4078704780
:1048000038B504000D4605D1DFF8341640F24310E8
:10481000FDF77AF861788D4201D3002032BDA0788F
:104820002044284432BD0078704770B504460D46D8
:1048300021680869164628B9DFF808164FF4A370F6
:10484000FDF762F8236820461C6932462946A047D6
:1048500070BD10B504462168486928B9DFF8E41531
:104860004FF4AA70FDF750F821684A692046BDE868
:104870001040104710B5040004D1DFF8CC1581209A
:10488000FDF742F8204610BD38B50400DFF8B855F2
:1048900003D129468D20FDF737F8216819B929463B
:1048A0008E20FDF731F820680C3032BD80B5002134
:1048B000FFF78EFF002104E080B50021FFF788FF9D
:1048C0000121FFF79DFFBDE80240ACE780B5FFF78F
:1048D000DBFF002100F8301F4170817001BD80B501
:1048E000FFF7D2FF90F8310000B1012002BD10B5F2
:1048F00000F040F8A16990F8320088428041C00F72
:1049000010BD70B500F036F800F036F82046FFF71D
:10491000EEFF002680B105F130018A78087883180F
:10492000A069B3FBF0F500FB153360692469DBB2C5
:104930004343521CE6188A7032E070B500F01AF852
:1049400000F01AF815F8310F6978DFF8FC64884236
:1049500004D3314640F21110FCF7D6FF2878A16944
:10496000884204D331464FF48970FCF7CDFF287894
:10497000401C3DE0044687E705460020FCF7FFBFEA
:1049800070B5FFF7F7FFFFF7F7FF2046FFF7A7FF28
:10499000002628B195F830206069216942438E18BD
:1049A0000020FCF7FBFF304670BD70B5FFF7E2FF5B
:1049B000FFF7E2FF3035DFF89064687820B93146C0
:1049C00040F24510FCF7A0FFA87820B931464FF41B
:1049D000A370FCF799FF6878411E6970A878411EA2
:1049E000A9702878A169401CB0FBF1F201FB12000C
:1049F00028700020BDE87040FCF7D0BFFEB505462A
:104A0000FFF738FFFFF740FF04462846FFF754FF43
:104A100005461F21601CFDF73FF800BF07A191E884
:104A20004C006846671C80E84C00009769462846A1
:104A300001F0DFFC08B902212170FEBD000000007A
:104A40001F00000000000000FEB506460D46FFF7FF
:104A500011FFFFF719FF04463046FFF727FF04F167
:104A6000280204F1280312695E6A04F12801B242A7
:104A700038BF32460A70170A130C120E4F708B7033
:104A8000CA700D714FEA0D0106A292E8680081E834
:104A9000680004F12007009701F0ABFC08B906217B
:104AA0002170FEBD000000000D00000000000000AD
:104AB0002DE9FF4180460F4615461C46FFF7DAFEFA
:104AC000FFF7E2FE06464046FFF7F0FE6A46002387
:104AD0009E46984682E8084100970195694601F094
:104AE00088FC00B9347031E1F8B504460D46FFF793
:104AF000C1FEFFF7C9FE06462046FFF7D7FE074670
:104B00002046FFF7D9FE04463846FCF7B3FD2046A1
:104B1000FCF7B0FD3846FBF720FE2046FBF71DFEF4
:104B20003570F1BD38B50446FFF7A4FEFFF7ACFEC3
:104B30000930FFF72CFE28B107212046FFF7D4FFEC
:104B4000002504E001212046FFF77EFF05462846A8
:104B500032BD0821C8E738B504460D46FFF794FE7C
:104B60006169406CA94288BF29464118491EB1FBC2
:104B7000F0F032BD4069814288BF01460846704767
:104B80002DE9F0410546FFF775FE0746FFF77CFE6D
:104B9000014601F12C060024307C002837D1707CBE
:104BA000A0BBB068DFF8C88AF8B13846FFF797FEB7
:104BB00068B33846FFF7E4FE0446B1683846FFF7AD
:104BC000D9FF074624B9414640F27E30FCF79CFEEF
:104BD0000120307404233A4621462846FFF768FF37
:104BE000040014D00020307411E0097804290ED19B
:104BF000F06858B931782846FFF726FF040006D040
:104C0000414640F28F30FCF77FFE00E0062420464C
:104C1000BDE8F0812DE9FE43FFF72CFE8046FFF74B
:104C200033FE064606F154050024287800284CD1AE
:104C3000687808B1062448E0B06C002845D04046AA
:104C4000FFF755FE002840D0D8F81C00B17B50F883
:104C50002170B16C4046FFF77EFF81464046FFF76A
:104C600050FE0400DFF8DC8105D108F18C0140F230
:104C7000AE30FCF749FE316D0091CDF804900294FE
:104C8000012129703A68906820B941464FF4897033
:104C9000FCF73AFE3968486920B9414640F21310E2
:104CA000FCF732FE39684A69384690470099006837
:104CB000814228BF072406D23A689368694638467D
:104CC0009847040001D0002028702046BDE8FE83EC
:104CD0002DE9FF410646FFF7CDFD0746FFF7D4FD5E
:104CE00000F134050024297A79BB286868B3384676
:104CF000FFF7FDFD48B33846FFF703FE0446296879
:104D00003846FFF737FF804624B94F494FF4747097
:104D1000FCF7FAFD0120287200F05AFEFFF7B4FDFF
:104D200007463046FFF7C8FD6946002200230026EB
:104D300081E84C000094CDF8048001F05AFB040097
:104D400004BF0520387004B12E72204604B0BDE8BF
:104D5000F0812DE9FE4F0746FFF78CFD8246FFF7F5
:104D600093FD83460BF1540500242878002863D175
:104D7000687800285FD10BF12C06DFF8C890F06945
:104D8000002809F18C0844D05046FFF7A8FD002800
:104D900052D0DAF81C009BF80E1050F82170F1691F
:104DA0005046FFF7D8FE83465046FFF7E9FD040062
:104DB00004D141464FF47D70FCF7A6FD716A009165
:104DC000CDF804B00294012129703A68D06820B966
:104DD00049464FF49770FCF797FD3968486920B948
:104DE000494640F22F10FCF78FFD39684A69384672
:104DF000904700990068814228BF072406D23A688C
:104E0000D368694638469847040015D000202870BA
:104E100012E09BF8001005290ED1306A58B931789C
:104E20003846FFF711FE040006D0414640F20C4020
:104E3000FCF76AFD00E006242046BDE8FE8F000076
:104E4000F4DC000010CD00009CCD0000F8B500F0AF
:104E500037F802B94CE0706920B104F10D073878D9
:104E6000020600D448E00846FFF730FD00F02EF8B7
:104E700000F034F8FFF7CEFE04001CBF2846FFF711
:104E800051FE2046F2BDF8B500F01AF802B92FE045
:104E9000706920B104F10D073878020600D52BE0C7
:104EA0000846FFF713FD00F011F800F017F8FFF7C0
:104EB0000FFF04001CBF2846FFF734FE2046F2BD5A
:104EC000144604F134060546B2697047B069716949
:104ED000884202D270610220F8777047B069716928
:104EE000706031600020307284F8540028467047AA
:104EF000BDE8F4400121A7E52846BDE8F24011E6EF
:104F0000002280F83C20426B8A4234BF0022521AB1
:104F10004263826B8A4234BF0021511A8163704719
:104F20002DE9FE4F5FEA0008DFF898598A4605F13F
:104F30008C0604D1314640F63F00FCF7E5FCBAF19F
:104F4000000F04D131464FF40460FCF7DDFC00F0A3
:104F5000CFFC8346FFF798FC81469AF800000024B6
:104F600001270E2800F2FD80DFE810F07F030F001C
:104F7000F5027F03FB001A00DC00FB00FB00FB00D6
:104F8000FB0004037F03190355030D21484601F07C
:104F9000FDFA0FF64820026809F120010A6064E377
:104FA000B8F1000F04D131464FF44870FCF7ACFC67
:104FB000BAF1000F04D1314640F22130FCF7A4FCD5
:104FC0009AF80100C109012951D1FFF7FCFB18B380
:104FD000012860D100F08CFC04469AF80200FE28FB
:104FE00001BFBAF803000028BAF80700012852D11F
:104FF000684601F052FE0546206A20B9314640F26B
:10500000CD20FCF781FC206A411E29804046FFF735
:10501000F5FC0122294625E09AF8010000F01F0066
:10502000012804BF9AF80200062834D1019402A88E
:1050300001F033FE044601A800909AF803209AF884
:1050400004102346404600F03AFD052800F0898010
:105050000198402804D3314640F25F20FCF754FC0D
:10506000019A21460AF1010001F0D9FDABE0FFF7FA
:10507000AAFB28B301280ED100F03AFCFFF704FC8C
:1050800005469AF80200FF2801BFBAF8030000287D
:10509000BAF80700002864D14046FFF707FC06462F
:1050A00000F012FB07463046FBF757FB3846FBF78C
:1050B00054FB2878022802D04046FFF79FFCD4E238
:1050C00000F016FCFFF7E0FB05469AF8010000F03F
:1050D0001F00022801BF9AF802000128BAF8030055
:1050E00000283ED12978082908BF0F24E7D09AF874
:1050F00005603046FCF70DFB3046FCF7CFFA300672
:10510000DDD52978072907D00929D8D100F0DCFAA4
:10511000FCF7C4FA022153E000F0D6FAFCF7BEFA1D
:1051200001214DE09AF80200010650D500F0E0FBA5
:10513000FFF7AAFB05469AF802006946FCF759FA00
:1051400000B100949AF8030000280BD12878C01E03
:1051500004283AD8DFE810F02F00070089028902FE
:105160000500062481E2009C00F0C2FB0546FFF723
:105170008BFB07462846796BFFF7FCFCA04204D066
:10518000314640F24B70FCF7BFFB21463846FFF733
:10519000B7FE2846FFF709FC4046FFF7F1FC040084
:1051A00003D14046FFF736FD0446002C02D04046AE
:1051B000FFF7B8FC59E2E96C0098091AE96400218C
:1051C0004046FFF741FC04464FE203244DE200F065
:1051D0008FFBFFF759FB07469AF8020001A9FCF77D
:1051E00008FA002500B101949AF8030001280AD1B9
:1051F0003878052851D0062818BF01284DD14046DF
:10520000FFF7FCFB9EE1032802D1012038702CE25D
:10521000397802280AD1052904D109214046FFF72F
:1052200063FC22E24046FFF794FC1EE2022935D0DF
:10523000052909D0062930D007291EBF314640F67E
:105240002D00FCF761FB83E1FFF797FB019C00F069
:105250004FFB0546FFF718FB06462846716BFFF724
:1052600089FCA0421CBF012086F85500214630462B
:10527000FFF746FE2846FFF760FB4046FFF728FD94
:10528000050003D14046FFF764FD054615B14046D1
:10529000FFF748FC0020FCF781FB5AE100F028FBF7
:1052A0000746FFF7F1FA0646282106F1300001F023
:1052B0006DF906F12400046000F006FA6946FCF777
:1052C00098F9002804BF00981F2806D104220FF285
:1052D0000871701C01F012FD002840F03581701D2E
:1052E00006F1240102680A6006F12C0406F10900A7
:1052F0002570B17B2175FFF74AFA2062217D386A5B
:1053000081425BD2317C002906F1580500F003810F
:10531000032900F0E18004294BD0082900F0CE8059
:105320000A2900F0BD80122971D015290ED01A2942
:105330005BD01B290AD01D2908D01E2906D025299B
:1053400035D0282928D02A291BD0552900F0ED80F6
:105350005A2940F0EC80F27B092A2AD9B17B81429C
:105360002CD200F0ADF9042828D800F0A9F90246A3
:1053700000200021C5E90001297006206870032380
:10538000C4E0F07B092814D900F094F900F081F909
:1053900000F08BF9A5618CE0F07B092809D900F0B9
:1053A00089F900F076F900F080F9A5618FE0F07BD3
:1053B000092840F2BF8000F083F9092880F0BA8004
:1053C00000F07EF9040008BF002100F0B88000F072
:1053D00071F9074629463868401EFFF7F0F97868EA
:1053E00006F15C01FFF7EBF98EE0F07B062859D35C
:1053F00000F066F9042874D800F062F90022032155
:105400006A70AA70EA702970024603237EE0B07CBD
:1054100008B100F08FB800F053F9252861D200F0F0
:105420004FF9040008BF002165D0002028708021BA
:1054300069701220E87006222021AA7029710020CC
:1054400000906A46F869B37B50F823000121FFF70A
:10545000ECF90098A0B10168082206F1600001F0A3
:105460005DFC00984168102206F1680001F056FCCE
:1054700000988168042206F1780001F04FFC43E0B7
:1054800006F1600000210022C0E9001206F1680068
:105490000023002780E88E0006F17800016033E0E9
:1054A000F07B062846D300F005F900F0F7F800F08D
:1054B000E9F800F0DFF8FFF7E6FC43E0F07B0628B0
:1054C00038D300F0F7F800F0E9F800F0DBF800F06E
:1054D000D1F8FFF7BBFC35E0F17B06292AD3B17B7D
:1054E000814227D200F0ECF8122823D800F0E8F827
:1054F000040008BF002122D01221284601F046F8FE
:10550000F0200B212870E9710323224629464046EA
:10551000FFF7CEFA16E000F0D3F858B9F07B062872
:1055200008D1B07B396A884204D2002107E000F03C
:10553000C7F818B14046FFF7F5FA03E001214046ED
:10554000FFF782FA054604E04046FFF702FB00E061
:1055500006252C4689E00025DBF820008542F9D29B
:10556000DBF81C0050F8250000220021FFF75DF950
:105570006D1CF1E70021032001F00CFC05000CD0AC
:105580002E7876080D2E08D335F8170001F020FC90
:1055900018B17F1CB742F7D367E0062066E0DBF85E
:1055A0002000112804D3314640F69800FCF7ACF9EE
:1055B000A246D846D8F82000824556D2D8F81C100A
:1055C00051F82AB0DBF80020106818B92946F020FD
:1055D000FCF79AF9DBF800300FF261311C684246A3
:1055E0005846A047040013D1B9F87C0007FA0AF125
:1055F0000843A9F87C005846FFF72BF9D8F8141097
:105600004068814204D2314640F6A500FCF77CF99F
:105610000AF1010ACEE7DBF82000112804D3314655
:1056200040F6AE00FCF770F94E46A14619E0DBF8F3
:105630001C0050F829402168486818B92946FD2007
:10564000FCF762F921684A6820469047040006D1B9
:10565000B6F87C0007FA09F18843A6F87C0009F146
:105660000109DBF820008145E1D32046BDE8FE8F2B
:105670009CCD0000606205FB09F5E56132463946C4
:1056800040467047717CA561090401F4F811084394
:105690007047456806F11700FFF774B8456896F83B
:1056A000149006F11200FFF76DB8814606F1120062
:1056B000FFF779B8F869B17B50F82100FFF7C9B856
:1056C00006F10900FFF763B84046FFF7F5B82DE98A
:1056D000F0470546884614469A4640467A4FFFF7FB
:1056E00075F8387000F004F9814625B9774940F61D
:1056F000D600FCF709F92868002609F1280948B303
:1057000040F6DD01401A32D0401E39D0401F46D04D
:10571000401E4CD0401E52D0401E59D0401E61D079
:10572000401E69D0401E6FD00B3800F07E80401EB6
:1057300000F08480001F00F09080401E00F09680F2
:10574000401E00F09C80401E00F0A180401E00F032
:10575000A680B2E07E7078783978884280F0A880A0
:10576000092256452A7128BF40F6DD0026D200F0F6
:10577000B3F804215645297128BF40F6DE001DD23A
:1057800000F0A6F840467978FFF722F87860761C9A
:1057900000782871564528BF40F6E3000ED200F08D
:1057A00097F800F0A8F828BF40F6E40006D200F011
:1057B00098F82871564528BF40F6E5007AD200F0E7
:1057C0008BF808215645297128BF40F6E60071D2B2
:1057D00000F082F899F800102971564528BF40F66C
:1057E000E70067D200F078F899F801002871564573
:1057F00002D340F6E80116E000F06AF800F07BF80A
:1058000028BF40F6E90055D200F06BF8B8700020D0
:10581000F870B978F878884246D207205645287142
:1058200003D340F6F401296045E000F055F8052166
:105830005645297128BF40F6F5003BD200F048F8E4
:10584000F9787868FEF7DCFFFEF7EDFF761C28712B
:10585000564528BF40F6F9002CD200F03DF8022151
:105860005645297128BF40F6FA0023D200F034F8DB
:1058700040215645297128BF40F6FB001AD200F09E
:1058800027F800F038F828BF40F6FC0012D200F0EC
:105890001FF800F030F828BF40F6FD000AD200F0F3
:1058A0001BF8F878401CB3E77878401C787052E712
:1058B00040F602102860012001E02E600020BDE8C3
:1058C000F087000010CD0000102C00209CCD0000BF
:1058D0000CB12879A05570470CB12879A055761CD9
:1058E00070470CB12879A055761C7868FEF786BF02
:1058F0004046FEF7BFBF761C002156452971704710
:1059000010B50C46A068FEF7B5FFFEF7BDFF616855
:105910004A68416C036D5143D2180265826C8A4219
:1059200034BF0022521A8264C26C8A4234BF002102
:10593000511AC164002180F8541010BD2DE9F041C6
:105940000D4604462978022902D003291DD03CE0E7
:10595000FFF713F800F03BF88046FEF795FF074687
:105960004046FEF7EAFF687820B929462046FFF74F
:10597000C7FF02E0012087F83D003046FFF700F93D
:10598000D0B93046FFF746F916E0FEF7F6FF00F013
:105990001EF8FFF70AF8687820B929462046FFF775
:1059A000AFFF02E03046FFF7BDF83046FFF790F951
:1059B00010B93046FFF7CDF910B13046FFF7B2F815
:1059C000BDE8F0410020FBF7E9BFBDE8F081AE681B
:1059D0003046FEF74FBF00005553424355534253E4
:1059E00080B5FBF70DFB002002BD007A704738B58B
:1059F00004000D4605D1DFF8DC184FF48870FBF782
:105A000083FF2046FFF7F1FF854201D3002032BD1E
:105A100005EB45056019093032BD38B504000D4667
:105A200005D1DFF8B01840F24310FBF76DFF617845
:105A30008D4201D3002032BDA0782044284432BDDD
:105A40000068704710B5040005D1DFF88C1840F2EB
:105A50004320FBF759FF2046FFF7F2FF006810BD17
:105A600070B504000D46DFF8746804D1314640F289
:105A70000F10FBF749FF606820B931464FF488707A
:105A8000FBF742FF6168086820B9314640F2111007
:105A9000FBF73AFF6268136829462046BDE870406C
:105AA0001847DFF83C281268002A18BF10477047D3
:105AB000DFF82C184968002918BF084770472DE9FE
:105AC000F04F85B005460020884692461F4601905B
:105AD000002400E0641CD5F804C0DCF80460012355
:105AE0000022294601A8B0470028F3D18DF8000014
:105AF00003904FF000090E9ECB460FE00BF1010B17
:105B0000D5F804C09DF80030DCF804C09B1E0022CC
:105B1000294603A8E0479DF800008144A14529D209
:105B200000F02AF86A46294603A8E04700F024F866
:105B30000DF10102294603A8E0479DF80100404508
:105B4000DED15FFA8BF05045D8D19DF8002032604D
:105B500029469DF80000387087F80180BA1C6C68EF
:105B60009DF8003065689B1E03A8A847002005B07B
:105B7000BDE8F08F0520FAE7D5F804C0DCF804C0D2
:105B80000123704710B500F00F040006DFF84C1732
:105B90000CD5092CA4BF4FF4CC70FBF7B5FEDFF891
:105BA000401701EBC40000F5C47010BD092CA4BF60
:105BB0004FF4CF70FBF7A8FEDFF8240700EBC40119
:105BC00001F1140010BD80B5FFF7DCFF006802BDD5
:105BD00070B505460C46FFF7D5FF0646346064B93C
:105BE000280018BF802D05D1DFF804174FF4E170AD
:105BF000FBF78AFE0020706070BD6068016871600C
:105C000070BDDFF8DC260146506992691047F8B58F
:105C10000646307805280AD1DFF814174868096865
:105C2000C9B2002902BFC0B205280FF2B806307809
:105C3000DFF8AC5688BB00F077FB0446DFF8B0769F
:105C400014E0206820B939464FF48D70FBF75CFEF4
:105C50002168886820B9394640F21B10FBF754FED2
:105C6000216870888A68904720684468002CE8D1D1
:105C70000020FBF784FEE86D08B9708828820121B6
:105C800005F15C00FCF74EFD0020FBF787FE0121CB
:105C90003046FFF706FFE86DF1BD05F5BC776946B4
:105CA000384601F0B9F804001AD0306820600020AE
:105CB000FBF765FE298AE86D091A491CE18005F1A8
:105CC0005C000021FCF70AFDA0800020FBF766FEC7
:105CD0006946384601F0C2F801463046FFF7E1FE5A
:105CE000F1BD00008500000018B1022806D003D3E2
:105CF00006E000BF05A002E005A000E005A086E7E1
:105D0000DFF8EC1540F26220FBF7FEBD0800000052
:105D1000090000000A00000079E7000080B528B102
:105D2000DFF8CC1540F27B20FBF7EEFDBDE802402A
:105D300000A06CE78000801E02D0C01E032801D89E
:105D40000120704700207047022818BF082801D1A1
:105D5000012070470020704770B50446FFF7EBFF45
:105D6000DFF87C550646287BFFF7E5FF86420BD01F
:105D7000A01E02D0C01E032804D805F5E87001F06B
:105D80000AF901E001F03DF92046FFF7DDFF064684
:105D9000287BFFF7D9FF864208D02046FFF7D4FFC3
:105DA00010B1FBF79BFA01E0FBF795FA2C7370BD7D
:105DB000DFF86807C0897047F8B5044601F09AF823
:105DC000DFF8185520B9294640F23130FBF79CFD29
:105DD000DFF80C6508234FF4847206F1700106F5B4
:105DE000BC7001F005F808B10320F2BDDFF8300700
:105DF000FBF7C6F8002848D1002130733166706681
:105E0000482106F5C47000F0C1FB482106F11400DA
:105E100000F0BCFB002C03BF00200021002294E80E
:105E2000070086E80700002001F032F9002818BFBB
:105E3000852804D02A4640F25F3101F04FF9002551
:105E4000DFF8E066E9B23046FFF7D1FD04466D1C8D
:105E50005CB10027F9B200F04EFA7F1C0028F1D0A7
:105E600000783146FFF7B4FEF4E70FF2F8600178EE
:105E70008DF8001030466946FFF7F2FD040003D0AC
:105E8000FFF7AEFD2046F2BD0020F2BD80B5FBF766
:105E9000BCF910B1FBF7BFF908B1082002BD0FF241
:105EA000C86001F007F928B1DFF8442440F2C2319C
:105EB00001F014F9002002BDFBF7B1B880B5FBF783
:105EC000B3F928B1DFF8281440F2D130FBF71CFDFC
:105ED000BDE80140FBF72BB980B5FBF79CF928B969
:105EE000DFF8F8134FF47670FBF70EFDDFF8380695
:105EF0000168890703D40068C007F7D401BDBDE875
:105F000002400FF2686082E680B50FF26460FFE73E
:105F100000F001F801BD01788DF80010684676E6C2
:105F200070B5DFF8BC63DFF8B443316E054621B9C4
:105F3000214640F22540FBF7E7FCFBF748FD062829
:105F400004DA214640F22C40FBF7DEFC2978307B56
:105F5000002900F07C80012900F08D80022900F0EA
:105F6000B980032900F09080042900F09F80052962
:105F700019D0062900F0BD80082900F0DE8009292B
:105F800000F0DD800A2900F0DC800F2900F0AF80EE
:105F900080293BD0812909D082291BD083293FD079
:105FA000842946D0852900F09E80D1E00FF2C454A8
:105FB0002046FFF726FE204600F0F4F90D20FFF7FB
:105FC00077FD00F0B9FA00F021FE0120FBF7CEF8D2
:105FD00001207CE000F0B0FAFBF7F2F80020FFF7B8
:105FE000BBFE0FF29454204600F0DCF92046FFF788
:105FF00008FE0E20FFF75CFD307B801E02D0C01E25
:1060000003280ED8BDE8704000F0FBBF05285DD026
:10601000C0F0A580072859D080F0A180082056E064
:10602000032840F09C80FBF70FF900281DD00420C6
:106030004DE0032805D1FBF707F910B10420FFF765
:106040008BFEFBF71BF900280FD006203FE0698884
:10605000F181032812BF08280FF22050FFF760FFDC
:106060000020FFF725FD746E002C78D000F0AAF90F
:1060700020684468F8E700F05FFA00F0BEFD0220F7
:10608000FFF76AFE01200BE0082805D10220FFF788
:1060900063FEFBF729F902E00520FFF75DFE032010
:1060A000FFF706FD2846FFF7ACFD4DE00320FFF7A4
:1060B000FFFC0FF2CC442046FFF7A3FD204600F082
:1060C00071F9307B062808BF072000D00220BDE808
:1060D000704041E60320FFF73FFE0220FFF7E8FC97
:1060E000284600F05FF92846BDE8704089E50F209A
:1060F00028E0A878FFF746FD0646306820B921461B
:1061000040F20250FBF700FC706820B9214640F2D3
:106110000350FBF7F9FB3068726829469047002866
:106120001CBFA87810F00F0F19D000F00F0108293C
:1061300015DABDE87040FBF79DBA082002E009209F
:1061400000E00A20FFF7B4FC2846BDE8704029E1D2
:106150002146BDE8704040F22650FBF7D5BB70BD2C
:106160007CB50FF22040DFF878410168E06E0091C5
:1061700004F5BC7504F5EC7620B93146284600F0EC
:106180007DFEE066E06EC8B1818871B1C188B1F56D
:10619000006F24BF0022C280C1884A1CC280ADF8B3
:1061A000021081884A1E82801EE0FFF7B9FE314648
:1061B000284600F08FFE0020E06618E0E06DB8B1E0
:1061C0000020FBF7DCFB208AB0F5006F28BF002021
:1061D000ADF802000121401C208204F15C00FCF7B4
:1061E000B9FA0020FBF7DAFB6846FFF799FE0120B9
:1061F00076BD2DE9FC410500DFF8E08004D1414681
:1062000040F26A50FBF780FB686820B9414640F2D3
:106210006B50FBF779FB6968086820B9414640F28A
:106220006C50FBF771FB2968086820B1414640F2C9
:106230006D50FBF769FBFAF7EEFF10B9FAF7E5FFCF
:1062400020B9414640F27150FBF75EFB0027F9B2DE
:106250002846FFF7CCFB04467F1C64B1002600F003
:1062600049F8761C0028F2D00078FFF7ACFC002833
:10627000F5D011202BE00027F9B22846FFF7B7FB35
:1062800004467F1C54B1002600F034F8761C002828
:10629000F2D000782946FFF79BFCF5E7DFF8904243
:1062A00008E0A84204D1414640F29750FBF72CFB8E
:1062B0002068046820680028F3D10FF2CC20256004
:1062C00001788DF8001028466946FFF7C9FBBDE844
:1062D000F6810000ACDC000030E0000070E000005F
:1062E0008C0000209148007800B101207047000028
:1062F00070E00000F1B22046FFF78FBB10B50446F6
:1063000004F00F00082805DA2046FBF702FA2046C1
:10631000FBF7C4F92046BDE81040FBF72EB8FBF7A9
:1063200078B87E48006E70477C48806E70470000E9
:10633000807402402DE9F041804600F040F80D469F
:1063400002E000F053F8044684B1277A002600E00A
:10635000761CF0B2B842F4DAF1B200F095F80078A9
:106360004045F5D105B12E70204600E00020BDE883
:10637000F0811146FFF774BB10B50C46020600F021
:106380000F0103D5092903DB102010BD0929FBDA11
:10639000FFF7F8FB00680028F6D02146BDE8104062
:1063A000FFF75EBB38B500F009F8002C04E000F000
:1063B00009F800F01BF80400F9D131BD0546574833
:1063C000046E704729462046FFF74ABB70B5FFF7B9
:1063D000F5FF062602E000F009F8044624B1FFF7B5
:1063E000F1FF0646062EF6D0304670BD2046FFF778
:1063F00029BB38B504460D46FAF7B8FF18B147482F
:10640000017B022901D0082032BD29462046BDE883
:106410003440FBF739B838B504460D46FAF7A6FF05
:1064200018B13E48017B022901D0082032BD29461F
:106430002046BDE83440FBF79DB870B504460D46D4
:106440006068836816461BB120469847062819D114
:10645000207AA84204D2374940F2F920FBF754FAD7
:106460000EB1072070BD00F00EF80446657805E017
:10647000FFF740FF761C0078FFF740FFF0B2A8421C
:10648000F6DB002070BD29462046FFF7B0BA70B594
:1064900004460D466068C2680AB120469047207ADB
:1064A000A84204D223494FF44670FBF72DFAFFF7B8
:1064B000EAFF04460026657805E0FFF71BFF761C1F
:1064C0000078FAF7A6FFF0B2A842F6DB70BD80B5FF
:1064D00043681B6900220BB198470246104602BD73
:1064E000F8B50E48134D046E002C11E00022F1B2F5
:1064F0002046FFF7A2FF20B1294640F26A70FBF761
:1065000003FA761CF0B2B842F0DBFFF76FFF04002D
:1065100002D0277A0026F5E7F1BD00008C000020AC
:10652000195D0000FCE90000380400400D2C00203B
:10653000EC00002070E0000070B5FFF740FF002C79
:106540000AE0E9B22046FFF7A2FF6D1CE8B2B042B4
:10655000F7DBFFF74BFF040002D0267A0025F5E7B2
:1065600070BD00000B000000E95C0000810000002D
:10657000820000000D0000000E000000030000007B
:1065800003000000000000000B000000002200F0EB
:10659000B5BD4300C0F341107047C009704710B546
:1065A000040005D1DFF8041740F24320FBF7ACF9F3
:1065B0002168086810BDDFF8F8160A7A82420AD00E
:1065C0000528087203D0487A00F0FD0048720FF2E7
:1065D0001870FFF7A5BC704764E3DFF8D4160020FD
:1065E00008607047DFF8C816086800B101207047DE
:1065F000002070472DE9FE4F0C4683466168154622
:10660000012669B92068FFF7CAFF002804BFA06807
:10661000002805D10026CBF80000CBF804605AE032
:10662000412D009505D3DFF88C1640F29710FBF74B
:106630006BF9FAF7DCFF8246009DE0684FF0000836
:106640008542C14602D9054600E00026002D3ED015
:10665000A26861682F46954288BF17460AEB08007A
:1066600029B13A46FBF778F9002060600CE05AB196
:106670002168D1F804E0DEF804C002463B4604F18C
:106680001000E0474FF00109A068E168C01BA0605E
:10669000C91BA068E160ED1BB84430B9B9F1000F27
:1066A00003D02068FFF77BFF2060E0680028CCD093
:1066B000A1680029CAD1206808B1019111E0B8F1A0
:1066C000000F606003D00098804538BF0026CBF8EB
:1066D00000A0CBF804803046BDE8FE8FA068401CC7
:1066E000A06001232168D1F804C0DCF80470002206
:1066F00001A8B8470028F1D12061A7E72DE9F84F9C
:106700000F4686B03978DFF8A855DFF8A86506246B
:106710000129804618D0022900F03082032915D0C3
:10672000052931D0062900F035820B2900F00982B5
:106730000C2900F00F820D2900F017820E2900F0BD
:106740001F82852918D048E203201AE005F12400B1
:10675000FCF710F838B1DFF8601501200860BFF3CE
:106760006F8FBFF34F8FFFF737FF002840F006828F
:1067700031464FF48760EAE1FFF72EFF032802D18C
:106780000420FFF718FF28E205208DF804000DF122
:106790000500FAF7E3FFFFF725FFFFF71EFF9DF85F
:1067A00005109DF8090001F01F01032922D8DFE838
:1067B00001F0A24D02D510F00F0F05D001A9FFF78F
:1067C000DBFD0446062C15D19DF80500FFF7E2FE1F
:1067D000002853D19DF80950FFF7FEFE0246BDF890
:1067E00007109DF8066005F00F00FEB1012E02D0E3
:1067F000032E0FD0B6E0072840DC00293ED1052A41
:1068000018BF002868D12846FAF783FF2846FAF710
:1068100045FF77E1072831DC00292FD1052A18BF71
:10682000002859D12846FAF725FF6BE1052A18BF41
:10683000002851D100F0DFF904462846FAF74AFF54
:1068400000B101202080022221463DE06946FFF789
:1068500071FD050008BF102400F0BD819DF80010F7
:1068600001AAFFF786FD0446062C15D19DF8058088
:106870009DF800604046FFF78DFE002840F0AB8198
:10688000FFF7AAFE07464046FFF787FE01289DF85E
:1068900006001ED178B10A2864D1052F1CD104A8A6
:1068A00000F0FBF9044631462846FFF710FE207041
:1068B0000122214608E0052F0ED104A800F0EDF9D1
:1068C00000210180022201460DF1050000F0A7F928
:1068D00047E00B28D2D1052F40F00481BDF8070016
:1068E000B0F5807F80F210819DF807203146284660
:1068F000FFF7A3FD35E0B8F1000F04D1314640F2B7
:106900005E30FBF701F89DF805703846FFF742FE50
:1069100020BB3846FFF741FE012840F0D1809DF8AA
:106920000600002800F0B080062825D0082813D1E2
:1069300000F061F90446FFF74FFE052808BF01206B
:1069400002D004280AD100202070012221460DF136
:10695000050000F064F90446062C03D101A8FFF7F6
:1069600035FD0446002C89D1FFF73CFE002800F0DD
:106970003F81FAF72AFF29E19DF80810BDF80B00C6
:10698000012900F07C80E7D3032901D00DD3E3E790
:10699000002875D0BDF809109DF8070000F0FAF93D
:1069A0000028DBD002780146D1E7002868D009280A
:1069B0008CBF4FF009088046FFF7B3FC09274FF062
:1069C000000912E00AF1010AD4F804C0DCF804B0AE
:1069D00001230022214604A8D8470028F2D1207ABA
:1069E00081442046FFF7DBFD5744040013D0606864
:1069F00020B9314640F2C720FAF786FF616848683F
:106A000020B931464FF43270FAF77EFF4FF0000A9A
:106A1000CDF810A0D8E700F0EEF804460098404505
:106A200004D2314640F2DD20FAF76EFF4FEA080249
:106A3000AAA12046FAF790FF84F804906780FFF738
:106A400051FC18B1E07940F02000E071FFF769FCDB
:106A5000E8602C61C5F81480BDF80B00A861002027
:106A6000FAF78DFFA3A18020FFF7D5FC040002D127
:106A700000F000F904460020FAF790FF6CE70028C8
:106A800040D0122290A162E700F0B5F804460098C9
:106A9000022804D2314640F29520FAF735FF002053
:106AA00020706070207840F001002070687AC0F398
:106AB000400018B1207840F002002070022245E723
:106AC0009DF80610BDF8070001291FD0032927D023
:106AD000052930D00929D1D1FFF77EFD052818BF3F
:106AE000042801D0082476E09DF8070018B9FFF7C4
:106AF00023FD042004E0012806D1FFF7F1FC052066
:106B0000FFF759FD00242FE7072464E0012817D17F
:106B1000FFF7E8FB48B1687A00F0FD006872F1E722
:106B200001280DD1FFF7DEFB08B90F2453E0687A86
:106B300040F00200F2E7314640F28230FAF7E4FE1C
:106B40000CE7FFF749FDC8B1314640F24C40FAF777
:106B5000DBFE13E0FFF740FD012804D0314640F290
:106B60005240FAF7D1FE002006E054480068C10701
:106B700048BF022000D40120FFF71DFD00242CE0B7
:106B8000FFF72AFD0128F6DC314640F26640FAF7AD
:106B9000BBFEF0E7F87803281FD0B878002818BFAC
:106BA000802804D0314640F27540FAF7ADFE2E68D9
:106BB000FC7830000ED0FFF710FD69682046B04722
:106BC000040008D1FFF70EFD58B1B87828B9FAF7DC
:106BD000E1FD02E00E24FAF7F5FD204607B0BDE81E
:106BE000F08F37480168082904BF40680028F4D0B6
:106BF000FAF7E5FDF1E768464FE080B50020FFF7C2
:106C00007DFBBDE802408020FFF778BB80B5002007
:106C1000FFF785FBBDE802408020FFF780BB7FB512
:106C2000C0881646B0420C4616D205460020029097
:106C3000009401950020FAF7A2FE69468020FFF734
:106C4000D8FB040002D100F015F804460020FAF742
:106C5000A5FE204604B070BD86423546E6D28020AF
:106C6000FAF77FFBB6FBF0F100FB1166701E804166
:106C7000C00FDCE71DA18020FFE738B504460D46B4
:106C8000FAF7A3FDA04201D0102032BDD5E90001E2
:106C9000074AC2E90001002032BD08B1402101606D
:106CA000084870470248007A70470000B0E00000D2
:106CB000002B002058DE00005C70024038040040C9
:106CC00030010010402A00201201000200000040A4
:106CD00015190D5200010102030100000902000014
:106CE000000104C0320000000F000000F165000048
:106CF00000000000F56500000C2B002003000020C0
:106D0000521E22BF13F8010B11F801CBB0EB0C009F
:106D1000F6D0521C08BF10467047FEE701B55AB1C5
:106D200011F8013B521E00F8013B03B1F8D11100EC
:106D30001CBF0022FAF714FF01BDFEE7F8B50E46AE
:106D40001F4901EB800757F82610087808B9881CFE
:106D5000F2BD0020FFF7A1FF57F82660194F044647
:106D600000250CE0E8B21F2803DB3946E620FAF7DD
:106D7000CBFD6D1C16F8011BEAB224F81210307816
:106D80000028EFD12D06ED0DAD1C45F44075258092
:106D90002046F2BD010002D1002100200FE00628AC
:106DA0000AD200BF08A1085C02001FBF044A0346C4
:106DB00052F82310002901D1002070470021BDE7BF
:106DC000680200209CDA00000001020304050000B4
:106DD000A0F16101062924BFA0F14102062A04D3D3
:106DE00030380A288041C00F704701207047FEE705
:106DF00050B509B90E2050BD144694FBF3F603FBC1
:106E000016440CB1092050BD01608460002141602E
:106E10008281C381002050BD3CB550E8015FAAB219
:106E2000C3891A4483899A4228BFD21A03899A4295
:106E300002BFBFF32F8F002407E0C2EA050240E83B
:106E40000123002BE9D14FF0010400F03AF81AB108
:106E500000680988084436BD002036BD0A88498884
:106E60008A4209D150E8011FC1EA014140E80112FC
:106E7000002AF7D101207047002070473CB550E848
:106E8000025F1FFAA5F2C3889A4202BFBFF32F8F99
:106E900000240DE0C3891A4483899A4228BFD21A7C
:106EA000C5EA024240E80223002BE8D14FF001047A
:106EB00000F007F81AB100684988084436BD002080
:106EC00036BD01958DF80040019B0B609DF80020B8
:106ED000704700000A8849888A4209D150E8021F99
:106EE000C1EA214140E80212002AF7D1012070478F
:106EF0000020704764480078704738B5624C2078AD
:106F000008B185250DE0A060002161602061E1608D
:106F10000FF25D1000F016F9054600F025F901208A
:106F20002070284632BD03681A4600E0126812B18C
:106F30008A42FBD170470B600160704770B500F06A
:106F40005BF819B92946E920FAF7DEFCB07830B1D0
:106F500014B161680120884700F04BF80BE0FAF7A4
:106F60000EFD24B1214606F11000FFF7DCFFF068AA
:106F700008B900F00FF9F068401CF0600020FAF743
:106F80000DFDF06830B92946BDE8704040F20510AB
:106F9000FAF7BABC70BD70B500F02EF821B92946D9
:106FA0004FF49370FAF7B0FC707830B114B16168A7
:106FB0000020884700F01DF80BE0FAF7E0FC24B150
:106FC000214606F10800FFF7AEFF706808B900F02F
:106FD000F4F87068401C70600020FAF7DFFC7068FD
:106FE00030B92946BDE870404FF4A170FAF78CBC67
:106FF00070BD0020FAF7C3BC234E244D31780446FF
:10700000704738B500F01DF820B9214640F247100E
:10701000FAF77AFC686820B921464FF4A470FAF7B1
:1070200073FCFFF7E6FF6868401E6860686818B97F
:1070300000F0D6F8002068700020BDE83240FAF772
:10704000ADBC114D114C2878704738B504000E487E
:1070500014BF00F1100500F1080504E0086828607D
:1070600020464968884729680029F7D131BD0000CA
:107070000200054903D101234B70002002E00128E2
:1070800001D18870E1E77047A82B002030E10000B3
:1070900010B5074C217809B1852010BD08B900BF93
:1070A0000DA000F0FFF808B90121217010BD00000B
:1070B0000E2C002010B5044600F007F8204600F022
:1070C0001AF900F023F9002010BD80B500F020F976
:1070D000BDE8014000F021B90000FEE700B583B033
:1070E000029000910192034871466A46FAF7E6FC65
:1070F00003B000BD014000007047FEE700B500BFCF
:10710000130096469446103928BFA0E80C50FAD8D0
:107110005FEA417C28BF0CC048BF40F8042BC90778
:1071200028BF20F8022B48BF00F8012B00BDFEE766
:107130004FF0804181B000220A5008580090009919
:1071400001B0704710B5040003D14049A420FAF7FC
:10715000DBFB3F4A1179002009B1852010BD146086
:1071600001211171507110BD10B5394C207918B939
:107170003649BD20FAF7C8FB36480168C90704D470
:10718000354BC0221A70012101600120334A106082
:10719000207210BD80B52E49087918B92B49EA2014
:1071A000FAF7B2FB4FF48270FFF7C2FF2D492E4B66
:1071B0000220086001221A6001BD80B524490879C7
:1071C00018B92249FF20FAF79FFB4FF48070FFF7B0
:1071D000AFFF244901204FF080430860186001BDD3
:1071E00010B51B4C207920B9184940F20710FAF766
:1071F0008BFB1E481E4A01210160116801F001113C
:10720000B1F1011FF9D00020607110BD70B5194EA9
:107210000F4C3068124D50B14FF48070FFF788FF6B
:1072200001212960607910B9617122689047706806
:1072300050B14FF48270FFF77BFF022028600120DD
:107240002168BDE87040084770BD0000F0E1000013
:10725000042C002000E100E000E400E018050040FC
:107260000803004004030040080000400400004000
:107270000C040040000100404FF0804181B000222A
:107280000A5008580090009901B0704710B54FF0AF
:107290008042115819B1FFF7EFFF012400E00024EC
:1072A000204610BD10B5040003D155497020FAF7EF
:1072B0002BFB5249087808B1852010BD227851482F
:1072C000520802F001028260227802F0010202609C
:1072D0004D480268D20704D44C4CC02323700122CD
:1072E000026001200870002010BD2068002100B15C
:1072F00001464248704710B5040003D14049ED20D3
:10730000FAF702FBFFF7F1FFC16010BD404900E052
:1073100040494FF460700860704738490020C860E9
:10732000704770B53A48364C0668344D71070DD534
:107330004FF48470FFF7AAFF40B1686820B9214676
:107340004FF48B70FAF7E0FA68688047B1060ED503
:107350004FF48A70FFF79AFF48B1A86820B9214618
:1073600040F21F10FAF7D0FAA9680020884770068B
:107370000ED54FF48C70FFF789FF48B1A86820B98B
:1073800021464FF49370FAF7BFFAA96801208847A5
:1073900030060ED54FF48E70FFF778FF48B1E868DD
:1073A00020B9214640F22F10FAF7AEFAE968002022
:1073B0008847F0050ED54FF49070FFF767FF48B18E
:1073C000E86820B921464FF49B70FAF79DFAE96806
:1073D00001208847B00510D54FF49270FFF756FF93
:1073E00058B1E86820B9214640F23D10FAF78CFA0E
:1073F000E968BDE870400220084770BDD02B00202E
:1074000070E200007805004000E100E000E400E0E8
:10741000040300400803004080B5FFF782FFBDE889
:107420000140FFF7F3BEFEE72DE9F14FB2B09946F8
:10743000924600230691CDE900333C9A0F930DF15B
:107440004A0114914A7011E0329E57462C4617F8B3
:10745000011B0698B0470028069000F026810F987F
:10746000401C641E0F90F2D13296AA449AF8000094
:10747000252808D10021002209910A920B910C9233
:107480000D910E920FE06A464FF0FF315046FBF728
:1074900060FC050002D10F9800F066BED4D501252E
:1074A000E3E741F001011AF8010F2028F9D0232861
:1074B0000CD02B2804D02D2805D0302809D00BE083
:1074C00041F00201EFE741F00401ECE741F008016F
:1074D000E9E741F01001E6E72A280FD1D9F80020AA
:1074E00052F8040BC9F800200028119003D540423F
:1074F000119041F004010AF1010A14E01192DFF841
:10750000EC3B0AE01198984205DA00EB800402EBAC
:107510004402303A11920AF1010A9AF80020A2F1CD
:1075200030000A28EED39AF800002E2803D04FF03E
:10753000FF32109229E01AF8010F2A2809D1D9F850
:10754000000050F8042BC9F8000010920AF1010A5B
:107550001BE02D280CBF0AF1010A00200022109226
:10756000DFF8882B0BE040B9109B934205DA03EB60
:10757000830504EB4504303C10940AF1010A9AF8A3
:107580000040A4F130030A2BEDD3ADF848100FF6FC
:1075900060309AF8001000F0ABFF08B11AF8010B48
:1075A0008DF84A009DF84A00682805D19AF8000035
:1075B00068280CD1622106E06C2804BF9AF800000C
:1075C0006C2804D171218DF84A100AF1010A1FA814
:1075D00008901AF801BBBBF125012DD01C3900F031
:1075E0006181091F022940F25D810E392AD0491FAD
:1075F00000F0B284093900F05581891E00F04885F9
:10760000491E00F0F484491E022940F24B81091FF3
:1076100000F0ED84491F00F0BA80491E00F09C8400
:10762000491E65D0C91E21D0891E00F09584C91E4F
:1076300000F0928400F04BBD25238DF87C300121B1
:1076400009912AE06C208DF84A00D9F8000050F822
:10765000042BC9F80000002A43D114994878002867
:107660003DD04FF0FF340FF6902012E09DF84A0015
:107670006C28EAD0D9F8000050F8044BC9F8000093
:107680000794D4B91499487898B14FF0FF340FF6A5
:10769000842000F039FF201A07D132981FAA04A9CC
:1076A00000F065FD00287FF5E1AE4FF0FF3000F0FF
:1076B0005BBD0FF67C200790EFE7109D002D04D5F1
:1076C0002046FBF751FB044607E02A46204600F01F
:1076D0003BFF002814BF041B2C460A94DDE70FF67D
:1076E0005422329804A900F0C8FD0028D5D5DCE763
:1076F000D9F8001051F8040BC9F8001020F000046C
:10770000002121F0FF351FABCDE904450793DDE9EA
:10771000042308993C2413B90AB9109898B102F0CF
:107720000F053035641EEEB23A2EA8BF2735120978
:1077300042EA03721B090D5508BF002A03D00798BF
:107740000D19A842EBD308190790C4F13C02109818
:107750000A92824209DABDF84810821A4FF6EF7099
:1077600001400C92ADF8481097E7002895D59DF898
:10777000480000F0140010288FD1119B09990C9833
:107780005B1A1B1A9A1A002A87DD0C9285E7149956
:10779000487820B14FF0FF340FF69C1079E79DF840
:1077A0004A00622862D0682819D06A2840D06C2824
:1077B00006D071284DD074282DD07A281ED064E0D0
:1077C000D9F8001051F8040BC9F8001020B94FF097
:1077D000FF340FF67C105CE70F9901605DE7D9F884
:1077E000001051F8040BC9F8001020B94FF0FF3415
:1077F0000FF65C104DE70F9901804EE7D9F80010A5
:1078000051F8040BC9F800100028E5D14FF0FF34FF
:107810000FF63C103DE7D9F8001051F8040BC9F8F9
:1078200000100028D8D14FF0FF340FF6241030E7B5
:10783000D9F8001051F8040BC9F8001020B94FF026
:10784000FF340FF60C1024E70F9AD317C0E900237A
:1078500023E7D9F8001051F8040BC9F800100028EC
:10786000F2D14FF0FF340FF6E80012E7D9F800101C
:1078700051F8040BC9F8001020B94FF0FF340FF68F
:10788000D00006E70F99017007E7D9F8001051F80A
:10789000040BC9F8001000289ED14FF0FF340FF6FA
:1078A000B000F6E6D9F80020D21D22F00702C9F890
:1078B0000020D2E900010832C9F80020CDE9040116
:1078C000C80F02D009982D210AE0BDF848008107B1
:1078D00002D509982B2103E0C00705D5099820217E
:1078E0001FAA1154401C09901FA809994BF02002AF
:1078F0004318DDE90401CDE92E01612A079315AC97
:107900000BD01098002802D50620109005E001BF8A
:107910004BF02000672801211091DDE904014800A7
:107920004015401C0A4611D109030FD0ABF1610587
:1079300003201A2D0A9002D20FF6A03101E00FF6B3
:10794000A03103221846FAF707F8A6E650B9120349
:1079500008D1ABF1610503201A2D0A9016D30FF65A
:107960008831EEE7DDE90401CDE93001DDE93023BE
:1079700023F00047B7F5801F22F000060DD2002249
:10798000002F08BF002E029203D116E00FF65431EB
:10799000D7E702AA00F004FE0FE0DFF8F00ADFF8F4
:1079A000F01A00EB17500290DDE930234FF0FF3062
:1079B0001940DFF8E07A10403943CDE904014BF07B
:1079C000200061280DD1079830210170821CBBF185
:1079D000610F07920CBF7821582141700998801CD3
:1079E0000990DDE9040120F0000231F0004308BFF6
:1079F000002A02D10026002571E14BF02008B8F1E1
:107A0000610F40F0BE801098002847BF21210391EC
:107A1000401C0390039FDDE92E017F1C0022002300
:107A2000DDE9044500F0F4FD02998DF8542038BFDB
:107A300085F00045091F002F02910DF155065DDD0F
:107A4000DFF8541ACDE9302140F2FF732E9320461F
:107A500029460022002300F0F3FD4FD24800400DDC
:107A600000F11C0315D0002B13DD2E9883420ADB96
:107A7000DDE9300121F0004005F000420243DDE97C
:107A80003001114611E06FF31E5141EA03512046C7
:107A90000BE024F0000035F0004108BF00280FBFC4
:107AA00029461C22294600F0E3FD04460D4600F05D
:107AB0007DFEFF1F002F804609DD00F095FE024687
:107AC0000B462046294600F0A1FE04460D46F01D57
:107AD0000721B8F1000F0CDD491E5EBF08F00F0250
:107AE00000F8012D4FEA2818F3D502E0002200F833
:107AF000012D491EFAD5C61D002FA8DC0DF1550039
:107B0000361A03988642D8BF304600280DF1550436
:107B100030D4B04206DA0DF155010A5C082AA8BF3C
:107B20000F2100DA0021024615AB134400E0401E8D
:107B300013F80159521E8D42F9D00F2904D10DF1CD
:107B400055018B5C5B1C8B54002A04D50299091DDE
:107B500015AC401C0291411E0CD46218ABF13A06E0
:107B600013783033DDB23A2DA8BFF318491E02F85E
:107B70000139F5D51099002940F1AF80421E1092CD
:107B8000ABE00299DFF8142947F29750414391FB8B
:107B9000F2F2DDE92E45029225F00045D2F107020E
:107BA00004DD2046294600F04DFC0BE05242002047
:107BB000DFF8EC1800F046FC02460B46204629464A
:107BC00000F096FE0446B8F1660F109806BF029FBB
:107BD0000A3706273F18142FC8BF142730208DF806
:107BE00054000D460020DFF8BC18CDE92E010DF140
:107BF0005506002F33DD2046294600F09DFF014643
:107C00000A4606F1080304200A26B2FBF6F606EB44
:107C1000860EA2EB4E02303203F8012C0A22B6FB8C
:107C2000F2F202EB820EA6EB4E063036401E03F84F
:107C3000026DE9D1083F002F03F10806D9DD08469F
:107C400000F08EFF02460B462046294600F0DEFD7E
:107C5000DDE92E2300F092FF04460D46CBE70DF13F
:107C60005500361A0DF1550404E00298401E761EA8
:107C70000290641C20783028F7D0B8F1660F02D14A
:107C80000299491C04E0B8F1650F0CBF01210021E5
:107C9000109808188642B8BF701E00281DD4B04244
:107CA00004DA215C3429C8BF392100DC30210246C6
:107CB000631E9D1800E0401E15F80169521E8E4299
:107CC000F9D0392902D1A15C491CA154002A04D55C
:107CD0000299491C1C46401C02910646029DFBF776
:107CE0003CF8406A0778DDF8408030B2002802DCBA
:107CF00001260FF2F8744BF02000662808BF6D1CB7
:107D000016D0672846D128B210F1040F48DB404551
:107D100046DA9DF848006D1C010703D430B2404597
:107D2000B8BF804628B2B8EB000848BF4FF0000843
:107D30000FFA85FB07980A99BBF1000F00F3B28098
:107D40004A1C0A9230234354B8F1000F03DC9DF81B
:107D50004800010704D50A98411C0A9107990F545D
:107D600018EB0B0FB8BFC8F100052DB268420D909B
:107D7000A84432B29045B8BF4646079B0A9836B22F
:107D80000B96324621461844F9F7E6FDA8EB0600AB
:107D90000E90CBE0BBF1610F17D14FF0700B19E0E3
:107DA00030B2404504DA9DF848100A0758BF8046B3
:107DB000B8F1010848BF4FF00008BBF1670F14BFCE
:107DC0004FF0450B4FF0650B04E0BBF1410F08BFCE
:107DD0004FF0500B0A98411C0A91B8F1000F079917
:107DE00014F8012B0A5403DC9DF8480001071AD54A
:107DF0000A98411C0A91B8F1000F07990F5412DD3F
:107E0000761E30B2804507980A9BB8BF464632B20C
:107E100021461844F9F7A0FD0A9936B271180A9163
:107E2000A8EB06000D9007980A9908442AB2002A88
:107E300080F800B003D42B224270811C04E02D2175
:107E400041701546811C6D4200202EAA0A2409E0CB
:107E50002B4693FBF4F505EB8506A3EB460302F8EE
:107E6000013B401C2DB2002DF2DC012806DC4BF05A
:107E70002002652A04BF302201F8012B00282EAA17
:107E800008D1302001F8010B06E0401E135C3033AE
:107E900001F8013B0028F8DC079A0A981044091AF7
:107EA0000B9143E0084431B22AB2914219DA32B25E
:107EB0002146F9F751FD0A9936B27118ABEB060667
:107EC000B8F1000F0A910D9603DC9DF848000207F7
:107ED00004D5079847540B99491C0B91CDF838806D
:107EE00024E02146F9F738FD0A98761B5844B8F18A
:107EF000000F0A9003DC9DF848100A0703D5411CC7
:107F00000A9107990F5430B2804507980A9BB8BF71
:107F1000464632B204EB0B011844F9F71DFD0A98EE
:107F200036B230180A90A8EB06000D909DF8480074
:107F300000F0140010287FF4B0AB099A0A990D984C
:107F40008A180B9982180E988A1882181198824202
:107F5000BFF6A3AB821A18E49DF84A00622808D045
:107F600068280ED06A2814D06C281FD0712810D031
:107F70001CE0D9F8001051F8040BC9F80010C0B289
:107F80001AE0D9F8001051F8040BC9F8001080B2BB
:107F900012E0D9F80020D21D22F00702C9F8002013
:107FA000D2E900010832C9F8002006E0D9F8001033
:107FB00051F8040BC9F800100021CDE904019DF827
:107FC000480001075AD5DDE90423002B08BF002A29
:107FD00054D04BF02000782850D109981FA93022A6
:107FE0000A54401C431C099301F800B046E09DF878
:107FF0004A00622808D068280ED06A2814D06C285D
:108000001FD0712810D01CE0D9F8001051F8040BD3
:10801000C9F8001040B21AE0D9F8001051F8040B6A
:10802000C9F8001000B212E0D9F80020D21D22F0E9
:108030000702C9F80020D2E900010832C9F800207F
:1080400006E0D9F8001051F8040BC9F80010C11768
:10805000CDE90401002902D509982D210AE0BDF8D7
:108060004800810702D509982B2103E0C00705D5F8
:10807000099820211FAA1154401C09901FA8099992
:108080000144079104A8594600F057F9FFF705BBD2
:108090009DF84A006C280BD001210991D9F8000005
:1080A00050F8041BC9F800008DF87C10FFF7F5BAF2
:1080B000D9F8000050F8041BC9F8000015914FF0E2
:1080C000FF3210920021169115AAFFF70ABB252155
:1080D0000122BBF1000F8DF87C1009923FF4DDAA5C
:1080E0008DF87DB00221FFF7ABBA0000CBCCCC0CF1
:1080F000686A6C747A4C00007072696E74665F73A3
:108100003A2062616420256C7320617267756D6529
:108110006E7400007072696E74665F733A206261FB
:108120006420257320617267756D656E74000000B0
:1081300000000000000000007072696E74665F73DA
:108140003A20256E20646973616C6C6F77656400FA
:108150007072696E74663A2062616420256E2061D7
:108160007267756D656E740033B0BDE8F08F2DE9F0
:10817000FC410F46064690467A6B7869396ABC6ABC
:10818000121AB869521A796A121AF869521A121A2E
:1081900097F83800141B41070FD42020002C8DF8CD
:1081A00000000ADD254601236A463946304600F0C4
:1081B0007DF900285DD16D1EF5D17B6942463946B7
:1081C000304600F073F9002853D130208DF80000BC
:1081D0003D6A002D09DD01236A463946304600F02C
:1081E00065F9002845D16D1EF5D1BB69FA6839469D
:1081F000304600F05BF900283BD130208DF80000BC
:108200007D6A002D08DD01236A463946304600F0BC
:108210004DF970BB6D1EF6D1F868B969FB6942185B
:108220003946304600F042F918BB30208DF8000086
:10823000BD6A002D08DD01236A463946304600F04C
:1082400035F9B0B96D1EF6D197F8380041070DD554
:108250002020002C8DF8000008DD01236A463946F5
:10826000304600F023F920B9641EF6D10020BDE8A5
:10827000F6814FF0FF30BDE8F6812DE9F8470D4655
:10828000A3B02F6B002F8246904648BF6FF0004787
:1082900000F045FD696B401801AA0021C2E90011F8
:1082A000812828BF4FF0FF3044D289461EE0A74204
:1082B00030DB6869201881280BD30021696303AA89
:1082C00029465046FFF753FF5FEA000922D40020F9
:1082D000686103AB6E69224669469819F9F73CFB61
:1082E000A6196E6158F8040BA0B13F1B002F11DDD9
:1082F000D8F8001001AA6846FAF72DFD0446002CB4
:1083000005D4D8F800000028D1D1641ECFD54FF095
:10831000FF390EE0B9F1000F504604D103AA2946F7
:10832000FFF725FF8146B9F1000F02D100206861F7
:108330006863484624B0BDE8F0872DE9FC43074652
:108340006F293E6908BF082405D041F02000782835
:1083500014BF0A2410243C25D7E90023642918BF40
:1083600069299046994605D1002B03D5D8F100081C
:1083700069EB4909B9F1000F08BFB8F1000F0CD142
:10838000386B50B9082C39D197F83800010735D52A
:1083900030203B2586F83B0030E08DF80010404649
:1083A00049462246E31700F0BFFC3032D0B26D1EC2
:1083B0003A28019504DB9DF80000A0F151018A18CC
:1083C0007255404649462246E31700F0ADFC804610
:1083D0005FEA010908BFB8F1000F03D0F86871190E
:1083E0008842DCD3082C09D197F83800010705D55D
:1083F000705D302802D06D1E30207055C5F13C02F2
:10840000BA617119F960386B824208DA821A3A62ED
:108410004FF6EF70398F01403987BDE8F3830028AC
:108420000ED597F8380000F01400102808D17B6BA7
:108430007969386A5B1A1B1A9A1A002AC8BF3A620D
:10844000BDE8F3832DE9D04306460F4614464FF0AE
:108450000008DFF8549012E0E00707D542464B468B
:108460003046394600F08AFB06460F4640464946EC
:1084700042464B4600F082FB641080468946002C41
:10848000EAD130463946BDE8D083000002FCFFFF48
:10849000FFFF0F800000E03F0000F07FA08601009A
:1084A0000000F03F84D7974100002440F8B505460E
:1084B0000E4617461C4600205CB117F8011BB06839
:1084C000A847B06030B1F06A401CF0620020641E22
:1084D000F3D1F2BD4FF0FF30F2BD00006E616E00CF
:1084E0004E414E00696E6600494E46003000FEE780
:1084F000C9B202788A421AB11CBF10F8012FF9E7FD
:1085000018BF00207047FEE780B500B906A00549F6
:108510000B681BB122220021984701E000F087FC84
:10852000222002BD502C0020636F6E73747261694B
:108530006E742068616E646C65723A2062616420BA
:108540006D65737361676500C9B2830706D0521EFB
:1085500022D310F8013B9942F7D11FE0083A13D318
:1085600002F1040241EA012141EA014150F8043BD1
:10857000121F21BF4B40A3F1013C2CEA030C1CF05D
:10858000803FF3D0C9B2001F083210F8013B521EE1
:1085900028BF91EA030FF8D818BF0120401E70478A
:1085A00010B5144600F002F8226010BDC1F30A5362
:1085B00043B14A0012F5001F28D2A3F2FE32A1EB0C
:1085C0000251704750EA410C20D001F0004C31EAD2
:1085D0000C01B1FA81F204BFB0FA80F3D2180B3A61
:1085E000B2F120032CBF00FA03F1914041EA0C01E3
:1085F0003EBFC2F1200C20FA0CF3194390405242C6
:1086000040F2FD33D21A01EB03517047002270474C
:108610004FF4001C1CEB410F94BF1CEB430F09E00F
:1086200041EA030C50EA4C0C52EA0C0C03D299427A
:1086300008BF9042704714BF8B4282427047FEE7EA
:108640004FF4001C1CEB410F94BF1CEB430F09E0DF
:1086500041EA030C50EA4C0C52EA0C0C03D28B4258
:1086600008BF8242704714BF994290427047FEE7AC
:10867000124254D440F2FF7C1CEA11530FD06345E0
:1086800031D09B1863453CBF01EB0251704701F0AC
:10869000004141EA0C510020AFF30080704750EADE
:1086A000410320D001F0004C91EA0C011CD0B1FA3A
:1086B00081F30B3B9A420DD9D21A994051EA0C0131
:1086C000C3F1200C20FA0CFC61449840531C40F28A
:1086D000FF7CD7E7914041EA0C01C2F1200C20FA5F
:1086E0000CF3194390407047B0FA80F31533202BF8
:1086F000E0D3202AEED3203A203B9A4209D9D21A5D
:1087000000FA03F141EA0C010020531C40F2FF7C07
:10871000B8E700FA02F141EA0C010020704752422A
:1087200040F2FF7C1CEA11530DD06345DBD0B2EB65
:10873000030C3CBFA1EB025170470CF1010221EA8E
:10874000035141F4801150EA410CCCD001F0004CAF
:10875000352A27DC30B481EA0C01B2F1200309DAB2
:10876000C2F12003044601FA03F5D0402843D1406A
:108770009C400CE0C3F12002450020FA03F418BF2E
:1087800044F0010421FA03F091400C43002174F1FC
:10879000004550F1000051EB0C01244230BC7FF445
:1087A0007BAF70476146002076E7FEE7C1F30A53CE
:1087B00040F2FE329B1A14DDD3F120034FEAE1723E
:1087C00008DDC90241EA505141F00040D84080180C
:1087D0005040704703F2E13010B1D24382F00040C4
:1087E000704700207047FEE7C11768B14840401A43
:1087F000B0FA80F29040D21CC907C2F5846241EA07
:10880000025202EBD02140057047FEE770B44FF0F2
:10881000004591EA030F40F10D836B40841A71EB20
:10882000030603D2001BB141121973414FF4001C1F
:108830001CEB410F34BF7CEB430442E00C0DA4EB76
:108840001356352E4FDC45EAC323DB0A45EAC12126
:10885000C912B6F120050DDD63FA05F6EB4086EA94
:108860000305124218BF45F00105C01851F100017F
:108870000CD213E062FA06F5F2405540F3415A403B
:10888000B340F3405A408018594107D349085FEA82
:1088900030005FEA350528BF45F0010501F580117C
:1088A000420875F1004250F1000041EB04514E00C6
:1088B00016F5001F70BC38BF70470020090D090570
:1088C00070471CEB410F10D252EA43060BD0BCEBB1
:1088D000410F05D80C0DAB43661E342EB6DD02E009
:1088E000AB438018594170BC704770BC7047FEE7BD
:1088F000F0B540F2FF7581EA030C0CF0004C15EA6C
:1089000011541DBF15EA1357AC42AF42E5E0BC411C
:10891000C1F31301C3F31303801A994143F4801385
:1089200004D2641E4000494180185941C90241EAFD
:108930005051B1FBF3F603FB1611A2FB0675D7EB02
:10894000C020A94102D2761E80185941C90241EACD
:108950005051B1FBF3FE03FB1E11A2FB0E75D7EBCA
:10896000C020A94103D2AEF1010E801859418902FD
:1089700041EA9051760546EA8E2EB1FBF3F603FBF1
:108980001611A2FB0675D7EB8020A94102D2761EF4
:1089900080185941C90241EA50514EEA060EB1FB16
:1089A000F3F603FB1611A2FB0675D7EBC020A94115
:1089B00002D2761E80185941C90241EA5051B1FBDA
:1089C000F3F703FB1711A2FB0735D3EBC020A94136
:1089D00067F100070CBF004247F0010766F3D52797
:1089E0004FEA1E31B80814F5806412DDBD0775F139
:1089F000004250EB0E5051EB045111F5801F5CBF4B
:108A000041EA0C01F0BD4CF07F6141F0E0410020F3
:108A1000F0BDBD076D0840EA0E5041F48011D4F15D
:108A20000104B4F120060ADAC4F120060200E04095
:108A300001FA06F3E1401843B24015430EE0342C2E
:108A400013DCC6F1200445EA40056D0820FA06F261
:108A5000154321FA06F0A1400D43002175F10042B3
:108A600050F1000051EB0C01F0BD00205FEA0C0159
:108A7000F0BDCFB992185B41B3FA83F704BFB2FAE5
:108A800082F6BF190B3FB7F120062FBF02FA06F39B
:108A9000BB40C7F1200622FA06F638BF3343BA407E
:108AA0001CB1E419641E33E77F4231F00041B1FA92
:108AB00081F404BFB0FA80F6A4190B3CB4F120068F
:108AC0002FBF00FA06F1A140C4F1200620FA06F6F5
:108AD00038BF3143A0403C1B1AE7AC421ABF05EA3D
:108AE0001357AF4212E050EA41061CBF52EA430658
:108AF000BFE750EA4107304661461CBF41EA0551D5
:108B0000F0BD52EA430C08BFC143F0BD00204FF452
:108B1000001616EB410F98BF16EB430F08BF16EB7C
:108B2000410F24BFC14305E016EB430F0CBF614664
:108B30004CEA0551F0BDFEE7400D491840EA81209E
:108B40000CD2490DA1F58061491C40F0004005DBC5
:108B5000D1F11F0154BFC840C017704700207047B3
:108B6000014648B1B0FA80F18840C91CC1F5846162
:108B7000090501EBD02140057047FEE7B0B581EA59
:108B8000030C0CF0004C40F2FF7515EA11541DBFA8
:108B900015EA1357AC42AF4239E0E41923EA4553D2
:108BA00043F48013C90241F0004141EA505EC7021C
:108BB0001100A7FB020200284FF00000EEFB01208D
:108BC0004FF00001E3FB072118BF42F001024018FB
:108BD00000214941E3FB0E01A4F580640F0302D29A
:108BE00052004041494154F101046CDD470872F1E3
:108BF000004250F1000051EB0451A1F580115CBF1F
:108C000041EA0C01B0BD4CEA05510020B0BD05EAB7
:108C10001357AC4214BFAF4241E050EA410E1CBFB3
:108C200052EA430E02E061460020B0BD24423C44BB
:108C30001BD15FEA070EF6D0090302BF01460020F0
:108C4000AEF1140EB1FA81F7AEEB070401FA07FE9C
:108C50000C37C7F1200100FA07F7C8404EEA000EB2
:108C600023EA455343F48013A2E733F00043B3FAF9
:108C700083F704BFB2FA82FE77440B3FE41BB7F1DF
:108C8000200E2FBF02FA0EF3BB40C7F1200E22FACE
:108C90000EFE38BF43EA0E03BA40641C82E750EA76
:108CA000410E14BF52EA430E6FF000014FF400175B
:108CB00017EB430F8ABF194617EB410FB5E74CEA94
:108CC00005510020B0BDD4F10104B4F120070FDA42
:108CD000C4F12007520828BF42F0010210FA07F53C
:108CE00001FA07F7E1BF2A43E0403843E1400FE0D3
:108CF000352C98DCC7F1200452EA400220FA07F232
:108D000018BF42F0010231FA07F0A1400A430021E6
:108D100072F1004250F1000051EB0C01B0BD80B582
:108D2000F9F7E3FF006C02BDD3BBD9B1B2F5803FC8
:108D30005BD2022A1ED98C46B1FBF2F102FB11C3B1
:108D40001B0443EA1043B3FBF2FC02FB1C3380B26A
:108D500040EA0343B3FBF2F002FB103240EA0C405E
:108D600000237047022A05D98446B0FBF2F002FBCB
:108D700010C270474AB105D100F0010249085FEA0C
:108D80003000704700220023704700F009B90B0043
:108D90000200002100207047F7D300220023704713
:108DA000904271EB030CF2D370B5B1FA81F4B3FACF
:108DB00083F52C1BA340C4F1200532FA05F633439A
:108DC000A2405FF00046E64002E05B085FEA320244
:108DD000841A71EB030524BF204629467641F4D35B
:108DE00002000B003000002170BD70B5B1FA81F4B3
:108DF000B2FA82F5C4F120046419B4F12006DAD382
:108E0000B2405FF00044F440002502E052085FEAFF
:108E10003303C61A71EB020E24BF3046714664411B
:108E20006D41F3D302000B002000290070BD01202A
:108E300000F0B8B8841A71EB030604D26E40001B30
:108E4000B141121973414FF4001C1CEB410F34BFA8
:108E50007CEB430683E00C0DA4EB1356362E00F397
:108E60007C80012E45EAC32341DC43EA525312BF02
:108E7000D20292025B08240545EAC12141EA505121
:108E8000D2EBC020994125D407D1B0FA80F610FA70
:108E900006F162D00020203608E0B1FA81F6B14038
:108EA000C6F1200220FA02F21143B0404FEAF474F6
:108EB000B4EB465434F001064FEA74040AD8D6F5F0
:108EC0000016760D04F00044F04061FA06F25040BE
:108ED000F1404840C00A40EA415021F0004128BF1B
:108EE0005FEA500550F1000044EBD12135E0DB0A88
:108EF00045EAC121C90AB6F120050EDD42EA024267
:108F0000120CC5F1200603FA06F6EB4042EA06050C
:108F10006D42984161F100010DE062FA06F5F24000
:108F2000554063FA06FC82EA0C02F3405A406D4257
:108F3000904161EB030111F4801F05D1641E6205AD
:108F400002D06D004041494121F48011430875F180
:108F5000004350F1000041EB045170BC70471CEB22
:108F6000410F15D223F0004352EA43060BD04FEADB
:108F70004C0CBCEB410F04D80C0D661E342EB7DD33
:108F8000EBE7801A994150EA410608BF0021E4E767
:108F900008BF1CEB430F28BF6FF00001DDE7FEE7C1
:108FA0007047FEE72021090326311820ABBEF9E700
:108FB00070B5DFF8F0444FF40C71201DF8F76CFD2C
:108FC000012104F50D70FBF7C5FB00F0C7F80FF2A7
:108FD000FC41451BED082D0445F003063046F8F72B
:108FE00048FF0020FBF728FA45F0010510B10FF209
:108FF000FC410EE00FF210513046F8F73AFF012223
:10900000AFA1201DFAF7A6FC68B10D2804D1DFF846
:10901000981400F0A8F904E002460FF2005100F0A5
:109020009FF9002070BD012070BDF8B5DFF87C0409
:10903000DFF87C44DFF86C643178041BE408240416
:1090400044F0010511B1DFF86C1414E044F003049E
:109050000FF2DC4100F07FF84FF40070009098A709
:1090600006F510734FF4806201213846FAF7FCFED2
:1090700018B10FF2D841284610E00FF28C4100F0F1
:109080006AF801223946301DFAF764FC002819BF3E
:109090000FF2C84128460FF2D4412046BDE8F44003
:1090A000F8F7E7BE2DE9F04300F058F8451BDFF86C
:1090B000F4030178ED082D0491B045F0010421B1CD
:1090C000DFF8F01300F047F836E00FF2A84145F062
:1090D0000300F8F7CEFEA1A106A8FAF761FE020090
:1090E00002D00FF2A8412DE0002645F005050DF154
:1090F00009070FF2E4480FF2D049694606A8FAF7CB
:1091000082FEE0B99DF8090038B19DF80800C1065B
:109110001AD53A46494600F023F9761CF8F7E4FEE2
:109120000028FBD19DF809000028E6D10FF2B441D8
:1091300032462846F8F7A0FE11B0BDE8F08302469B
:109140000FF268412046F5E7009A3B464146284623
:10915000F8F798FEE1E72046F8F78BBEDFF84C03FE
:10916000DFF84C53704770B50FF20861DFF83C63CD
:10917000DFF83C5391E81C00ADF5127D01A8751B8A
:1091800080E81C00C749CB4C0878ED082D0445F059
:10919000010610B1214630463DE000F0FDFA0346DD
:1091A0000FF25442102104A800F044FB45F00505DD
:1091B00004AA0FF250412846F8F75EFEF8F794FE35
:1091C0000028FBD10A2204A908A8FAF7F1FB020043
:1091D00018BF04F1380113D14FF4806401A8F9F7E6
:1091E000C3FD02466B4601A908A8FAF7BFFC641E3E
:1091F000F4D108A8FAF7BAFD50B102460FF22441A3
:109200003046F8F739FEF8F76FFE0028FBD104E08E
:109210000FF22C412846F8F72CFE0DF5127D70BD9B
:10922000704738B5A149A24C9E4D0C1BE40824049C
:10923000022844F003040CD003280FD008281CD0C7
:1092400009282BD00A2831D00D2809D00E280CD09F
:1092500031BDBDE83240002000F072BB002000E0CC
:109260000120BDE8324000F05DBBFFF7A1FEFCF736
:1092700025FEBDE8314000F071BB0FF2CC31FFF7A5
:109280006AFFF7F7C8FFC8B98B49FFF764FF0020F2
:10929000FBF720F9BDE83140FCF70EBE0FF2BC3100
:1092A000FFF759FFFCF730FE002006E00FF2C03157
:1092B000FFF751FFFCF710FE0120287031BD0000C0
:1092C000000000000E287D4A04D007D3102808D0E3
:1092D00005D3704701211046F9F70CBA70470221F7
:1092E000F9E70421F7E770B50FF294430FF28C31E0
:1092F00093E87000ADF50E7D01A80A2280E87000A9
:1093000004A8FAF755FB6949694D4D1BED082D047A
:1093100045F0030520B102460FF26C3100F020F851
:109320004FF4805401A8F9F71FFD02466B4601A9CE
:1093300004A8FAF71BFC641EF4D104A8FAF716FD82
:1093400020B102460FF25C3100F00AF80FF27431DE
:1093500000F009F80DF50E7D70BD00002F00000033
:109360002846F8F789BD2846F8F783BD2DE9F04176
:109370004FF480415248534CF8F708FC20B1224684
:1093800040F21721FDF7AAFE00F05CFBFDF7B5FDEA
:1093900020B1224640F21B21FDF7A0FE0020FDF780
:1093A000CDFD00F0A9FC20B1224640F22621FDF7B8
:1093B00095FE4549022000F065FE20B122464FF49B
:1093C0000A71FDF78BFE012000F012FBFFF7F0FDA4
:1093D00018B1FFF767FEFFF7C6FE0FF2B030FCF7DB
:1093E000EBFC20B1224640F23321FDF777FE04F179
:1093F0008400FCF7FEFE20B1224640F23721FDF743
:109400006DFEFFF7ABFE00BFB5A1451BED082D04B7
:1094100045F00305FFF7A7FFFCF738FD20B1224612
:1094200040F23E21FDF75AFEFCF79AFE0028FBD1E0
:1094300000212248F9F752F90646F00725D500BF6A
:10944000AEA10FF2F828FFF78EFFFFF7EEFD00BF89
:10945000AEA1FFF788FFFFF746FF00BFB1A1FFF7FE
:1094600082FF00277F1C3A464146FFF779FFFFF74E
:109470007AFEFA2FF6D300BFB8A1FFF774FFFFF70B
:1094800011FE04F13C01FFF76EFFB00748BFFFF784
:1094900009FE700748BFFFF7C8FDF8F725FD20BF9C
:1094A000C2E70000EC02002030E3000090D400008E
:1094B00058D400009CD9000074E50000482C00201E
:1094C000B15D000020D30000C5920000496E6974B0
:1094D00069616C697A696E67206469736B203020FA
:1094E0002851535049292E2E2E0000004469736BD9
:1094F00020696E697469616C697A6174696F6E2044
:109500006661696C65642E004D6F756E74696E6777
:1095100020766F6C756D652E2E2E00004D6F756E6A
:1095200074206661696C65643A202575000000004E
:109530000D0A4372656174696E672066696C6573B4
:10954000797374656D2E2E2E000000004D6B6673CE
:10955000206661696C65642E000000004D6F756EB9
:1095600074206661696C65642E000000446F6E654E
:10957000000000000D0A4C697374696E672064690D
:10958000726563746F72793A202F000044697265C6
:1095900063746F7279206C697374696E6720666199
:1095A000696C65643A2025750000000044697265A5
:1095B00063746F72792072656164206661696C659D
:1095C000643A2025750000002020203C4449523E8A
:1095D00020202025730D0A0025396C752020257365
:1095E0000D0A0000456E747269657320636F756EB5
:1095F000743A2025750D0A00253038782E74787459
:10960000000000004372656174696E672072616ECC
:10961000646F6D2066696C653A202573202E2E2EAE
:10962000000000000D0A556E61626C6520746F20A9
:10963000636C6F73652066696C653A202575000060
:10964000646F6E650D0A000055534220706F776598
:10965000722064657465637465640000555342202C
:10966000706F7765722072656D6F766564000000BB
:10967000555342207265616479000000746573740B
:10968000312E7478740000000D0A2331556E61622A
:109690006C6520746F206F70656E2066696C653A2A
:1096A000202575000D0A2331556E61626C652074AA
:1096B0006F20636C6F73652066696C653A20257551
:1096C000000000000D0A2054657374312E65787413
:1096D000206372656174656420446F6E65000000EC
:1096E00055534244204D5343206578616D706C653D
:1096F00020737461727465642E000000312E204660
:109700006F726D6174204469736B2E00322E20439A
:10971000726561746520546573742066696C652E8A
:1097200000000000332E2043726561746520526191
:109730006E646F6D2066696C65732E0046696C659A
:109740002063726561746520636F756E74286D6146
:109750007820323530293A2025640000342E204309
:109760007265617465642066696C65206C697374E8
:109770003A0000006162636465660D0A0000000043
:109780003132333435360D0A00000000000000008D
:109790002392000000000000F0B42249224AD1F8D0
:1097A000807056681078214C214D6FF0004320BB2B
:1097B000082005FB064637461E46B7FBF6F6401E58
:1097C00003FB1676F5D10F46102005FB06469C4696
:1097D000B6FBFCFC03FB1C6647F8046B401E05FB54
:1097E0000646B4461E46BCFBF6F603FB16C647F813
:1097F000046BEAD1CF6F0120107005FB06461C46B2
:1098000007F01F07B6FBF4F451F8270003FB1466BA
:1098100041F827605660C1F8800020F04040F0BC5D
:1098200070470000CC270020900700205FF36E3CBB
:109830000D66190008B438B585B009AC002504944C
:10984000039500290EBF01950190491E02910095D4
:1098500004AB01A9074878441A30FDF7E5FD0199EA
:1098600001B10D70002858BF039806B030BC5DF8F8
:1098700008FB00BFFF82FFFF10B5044620683028B8
:1098800004D3584940F2CD10F8F73EF820681F285D
:1098900002D84FF0A04010BD00F01F0020605248D9
:1098A00010BD2DE9F14181B0089D099C0E46174677
:1098B000984601A8FFF7E0FF46EA4706019946EA05
:1098C000880646EA052600EB810046EA0446C0F811
:1098D0000067BDE8F3811CB50124009000296846AB
:1098E00006D1FFF7C9FF00998C40C0F80C4513BDA5
:1098F000FFF7C2FF00998C40C0F8084513BD1CB5A6
:109900000446042C03D339493A20F7F7FDFF00F051
:1099100003F8D0F804054BE048A1085D00906846C4
:10992000AAE7000010B50446042C03D32F494120B8
:10993000F7F7EAFF41A0005DBDE810400021CAE74B
:1099400010B50446042C03D328494720F7F7DCFF61
:109950003AA0005DBDE810400121BCE710B500242D
:109960002046FFF7EDFF641C042CF9D310BD10B5A1
:1099700000242046FFF7D6FF641C042CF9D310BD49
:109980001CB50446042C03D318495F20F7F7BCFF2D
:10999000FFF7C2FF00F2045101230A68009C03FA9A
:1099A00004F494434C60009883401A408A6013BDCD
:1099B0000099C84000F00100401E8041C00F16BD54
:1099C0000000000010B501464FF0FF305FF00002CC
:1099D0001BA39C5C8C4203D0521C042AF9D310BDFB
:1099E000104610BDD8D4000000030050DCE3000096
:1099F000FEB50446E00710D55FF000050FA600276E
:109A0000019700970023705D01220121FFF749FFB4
:109A10006D1C042DF4D3FFF7A1FFA0070DD5002482
:109A200007A500200190002100910323285D00225A
:109A3000FFF737FF641C042CF3D3F7BD0D0E0F1096
:109A40000B0C181980B500F0C6FB04210648F8F786
:109A500057FB002803D505494820F7F755FF04496F
:109A60000120487101BD00BF4CEA00004CDA000043
:109A70004407002038B5DFF8684304F11C0000F00B
:109A80008EFDD4E902230021D4E904451018594180
:109A9000A94206D828BFA04203D2B0F17F4061F1AD
:109AA000FF3134BDD1E90223D0E902018B4204D356
:109AB00001D8824201D3012070470020704770B561
:109AC0000446606920B9DFF81C13A220F7F71CFFD9
:109AD000DFF80C0301780025012926D1002C1CBFDA
:109AE000207F002821D0FFF7C5FFD4E90223994247
:109AF0000FF2003614D301D8904211D3206900B977
:109B00002577A069616988472269002A1CBF207FE8
:109B100000280AD0D4E9020180186941C4E9020191
:109B20002146304600F070FD0125284670BD00003A
:109B3000B0A000F085BD2DE9FC4D804600F022FD6F
:109B4000A74D38B1D5E90201B0F17F4261F1FF3391
:109B5000C5E902230021404600F01CFD00281CBF7F
:109B6000A8690028DFF87CB216D0AE69404600F044
:109B700016FDD6E9022322F07F4100F02DF9B0F561
:109B8000960F04D3594640F22B10F7F7BDFEA86993
:109B9000FFF795FF0020A8610121404600F0FAFC84
:109BA00018B1FFF767FFC5E9040100F086F80FF26E
:109BB000442A0EE04168087F20B901220A77504606
:109BC00000F022FD694605F17C00FDF783F900F005
:109BD00074F808B301780029ECD002290CD0F1D236
:109BE0004168A869814207BF0021A961504600F081
:109BF0003FFDE7E700220277FFF79AFF0028F9D13F
:109C000001202870DEE7002105F11C0000F0BDFCFA
:109C10003046FFF754FFAF61504600F01FFD0028AB
:109C200044D0A96981B1D0E90201AA69D2E90262EE
:109C3000914240D828BFB0423DD2A869007F18B1F8
:109C4000A969504600F0E0FCFFF772FF0646FFF7F7
:109C500011FF02460B46D6E90201821A61EB0303AB
:109C600001240027BB42CEDB01DCA242CBD35E4CF9
:109C7000A24204D905F11C0000F091FC20440246E8
:109C80004FF49603002105F11C0000F005FC30B1F3
:109C90000D28BDD05946F520F7F736FEBBE7A86979
:109CA00010B9404600F085FBAE6104E0A86910B928
:109CB000404600F089FBBDE8F38D694605F17C0064
:109CC000FDF7DCB87CB504460D46454E694606F105
:109CD0007C00FDF7A1F868B104704560694606F1A3
:109CE0007C00FDF7BBF818B106F11C0000F05BFC2E
:109CF000002076BD042076BD1CB500BF40A0384CC6
:109D0000016800910823582204F1240104F17C0029
:109D1000FDF76EF8A8B9354A694604F11C0000F059
:109D2000D5FA70B9012104F11C0000F028FC0123D0
:109D30002F4A012104F11C0000F052FB0120207089
:109D4000002016BDF8B504000D461646254F04D177
:109D5000394640F22E20F7F7D7FD300006D13946BC
:109D600040F22F20F7F7D0FD0720F2BD2068012D2B
:109D70000CBF01210021466101610020F2BDF8B550
:109D800004000E46154604D1164940F23E20F7F76E
:109D9000BBFD207F08B10020F2BDA561FFF76AFE80
:109DA000002780197941C4E90201206900B12661C8
:109DB0002146BDE8F440002084E710B5040004D13A
:109DC00008494FF41570F7F79FFD00212177012016
:109DD0002146BDE8104075E7401A20F07F407047EB
:109DE00000000020F0DF0000FFFFB400379B000000
:109DF000FFFF7F0000000000402C0020A59A00001B
:109E0000010006002DE9F84380468946FFF7DAFD98
:109E1000002404282FD2DFF8206300EB40017518DE
:109E20003718B9F1000F14D0B9F1020F1AD01AD2B5
:109E30002C78687850B106F10F024FF4804106F19A
:109E40006000FFF79CFF08B986F80F80A878387487
:109E500009E006F16000FFF7B0FFAC78387CA04263
:109E600009D100E06C7820001CBFB169002902D044
:109E7000BDE8F4430847BDE8F18380B50078FFF7FB
:109E8000A1FD04280DD2DFF8B01200EB4000084419
:109E9000407802001CBF8969002902D0BDE8044057
:109EA000084701BD10B5DFF89012887B50B100243F
:109EB00001E0022C02D02046FFF742FD641C042C76
:109EC000F7D310BDBDE81040FFF748BD2DE9F041C4
:109ED000994C0746607B002510B16573FFF7E2FFE0
:109EE0003E46172E40F2666865D8DFE806F00C158E
:109EF00015242B36464C50585058AB656565656542
:109F000090949AA1ABABFFF7CDFF04F12000FFF7CF
:109F100054FF0546002093E000F0A2F830B100F0B5
:109F2000A2F8022F14BF854885481FE0FFF7FAFC0E
:109F3000022F1AD00FE000F093F8A0B100F093F8D0
:109F4000804813E000F08CF818B100F08CF87B48E2
:109F50000CE0FFF7E7FC7C4808E000F081F810B166
:109F600000F081F801E000F078F87848002100F076
:109F70006FF827730146002218E00020FFF700FD6C
:109F80000620207308E000F068F8072058E001215F
:109F900061730120FFF7F4FC0022414606E0012036
:109FA0006073FFF7EDFC00224FF4005104F1200034
:109FB000FFF7E5FE054648E004F14000FFF7FDFE2F
:109FC000D6F1110605461CD0DDB9012E14D9B6B262
:109FD000C8204643F717FF0347EA5647F60316F52E
:109FE0007A7047F1000100F033F80146002204F1D5
:109FF0004000FFF7C4FE05460220FFF793FC012056
:10A0000003E00220FFF79CFC0020A0731DE0FFF797
:10A0100049FF122014E0FFF745FF00F01EF813205F
:10A020000EE0FFF73FFF0120FFF77CFC142007E064
:10A03000FFF738FF00F011F80120FFF773FC15203F
:10A04000207302E0FFF793FC27732846BDE8F081F8
:10A050004FF4FA620023FEF767BE0020FFF762BCF0
:10A060000020FFF74CBC0020FFF76ABC3248017D9E
:10A07000CA0744BF007BFFF729BF70470220FFF7E4
:10A080007FBC000070B505462B4800244561816106
:10A09000A8071ED5002601220121304600F02FF826
:10A0A000761C042E044601D2002CF4D08CB940F268
:10A0B000333204212CA000F0CFFB04464CB900F051
:10A0C00002FC04462CB9224A26A00021FFF73AFEE2
:10A0D0000446E80711D50120FFF78AFC6CB91D4A38
:10A0E0001EA00021FFF72EFE044634B9DFF86820D9
:10A0F0001BA00121FFF726FE0446204670BD30B5A7
:10A1000003460020042B15D20B4C03EB4305012A18
:10A110002C4405D1012908BF03F10E0204D000220E
:10A1200031B1022902D005D2227030BD627030BD3B
:10A13000A27030BD072030BD50280020E803D007B2
:10A14000E8038403E8039001E803C800E80364001F
:10A150007B9E00006DA000007DA000007028002004
:10A1600090280020B02800200B000300059E00006E
:10A170000C000300059E000018000300059E00006F
:10A1800019000300059E0000304901200870704747
:10A1900038B588B00446684632A12022F7F7DCFBC8
:10A1A0004FF0FF31019102910391062500954FF088
:10A1B000EB710691220014BF254A0022234D694607
:10A1C000281D00F0B9FB18B1224A4321FCF786FF95
:10A1D0006C7009B030BD0120DAE770B51B4C1E4D24
:10A1E00000202070D2B22679AB5D23B104F10800C3
:10A1F00000F055FD03E004F1100000F0FEFF18B17F
:10A20000144A5321FCF76AFF617811B120780028C5
:10A21000FCD070BD80B5114A00924023104A01F075
:10A2200045F901BD704780B508490B4A0B79D05CF0
:10A2300020B101F1080000F0D1FC03E001F11000B1
:10A2400000F079FFBDE802400020A1E72C070020C4
:10A2500089A1000018DC0000BC2B0020DBA100005D
:10A26000802A0020FFFFFFFFFFFFFFFFFFFFFFFF30
:10A27000FFFFFFFF00000000000000000000D6010B
:10A2800006010000000000000000000000000000C7
:10A2900028B10FF26C31800141F00101084770478D
:10A2A00000EB8100C0F840257047C0F808137047E4
:10A2B00081B00022425040580090009901B0704790
:10A2C000C0F844137047C0F8481370472DE9F047B1
:10A2D0000400DFF8F4820D46164608F1F00703D1BA
:10A2E00039465520F7F710FB1DB939465620F7F7C8
:10A2F0000BFB1EB939465720F7F706FB6079DFF8EC
:10A30000CC92DFF8CC2209EB800109F104008E60C9
:10A310006179B04E10F83100961BF608360438B15A
:10A3200008F5987146F00200F7F7A3FD082037E022
:10A330002F88D4F800A0B7F5805F05D308F1780125
:10A340004FF4BE70F7F7E0FACAF80875AF7894F9E1
:10A350000450082F03DB41466B20F7F7D5FA78014C
:10A36000290006D59C4905F00F054A1902F8040C8E
:10A3700001E09A4B5855012294F90410984B00F0D3
:10A3800011F809F104006179012200F831206079A7
:10A3900096A149F8304046F00300F7F76AFD002027
:10A3A000BDE8F08701F01F008240490943F82120F1
:10A3B000704710B5040003D18A498720F7F7A4FA43
:10A3C00020680121016010BD10B5040003D185494A
:10A3D0008D20F7F799FA2068012140F8041F10BD7D
:10A3E0002DE9F04104000F4690461E4603D17D49F9
:10A3F0009620F7F789FA20684FF4803500F542710E
:10A40000BD400D600D64B90001F5A07109B2FFF700
:10A410004FFF206828F07F423946FFF741FF206850
:10A4200000F54170056406B10560BDE8F08170B5C6
:10A4300004000D46164603D16A49A920F7F764FACD
:10A4400020682946FFF73CFF16B12068C0F8045386
:10A4500070BD38B504000D4603D16249B320F7F74B
:10A4600053FA20682946FFF72EFF20682946BDE8E9
:10A4700034401AE738B504000D4603D15949BA20D3
:10A48000F7F742FA2068415921B12946FFF710FF3A
:10A49000012032BD002032BD2DE9F84F040088466E
:10A4A0001546994603D14F49CD20F7F72DFA4FF4C1
:10A4B000803000FA08FA51462046FFF7CAFF2068AC
:10A4C000D0F8047500EB88013A46D1F840B5414612
:10A4D0004FEA8806FFF7E4FE06F5A076206831B261
:10A4E000FFF7E6FEABEB070727F07F47012F25F0CC
:10A4F0007F4506D11020FFF7CBFE206831B2FFF771
:10A50000D7FE2068D0F80475C0F844A3E91B6E1C80
:10A5100021F07F41012913D132464146FFF7C0FEA9
:10A520001020FFF7B5FE2068D0F80405874224D13B
:10A53000012251462046FFF77AFF0020BDE8F28F46
:10A540002A464146FFF7ACFE2368D3F804756D1E1A
:10A55000ED1B6FF07F4125F07F45A1EB0900A8427C
:10A560000BD3002DE4D1324641461846FFF798FE42
:10A570002068D0F804058742DAD00D20DEE70A46CD
:10A58000022154E74FF4827174E74FF4803202FAEB
:10A5900001F15EE7890001F5A07109B26AE7006880
:10A5A000D0F80405704790F904100F4B012201F018
:10A5B0001F008240490943F8212070470349086879
:10A5C000896808470000000058C80000EC2B0020F4
:10A5D00060D4000058D4000018ED00E000E400E072
:10A5E00000E100E048C9000000E200E05254433AB4
:10A5F00020696E697469616C697A65642E00000077
:10A600000338FDD87047000070B505000C46264E93
:10A6100003D131463A20F7F777F91CB931463B2090
:10A62000F7F772F96E6800E03668306820B1AA6802
:10A63000214690470028F7D130682060346070BD13
:10A6400010B5040003D118495120F7F75DF962688D
:10A65000116808001CBF0968116010BD10B5040026
:10A6600003D111495D20F7F74FF96068006810BD0C
:10A6700070B505000C460C4E03D131466920F7F742
:10A6800043F91CB931466A20F7F73EF96A680021A0
:10A6900000E00246106820B1A042FAD120681060A4
:10A6A0000121084670BD0000CCDD000010B5914BC3
:10A6B000C20703EB500052BFF0220F2209010479B8
:10A6C00022401143017110BD38B58A4A136B002135
:10A6D00000E0491C1478A14206DA13F83150A84270
:10A6E000F7D103EBC10032BD83498820F7F70CF99D
:10A6F000002032BD38B504460D46FFF7E5FF0028BF
:10A700001CBF4268002A04D029462046BDE83840D4
:10A71000104731BD2DE9F8430E46DFF8D88108EB2C
:10A72000500181460F795FEAC9704CBF3F0907F0BD
:10A730000F07012000214A4600F01EFF042F0446A7
:10A740000D4642D8DFE807F0031116222500002E3F
:10A750003BD001214846FFF7A9FF0020F7F70FF98A
:10A76000D8E90A012043294328E0002E0CBF00212C
:10A77000022110E046B103214846FFF797FF484603
:10A78000BDE8F4430121B5E7012104E0EEB904215D
:10A7900001E026B103214846BDE8F44386E70021E5
:10A7A0004846FFF783FF00214846FFF7A3FF00203C
:10A7B000F7F7E5F8D8E90A01A043A943C8E90A0177
:10A7C000BDE8F2430020F7F7E9B8BDE8F183494856
:10A7D000416B002249083830FFF7D1BA70B5002428
:10A7E000444D12E0002108E0296B01EBC4063078EB
:10A7F00001F0BDF871780129F4D14140491E894129
:10A800003078C90FFFF786FF641C28788442EBDBA1
:10A81000D5E90A23002B08BF002A02D0BDE870400A
:10A82000D5E770BD10B5C0B2FFF74EFF04462078E3
:10A8300001F09DF86178012918BF002190EA010F0D
:10A8400002BF2C48D0E90A23002B03D112B9BDE87E
:10A850001040BCE710BD0000F8B516460A2E0446AD
:10A860000D4601D20720F2BD00F0BCFF10B900F088
:10A8700084FF38BB1F4F20213C633D707E63381D31
:10A88000FBF784FE0020C7E90A001C4E1EA72846DD
:10A89000451EC0B280B138680090E8B204EBC00138
:10A8A0008A788DF80120324614F83000694600F0AD
:10A8B000A5FF0028EBD0F2BDDFF8442011A0002155
:10A8C000FFF740FAF2BD38B50A4C206B20B90A49AF
:10A8D00040F23510F7F718F8002506E0206B10F865
:10A8E0003500012100F0EFFF6D1C20788542F5D383
:10A8F000002032BDE829002014DE000025A8000059
:10A90000DDA70000202A002003000000F8B500E0C9
:10A91000F8B502788DF800204368019382688DF8BD
:10A920000820C068214A039002EB81026846D16882
:10A930005268904705B000BD2DE9F041044688B04B
:10A940002678DFF8688008EB86000F4615464560DC
:10A95000012E3969C16004BF787F002803D11449F2
:10A960007620F6F7D1FF787F08F80600394668466A
:10A970002022F6F7F1FF0496217818F8010040B183
:10A98000002D14BF0B4A00226946201D00F07BF801
:10A9900008E0002D14BF084A0022694604F10C00AB
:10A9A00000F028FB08B0BDE8F0810000BC2B0020BF
:10A9B00070E100000DA9000011A9000081B0002283
:10A9C000425040580090009901B070474058DFE174
:10A9D00000F20C5001E000F5A16001608260704758
:10A9E00010B504462068302805D3DFF8E41440F29F
:10A9F000CD10F6F789FF20681F2802D84FF0A0403D
:10AA000010BD00F01F002060DFF8C80410BD2DE964
:10AA1000F14181B0089D099C0E461746984601A851
:10AA2000FFF7DEFF46EA4706019946EA880646EA4E
:10AA3000052600EB810046EA0446C0F80067BDE841
:10AA4000F381E0B500F00FF8012105E0E0B50B4619
:10AA50000021002201910092FFF7D9FF07BDE0B568
:10AA600000F001F8F8E70021019100910023012294
:10AA7000704701B56846FFF7B3FF009901228A408D
:10AA8000C0F8082501BD2DE9F0410C000546164629
:10AA9000DFF8448404D108F17801CF20F6F734FFC1
:10AAA0002979DFF83824242313FB01F3D71897F80A
:10AAB000200008B108208FE00FF2504050F821101C
:10AAC000286801F04BF808B1112085E0206810F1EA
:10AAD000010F04D0FFF7CDFF2068FFF7B2FF6068D9
:10AAE00010F1010F1CBF0021FFF7B0FF2868A1691A
:10AAF00000F224521160637D217D0B4393646268F0
:10AB00002168FFF765FF207D012814D1A06810F1AE
:10AB1000010F1CBF0021FFF799FFE06810F1010F42
:10AB200004D0FFF7A6FFE068FFF78BFFA268E1689B
:10AB30002868FFF750FF7E60786821693960002837
:10AB40003ED0267F28684FF48871FFF737FF2868CA
:10AB50004FF49071FFF732FF28684FF49271FFF7BE
:10AB60002DFF28684FF4A271FFF728FF286800F036
:10AB700006F92C68DFF86803C4F8040324032416DC
:10AB8000082E03DB41466B20F6F7BEFE7001002C59
:10AB900007D5DFF8501304F00F040A1902F8040C6B
:10ABA00002E0DFF84413085501222968DFF83C333E
:10ABB0000903091601F01F008240490943F82120CA
:10ABC00008202968C1F800050022BA61FA617A619B
:10ABD000012087F820000020BDE8F0812DE9F8432E
:10ABE00000F0F9F82268686870B1DFF8F412DFF855
:10ABF0000063C2F8081301231103091601F01F00B6
:10AC00008340490946F821300123D2F8000220F0A0
:10AC10002000C2F8000253604FF4AC711046FFF7F9
:10AC2000CDFE20680122C26000F0D1F80028FBD0E0
:10AC30000022206800F5A0610A604FF0FF32CE6864
:10AC40004F69D1F80880D1F810901146FFF7C0FE87
:10AC50004FF0FF3220681146FFF7BDFE16F1010FDD
:10AC60001CBF3046FFF7FBFE17F1010F1CBF384633
:10AC7000FFF7F5FE19F1010F1CBF4846FFF7EFFE85
:10AC800018F1010F1CBF4046FFF7E9FE206800F0F5
:10AC900084FF002085F820006860BDE8F1832DE97D
:10ACA000F0410646154632790C462420DFF82C1276
:10ACB000DFF8248242438F1897F82020012A05D01C
:10ACC00008F1780140F22D10F6F71EFE2CB908F1BC
:10ACD00078014FF49770F6F717FE2DB908F1780157
:10ACE00040F22F10F6F710FE307910B9B5F5803F1D
:10ACF00005D308F178014FF49870F6F705FE04F0DB
:10AD00006040B0F1005F26D1304600F03BF820BB38
:10AD10007D61BC604FF490713068FFF74FFE306882
:10AD200000F02DF878693168BB6801F244520025C3
:10AD30001360506001228A607868C8B930684FF4A7
:10AD40009071FFF743FE044600F015F80443F5D078
:10AD500028B10F250AE010200BE0112009E031682E
:10AD60000120C86000F007F80028FBD000207861BF
:10AD70002846BDE8F08130684FF4AC7126E64FF408
:10AD8000AC711BE60279554924204243881840697A
:10AD900000B10120C0B270471FB5034601240291E3
:10ADA0008DF800400192684619685A6890471FBDA7
:10ADB000F8B5024600238DF80030029190680190AA
:10ADC0005361684611685268904705B000BD20681D
:10ADD0004FF4AC71FAE50446242122793F484A43F6
:10ADE000851870477FB5434E4FF4927100F08AF892
:10ADF0003A4C414DB0B14FF4927100F085F8022009
:10AE00008DF800003D480168016003910021286829
:10AE100062680290A161E161E06821680190684682
:10AE200090471FE04FF4887100F06CF8D0B14FF4F8
:10AE3000887100F069F82968A069814212D1E2683E
:10AE4000E06958B12E48036823F020030360E069ED
:10AE50002369A061E3600020E06100E0A06120467A
:10AE6000FFF79AFF4FF4A27100F04CF868B14FF46D
:10AE7000A27100F049F8A06938B10021A161E16137
:10AE800020462968E268FFF787FF4FF4907100F0D1
:10AE900039F858B14FF4907100F036F80121F160A3
:10AEA000606918B129692046FFF782FF4FF4AC7141
:10AEB00000F028F848B14FF4AC7100F025F8606953
:10AEC00018B129692046FFF773FF7FBD000000001D
:10AED000B8D6000000030050B0D100004C2B002079
:10AEE0001003420018ED00E000E400E000E100E0A3
:10AEF00080E100E0002000403C250040802400402C
:10AF000000220040304661E5304657E5E5AD0000DF
:10AF100081B00022425040580090009901B0704723
:10AF20004058D9E1D0F80403084018BF0120C0B24E
:10AF3000704700F20C5082600160704700F5A1601C
:10AF4000016082607047D0F81805C0B2704710B534
:10AF500004462068302805D3DFF8141540F2CD10E0
:10AF6000F6F7D2FC20681F2802D84FF0A04010BD91
:10AF700000F01F002060DFF8FC0410BD2DE9F14156
:10AF800081B0089D099C0E461746984601A8FFF718
:10AF9000DEFF46EA4706019946EA880646EA0526A4
:10AFA00000EB810046EA0446C0F80067BDE8F38183
:10AFB000E0B500F00FF8012105E0E0B50B460021F7
:10AFC000002201910092FFF7D9FF07BDE0B500F024
:10AFD00001F8F8E700210191009100230122704758
:10AFE00001B56846FFF7B3FF009901228A40C0F817
:10AFF000082501BD2DE9F8430C0006461546DFF88B
:10B00000789404D109F17801AA20F6F77DFC317912
:10B01000DFF868042C2212FB01F2871807F12908D7
:10B0200098F8010008B1082083E00FF27C4050F846
:10B030002110306800F092FD08B1112079E02068FD
:10B0400010F1010F04D0FFF7CBFF2068FFF7B0FF2E
:10B05000606810F1010F1CBF0021FFF7AEFF3068E0
:10B06000A16900F224521160637D217D0B4393643A
:10B0700062682168FFF75DFF207D012814D1A06878
:10B0800010F1010F1CBF0021FFF797FFE06810F1DE
:10B09000010F04D0FFF7A4FFE068FFF789FFA26863
:10B0A000E1683068FFF74AFF7D60216978683960A0
:10B0B00088B3257F30684FF48E71FFF729FF306821
:10B0C0004FF4A271FFF724FF3468DFF8B403C4F82B
:10B0D000040324032416082D03DB49466B20F6F7EE
:10B0E00013FC6801002C07D5DFF8981304F00F0457
:10B0F0000A1902F8040C02E0DFF88C13085501224B
:10B100003168DFF888330903091601F01F00824017
:10B11000490943F8212004203168C1F800050022C4
:10B12000BA61FA6188F800207A61012088F801008C
:10B130000020BDE8F2832DE9F84304462C20227953
:10B14000DFF83813236842438D1803F5A06100220D
:10B150000A60686870B1DFF83823DFF83873C3F825
:10B16000082301261A03121602F01F008640520916
:10B1700047F822604FF0FF32CE684F69D1F808805F
:10B18000D1F8109011461846FFF7D3FE4FF0FF326A
:10B1900020681146FFF7D2FE16F1010F1CBF3046A2
:10B1A000FFF714FF17F1010F1CBF3846FFF70EFF22
:10B1B00019F1010F1CBF4846FFF708FF18F1010FF6
:10B1C0001CBF4046FFF702FF206800F0E6FC0020AD
:10B1D00085F82A006860BDE8F18338B50D4604465D
:10B1E0004FF48E71FFF794FEA868296A405C2A6AC2
:10B1F000521C2A62C4F81C0531BD2DE9F8430746EC
:10B2000016463A790D462C20DFF87012DFF8689266
:10B2100042438C1804F1280898F80200012805D050
:10B2200009F178014FF48C70F6F76EFB2DB909F136
:10B23000780140F21910F6F767FB2EB909F1780191
:10B240004FF48D70F6F760FB384600F03EF808B119
:10B25000112038E06661A5602062002188F80010A6
:10B260004FF48E713868FFF753FE38680121816012
:10B2700000252146FFF7B1FF606818BBD7F80090A2
:10B28000666903E021464846FFF7A7FF206AB042FF
:10B290000CD24FF48E714846FFF742FE0028F1D1E0
:10B2A00098F800000028F4D00F2509E038684FF422
:10B2B0008E71FFF735FE0028F8D039680120C8608C
:10B2C000002060612846BDE8F2830279DFF8AC1106
:10B2D0002C2042438818406900B10120C0B2704759
:10B2E00070B50D460446A86900284FF484712046C5
:10B2F00005D1FFF70DFE2046BDE8704023E6FFF7BD
:10B3000007FE6E6A2046FFF71EFEE9688855686AE8
:10B31000401C686270BD1FB50346012402918DF880
:10B3200000400192684619685A6890471FBDF8B5F9
:10B33000024600238DF8003002919068019053611D
:10B34000684611685268904705B000BD2DE9FF417D
:10B35000514D4FF400712846484C504FFFF7E2FD25
:10B3600004F128064FF4017810B34FF4927100F005
:10B3700099F8E8B14FF492712846FFF7C9FDC7F874
:10B380000080707808B90121696002208DF8000002
:10B3900043480168016003910021A069626802903E
:10B3A000A161E161E068216801906846904729E069
:10B3B00004212846FFF7B6FD20B34FF4847100F056
:10B3C00071F8F8B121462846FFF78AFFA069616A43
:10B3D000884217D1E06940B1E268616AA061002348
:10B3E0002069E060E361636209E0707808B90121D7
:10B3F0006960C7F800800020E268A061616A2046A9
:10B40000FFF789FF4FF48E7100F04CF8A8B1606926
:10B41000216A814206D2307820B921462846FFF7BA
:10B42000DCFE0AE04FF48E712846FFF771FD60697B
:10B4300018B161692046FFF77AFF4FF4A27100F05E
:10B4400031F888B14FF4A2712846FFF761FD70789A
:10B4500008B101212960A06930B10021A161204615
:10B46000E268616AFFF757FFBDE8FF810000000056
:10B4700040D6000000030050F8D00000BC29002096
:10B480008000020018ED00E000E400E000E100E0D0
:10B490008402020080E100E0002000400823004018
:10B4A0008024004028463BE54DB30000F0B595B040
:10B4B0000D461A9C16461F462846F7F783F809A83A
:10B4C0001821FBF763F809960A970E9400230C22C3
:10B4D00001A92846F7F7E4F80398BDF80A1004908C
:10B4E0000C26BDF80800ADF8140000220198ADF854
:10B4F000161000F0030001288DF8192017D10198CB
:10B50000019CC0F3C2008DF818000C230198C0F311
:10B510008316B2000FA92846F7F7C2F809A80090D1
:10B5200004AB32460FA9A00AF6F71EFF1FE00198F0
:10B5300000F0030002281AD10198019CC0F3C20058
:10B54000A40D8DF818000827082C98BF274633460D
:10B550003A4607A92846F7F7A3F809AB04AA3946E3
:10B5600007A8F6F749FFBE19E41B002CEBD12846CB
:10B57000F7F72CF815B0F0BDD2B2203A22BF00FA8E
:10B5800002F1002070475242D041D2F12002914096
:10B590004140D040904041407047FEE700F180407C
:10B5A00000F5C0400068012818BF002070471CB596
:10B5B000044600F009F800210160204600F004F87C
:10B5C00000680090009913BD00F1804000F5C04074
:10B5D000704710B504462068302805D3DFF83415CD
:10B5E00040F2CD10F6F790F920681F2802D84FF0EE
:10B5F000A04010BD00F01F002060DFF81C0510BD4A
:10B600002DE9F14181B0089D099C0E4617469846E8
:10B6100001A8FFF7DEFF46EA4706019946EA8806D9
:10B6200046EA052600EB810046EA0446C0F80067BA
:10B63000BDE8F38111B581B00C4601A8FFF7C9FF41
:10B6400000F5E060019950F8212022F4403240F8E2
:10B650002120019A50F8221041EA044140F82210BA
:10B6600013BD01B500F007F800F007F80099C840D5
:10B6700000F0010002BD6846ABE7D0F81005704746
:10B68000FEB516460FF2B4420446D2E90037CDE9C2
:10B6900000370D19032D0DD3DFF8781440F2FD208B
:10B6A000F6F732F906E05DF82400D0F8100546F808
:10B6B000040B641CAC42F6D3F7BD0246012002F035
:10B6C0000703D2089840895C0840704710B5C2084B
:10B6D00001248B5C00F0070004FA00F01843885442
:10B6E00010BDDFF83814084490F93020082A804152
:10B6F000C00F7047DFF82414084490F93020082A5E
:10B7000001DB0120704700207047DFF81014084467
:10B7100090F93020D043C00F7047DFF80414D5E70C
:10B72000F0B5034614004FF0FF3007BF08240C2586
:10B7300000240825DFF8E46300E0641CAC420ED26C
:10B7400056F8247017F1010FF7D1F01880F8304047
:10B7500046F8241012B9301980F85830204640B20B
:10B76000F0BDDFF8B8134FF0FF3241F82020082871
:10B77000A4BF081880F85820704738B5DFF89C43FC
:10B7800094F86A0008B1082032BD4FF0FF31C2B210
:10B79000401C2244C3B2302B82F83010F7DB002566
:10B7A000E8B2FFF7DEFF6D1CE8B20C28F8DB0621DB
:10B7B00004F16400FAF7EAFEDFF86813DFF8683393
:10B7C000C020087040221A604FF4BE70FFF7EFFEF1
:10B7D000DFF858134FF000400860012284F86A2017
:10B7E000002032BDDFF8340390F86A0000B1012078
:10B7F0007047DFF828030519204672E7FEB50546B5
:10B80000302D0F46164605D3DFF8241340F20720EB
:10B81000F6F77AF82846FFF778FF002408B10824E5
:10B820004FE0BA78520802F0010231462846FFF78D
:10B8300077FF064616F1010F42D0B878410719D4B8
:10B84000C0070CD50095FFF716FF009900EB8100AB
:10B85000D0F8002722F00202C0F8002707E00021FC
:10B860000194009100227B782846FFF7C9FE284604
:10B87000FFF753FFB878810716D53978DFF8B4227F
:10B88000DFF8B40252F82630034042F826302D0289
:10B89000090452F8263005F47C5501F440310D437B
:10B8A0001D4342F826500CE0DFF870023B57811927
:10B8B000304491F8582042EA831280F8582000E082
:10B8C00004242046FEBDF8B50446302C0E46DFF8B1
:10B8D000605204D3294640F23720F6F715F8204687
:10B8E000FFF713FF20B929464FF40E70F6F70CF856
:10B8F0002046DFF82852FFF7FDFE2F19B8B197F95F
:10B900003000284490F958000006800F032804D125
:10B910002046FFF7A6FE10B103E0012801D1022165
:10B9200000E003212046BDE8F440FFF783BEFFF7A7
:10B9300063FFD8B197F930407E4850F8241041F0A9
:10B94000010140F82410A00000F5807000B2FFF75C
:10B950002EFE002E1EBF97F9301055F8210000284A
:10B9600004D00121714801FA04F40460F1BD10B55E
:10B970000446302C04D36E494FF42270F5F7C4FF0F
:10B980002046FFF76EFE00B10120C0B210BD2DE9C8
:10B99000F84F88B00025CDE900554FF48076012797
:10B9A000082430B2FFF7FAFD00281EBF5F48006888
:10B9B000384203D030B2FFF7FAFD3D437F00361D19
:10B9C000641EEED14FF4BE70FFF7E8FD50B14FF4A6
:10B9D000BE70FFF7ECFD6A4602210020FFF750FE23
:10B9E00045F0004528064D4F19D001264FF00008BC
:10B9F000504C2E420DD054F8280054F8281057F817
:10BA00002820130005D0090C01F00301C0F3052024
:10BA10009047760008F10108B8F1080FE9D3002D2E
:10BA200073D504A90020C1E900004FF0FF31029155
:10BA3000039106E0069A049B0598009202930191F7
:10BA400003904FF0000AD14607EB090090F960001F
:10BA5000C5B210F1010F25F0C00440D002A9204664
:10BA6000FFF72BFE00283AD03819C5F3811590F95D
:10BA7000300057F82060310002D1032D2FD101E0B2
:10BA8000032D03D104A92046FFF720FE069406A843
:10BA9000FFF79FFD069900EB81006946D0F800078B
:10BAA000000C00F0030B2046FFF707FE18B1BBF1B6
:10BAB000020F14D102E0BBF1030F10D1032D09D105
:10BAC000BBF1020F0CBF032102212046FFF7B2FD9C
:10BAD0000AF1010A300002D029462046B04709F198
:10BAE0000109B9F1040FAFD35FFA8AF000280CD036
:10BAF00006AA02210020FFF7C3FD0698009A0799C5
:10BB0000904204BF0198814294D109B0BDE8F08F02
:10BB10000000000050D50000000300505029002014
:10BB2000B429002006E400E000E100E004630040E6
:10BB300030E2000010650040FFC0FCFF0000005034
:10BB40000003005010B51B4C206818B91A49512049
:10BB5000F5F7DAFE2168BDE81040084738B50D4614
:10BB600028B915497720F5F7CFFE002032BD1349DB
:10BB70008842FAD10020F5F702FF0E490879002427
:10BB8000002811BF01240D60012008710020F5F785
:10BB900005FF002CE9D0112032BD18B906499B20C1
:10BBA000F5F7B2BE0549884203D10248002202607F
:10BBB00002717047382C0020B0E2000000200040E5
:10BBC0002DE9FE43DFF840060C460168A14263D12F
:10BBD000E36ADFF838861D4605F12C062978891EB0
:10BBE000032905F1080700F2B480DFE801F00256EE
:10BBF0006B6B707800283ED0FE6839683A69D7F8D8
:10BC0000288001FB06F04FEA103902EB060C01FB1D
:10BC10000CF04FEA103EC84528BFC6452BD37869C3
:10BC20004FF48057C145B7FBF1F70DD1B6FBF7FCD8
:10BC300007FB1C66BF1B4E43BA4288BF3A464A43C5
:10BC400003F13801314414E007FB08F9A9EB0606BB
:10BC50004E43C645304408D1BCFBF7FE07FB1EC768
:10BC6000BA4288BF3A464A4301E04FF4805203F19A
:10BC70003801F5F771FE01212970E86800286DD0C0
:10BC80000FF2905090E84C00694605F1140781E8E6
:10BC90004C00019700F023F960E0296A3868726867
:10BCA0004143090B914203D04146CF20F5F72CFECA
:10BCB00005F12001204600F07FF900284ED04146D2
:10BCC000D32049E0B0682A7890FAA0F1052AB1FAA9
:10BCD00081F104D1012303FA01F14840B060B0685A
:10BCE00028BB686A70B12A6A38684243120B7260D6
:10BCF0000321297012034FF4805105F1380000F040
:10BD000059FC2BE001202870E96869B1307858B9F6
:10BD10000FF20C5090E88C00694605F1140081E8A0
:10BD20008C00019000F0DBF80020307016E090FAF3
:10BD3000A0F0B0FA80F039687268C0B2484300EBF6
:10BD4000023205F13803052418442C7000F011FC70
:10BD500004E0414640F21910F5F7D6FDBDE8F7833F
:10BD6000C06A00E030BF01780129FBD170472DE99E
:10BD7000F041040086B00D46904605D1DFF88C14E2
:10BD800040F22B10F5F7C0FD2069E76A010601BFFC
:10BD90004FF48052B2FBF0F25043D0F5805045D1C1
:10BDA000DFF86464306808B111205FE02246DFF8F4
:10BDB000601404F1180000F0DEFA002856D10FF2EA
:10BDC0006C42D2E90001CDE9010100F052F80028EF
:10BDD0004CD199208DF8040000F04BF8002845D193
:10BDE00003216846FAF7D2FB9F2104228DF8041044
:10BDF0008DF8052000216A4601A800F049FBA8BB88
:10BE0000684600F059FC88B18168B1F5805F0DD1BA
:10BE100022694068B0FBF2F141B14FF48053B3FBAB
:10BE2000F2F0B1FBF0F300FB131008B106201DE0A7
:10BE3000BA607960C7F81080FD60012038704FF05B
:10BE4000FF313963207D00F0010087F82D00346058
:10BE5000F86850B103A900200022002381E80D00FA
:10BE60003D6905952046FA689047002006B0BDE878
:10BE7000F0810022002101A800F00ABBFEB50400F9
:10BE800005D1DFF8881340F2AB10F5F73DFDE56A08
:10BE9000287801281CBF2046FFF762FFDFF868639F
:10BEA0003068A04204BF2978012901D01120FEBDCD
:10BEB000E86840B10FF27C3090E88C00694681E878
:10BEC0008C0000F00CF80020287000F02FFB41F2ED
:10BED00038012846FAF75AFB00203060FEBD286979
:10BEE00002902046EA6810472DE9F04104000D4613
:10BEF000C64E04D131464FF4EE70F5F705FD25B975
:10BF0000314640F2DD10F5F7FFFC00F02FF938BFA5
:10BF1000102027D3BC480168A14206BF3278012A0D
:10BF200011201FD100F029F995E8005187E8005150
:10BF300002253570B168326A706A4A434143B06A7B
:10BF400000F038FB10B1012131700BE0B06200212C
:10BF5000F068716228B9317801291CBF2046FFF7CB
:10BF6000FFFE0020BDE8F08170B5C36A93F82E0093
:10BF700003F1300298B950689968146890FAA0F0FB
:10BF8000B0FA80F0C0B24843052600EB04321D1819
:10BF90001E7005F13800BDE8704000F0EABA0420D8
:10BFA00011681870002283F82E200903BDE8704044
:10BFB000002000F02ABB00002DE9FF4705460E4691
:10BFC000EF6A3468BA68D6F80480D6F808A04FF44F
:10BFD0008050B0FBF2F0B4FBF0F100FB1144001B09
:10BFE0005443804588BF804602FB08F919F0030FCF
:10BFF00004D0864940F22620F5F786FCE96A081944
:10C0000000F1380200234FEA99004FF0010CD2F8FA
:10C0100000E0DAF80090CE450FD0D1F80890B4FBDC
:10C02000F9F90CFA09F91EF1010FD1F834E049EAE7
:10C030000E0E18BF0123C1F834E0241D5AF804EB9A
:10C0400042F804EB401EE2D107F12D020BB182F859
:10C0500001C07068A0EB0800706031684144316035
:10C06000B968B06801FB08F3C118B160507850B1ED
:10C07000B868796B4FF48053B3FBF0F00CFA00F022
:10C08000401E08437863796B09B11078B8B1F8683D
:10C09000A8B1706898B900BF69A090E81C00694613
:10C0A00007F1140681E81C0001960121386902900D
:10C0B00039706946FA6828469047002002E0284611
:10C0C000FFF752FF04B0BDE8F0872DE9F04104000E
:10C0D0000D464E4E04D1314640F29B20F5F714FC3C
:10C0E00025B931464FF42770F5F70EFC00F03EF805
:10C0F00038BF102038D344480168A14206BF3278C7
:10C10000012A112030D100F038F895E8005187E875
:10C110000051326AB068316B4243120B8A4205D13A
:10C1200006F120012046FFF747FF10E096F82D00AA
:10C1300018B12046FFF718FF09E032630320307082
:10C1400012034FF4805106F1380000F033FA10B1B9
:10C150000121317008E0F06828B9317801291CBF4D
:10C160002046FFF7FDFD0020BDE8F081E66A2A6861
:10C170006868716882189142704795E80E0006F170
:10C18000200006F1140780E80E00704770B5050026
:10C190000E46144604D11D4940F2F620F5F7B4FBD3
:10C1A000E86A16B1012E1BD021E00178012901D0E7
:10C1B000112070BD00F12C06707800281CBFB068FB
:10C1C000002803D18CB1002020700EE02846FFF734
:10C1D000CBFE68B90CB1012121700122327070BD13
:10C1E0000CB9072070BD281D2060002070BD0620FE
:10C1F00070BD10B5040004D104494FF44C70F5F73C
:10C2000083FBE06A001D10BD4C2C0020F8D9000013
:10C21000C1BB0000020000000000000000000000A0
:10C2200003000000000000000000000066010101A2
:10C2300001010000010000000000000000000000FB
:10C2400003000000000000000000000000000000EB
:10C25000012242507047405800B10120C0B27047DF
:10C2600010B50023891E072900F5C7641BD8DFE835
:10C2700001F01714110F0C090604D3791B069079ED
:10C2800043EA0043507943EA002310790343636093
:10C29000D0780306907843EA0043517843EA0123BB
:10C2A00010780343236010BD00F5C763891E5868EA
:10C2B0001B68072900D9704710B5DFE801F0110F9E
:10C2C0000D0B0A080604010ED171040C9471010AC9
:10C2D00051711071180ED070190C9170180A5070AD
:10C2E000137010BDD0F8340600F44030B0F5803F34
:10C2F00001D10120704700207047090241F48031CC
:10C300000AB141F40031C0F83416704738B5DFF88F
:10C3100050430146607908B1112032BDDFF8443343
:10C3200000221A60206820B10122DFF83C336271DC
:10C330001A60DFF838532846FFF78AFF206830B9C3
:10C340004FF480712846FFF786FF0028F8D00020C0
:10C3500032BD10B5642400F07EF950B90FF25031AF
:10C360004FF4207041F001018847641EF3D10D2085
:10C3700010BD002010BD2DE9F84304000D46904685
:10C38000DFF8EC9204D109F178018320F5F7BCFACB
:10C39000DFF8CC62307908B1082077E02079FF28F7
:10C3A0001CBF6179FF293CD0A179FF291CBFE1792D
:10C3B000FF2936D0DFF8BC7278624FF0FF31607928
:10C3C000FF2808BF0846B862A079FF2808BF0846C2
:10C3D0003863E079FF2808BF08467863207AFF2891
:10C3E00008BF0846B863607AFF2818BF0146F963A2
:10C3F00020683864A17AE07A227B41EAC001607B40
:10C4000041EA821178B9DFF87022DFF870027964AE
:10C410001368A17B0340E07B0B4338B143F080738A
:10C4200004E0072032E041F08001ECE7207C617CF1
:10C4300043EA406343EA0173136000207071356082
:10C44000C6F808800121DFF8380201607DB1A47CC4
:10C45000082C03DB49466B20F5F756FADFF8240277
:10C46000DFF82422640104704FF400711160012090
:10C4700030710121DFF8EC0139600022DFF8EC11A6
:10C48000026001230B60BDE8F14362E7BDE8F2837F
:10C490002DE9F843DFF8C861DFF8D4810746307929
:10C4A0000C46154620B908F17801B020F5F72CFAB2
:10C4B000707908B1112037E0DFF8A861DFF8AC919E
:10C4C000306024B1797822464846FFF7C9FEDFF88C
:10C4D000B011012008603A787878B97842EA0022F1
:10C4E000F87842EA0132397942EA4032787942EA10
:10C4F0008132DFF8981142EAC0320A60FFF729FF63
:10C500000D2808D1387920B908F17801C920F5F74C
:10C51000FBF90D2008E00020306025B179782A462B
:10C520004846FFF7C1FE0020BDE8F28338B54C4C09
:10C53000207920B9564940F24F10F5F7E5F94B4DF7
:10C540002846FFF7CFFE20B1012201212846FFF740
:10C55000D4FE4B49474A4F4B01200860286168656B
:10C56000002111604FF400703E4A18601160217183
:10C5700031BDF8B500F03FF828B907F1780140F275
:10C580006710F5F7C1F92CB907F178014FF4B470D1
:10C59000F5F7BAF904F06041B1F1005F08BF14F09B
:10C5A000030F05D13C490E604C608D60082029E0E6
:10C5B0001020F2BDF8B500F01EF828B907F1780197
:10C5C00040F27710F5F7A0F92CB907F178014FF494
:10C5D000BC70F5F799F904F06041B1F1005F08BF54
:10C5E00014F0030F05D12D490E604C608D600420BE
:10C5F00008E01020F2BD0D4619491D4F0446087988
:10C6000016467047BDE8F24080E638B50D4614493D
:10C610000446087920B91E494FF4C370F5F774F940
:10C6200015F0030006D11E48056044600C20BDE8EB
:10C6300032406BE6102032BD80B500F00CF848B1F6
:10C64000074A084B00205071186091681268BDE8D5
:10C650000840104701BD4FF480710448FBE500001D
:10C66000F82B002000910240049302400090024009
:10C6700088CF0000009502400096024000FFFF00B6
:10C680000893024029E400E004E100E0349602400F
:10C6900000D0000084E100E01095024004950240C3
:10C6A0001C95024000000000000000000000000097
:10C6B0000338FDD87047000010B5014604A40322DA
:10C6C0002046FAF71BFB08B9204610BD002010BD1C
:10C6D000C2281700000080000010000000010000C8
:10C6E00030B54A4800210160416000204849086097
:10C6F000484949480A6802604B6843608A6882601A
:10C70000CB68C3600A6902614B6943618A6902624E
:10C71000CB6943620A6A82624B6AC3628A6A0263B5
:10C72000CB6A43630A6B02644B6B43648A6B82641B
:10C73000CB6BC364096C016538490868082804BFDD
:10C740004868002802D13648364A02600B68082B38
:10C7500004BF4868002802D13348FB2202600B68FE
:10C76000082B04BF4868002809D13048304B0268C4
:10C770001C78120904F00F0444EA021202600868EF
:10C78000082804BF4868002803D12A484FF40071E4
:10C79000016029480168CA0744BF6FF001010160C8
:10C7A0002649C86F40F47000C867BFF34F8FBFF3CE
:10C7B0006F8F234A106800285CBF506800281CD582
:10C7C000204B01241C60204C00F042F8122515601B
:10C7D00000F03EF8556000F03BF800221A6000F0CF
:10C7E00037F8BFF34F8F0A68184802F4E06202433B
:10C7F0000A60BFF34F8F00BFFDE7024A0249116094
:10C8000030BD00008C0700200090D0030C010040D8
:10C81000380500400404001020C50040300100101D
:10C820008C5600404881030018F50040E40E00409B
:10C830005802001040960240000400400CED00E059
:10C840000012001004E5014000E401400400FA0574
:10C8500020680028FCD07047443A5C6E6F726469AF
:10C86000635C73646B31365F305F7472756E6B5CE2
:10C870006578616D706C65735C7065726970686510
:10C8800072616C5C757362645F6D73635C7063612D
:10C8900031303035365C626C616E6B5C6961725C44
:10C8A0002E2E5C2E2E5C2E2E5C2E2E5C2E2E5C2EC2
:10C8B0002E5C696E746567726174696F6E5C6E720E
:10C8C00066785C6E7266785F676C75652E680000CE
:10C8D000443A5C6E6F726469635C73646B31365F9B
:10C8E000305F7472756E6B5C6578616D706C6573CA
:10C8F0005C7065726970686572616C5C75736264A6
:10C900005F6D73635C70636131303035365C626CCF
:10C91000616E6B5C6961725C2E2E5C2E2E5C2E2E1D
:10C920005C2E2E5C2E2E5C2E2E5C6D6F64756C65FD
:10C93000735C6E7266785C68616C2F6E72665F7293
:10C9400074632E6800000000443A5C6E6F72646984
:10C95000635C73646B31365F305F7472756E6B5CF1
:10C96000636F6D706F6E656E74735C6C696272611B
:10C97000726965735C74696D65725C6472765F720E
:10C9800074632E630000000052544320696E737478
:10C99000616E636520616C726561647920696E699E
:10C9A0007469616C697A65642E0000002DE9FC47AA
:10C9B0000446F5F7CDFBF5F797FA0028FBD12E4892
:10C9C0002E4F2F4DDFF8BC802E68C71BFF083F0499
:10C9D00047F00107BCB1A2692FA100F059F8E06847
:10C9E00001903846A1680091636822684146F5F7D6
:10C9F0005CFAE06900906369226908F13801384601
:10CA0000F5F748FA04E008F160013846F5F731FA25
:10CA10006868810704D508F194013846F5F729FACA
:10CA20004FF0000A0FF28808DFF85C9026FA0AF04F
:10CA3000C00705D559F82A2012B1414600F028F860
:10CA40000AF1010ABAF11A0FF0D3300603D5EA68E9
:10CA50001AA100F01DF8300403D52A691FA100F0C7
:10CA600017F80A480168CA0700D500BE2046BDE88D
:10CA7000F64700F041B8000080D4000058D4000010
:10CA800028ED00E0E8CD000080020020F0ED00E09D
:10CA90003846F5F7F1B90000484152442046415567
:10CAA0004C54206174203078253038580000000044
:10CAB00043617573653A2025732E00004D656D4DF9
:10CAC000616E616765204661756C742041646472B3
:10CAD0006573733A203078253038580042757320DA
:10CAE0004661756C7420416464726573733A2030DA
:10CAF0007825303858000000BFF34F8F05490648AD
:10CB00000A6802F4E06202430A60BFF34F8F00BF7D
:10CB1000FDE700BF0CED00E00400FA050000000096
:10CB2000B0EA00000100000094E6000002000000EE
:10CB300098E500000300000060E900000400000028
:10CB400074E900000500000088E90000060000000C
:10CB500050E800000700000068E80000080000003E
:10CB600080E800000900000064E700000A000000FF
:10CB700098E800000B000000B0E800000C00000086
:10CB80009CE900000D000000B0E900000E0000006C
:10CB90001CEA00000F000000C4E9000010000000C3
:10CBA000C8E80000110000002CEA0000800000002E
:10CBB000BCE500008100000080E70000820000006A
:10CBC0009CE7000083000000B4E600008400000041
:10CBD000E0E5000085000000FCE4000086000000A5
:10CBE000E0E8000090000000D4E6000091000000A2
:10CBF000F4E6000092000000F8E800000082000067
:10CC000014E7000001820000B8E700000282000083
:10CC1000D4E700000084000004E600000184000066
:10CC2000A8E400000284000024E500000384000062
:10CC300028E6000081B00022425040580090009940
:10CC400001B07047405800B10120C0B2704710B524
:10CC500004462068302805D3DFF8981040F2CD1044
:10CC6000F4F752FE20681F2802D84FF0A04010BDF4
:10CC700000F01F002060DFF8800010BD01B568469D
:10CC8000FFF7E5FF009901228A40C0F8082501BDA1
:10CC900001B56846FFF7DBFF009901228A40C0F822
:10CCA0000C2501BD10B5174C00F02EF800B34FF461
:10CCB0008C712046FFF7BEFF104C206820B9104948
:10CCC0004FF42770F4F720FEE07FFF2806D0A17F05
:10CCD00011B1FFF7DDFF01E0FFF7D0FF0020607723
:10CCE00020726168226804F10800BDE81040104716
:10CCF00010BD0000C8D5000000030050282B002004
:10CD0000B8D00000003000404FF48C71204699E705
:10CD1000443A5C6E6F726469635C73646B31365F56
:10CD2000305F7472756E6B5C6578616D706C657385
:10CD30005C7065726970686572616C5C7573626461
:10CD40005F6D73635C70636131303035365C626C8B
:10CD5000616E6B5C6961725C2E2E5C2E2E5C2E2ED9
:10CD60005C2E2E5C2E2E5C2E2E5C636F6D706F6EB3
:10CD7000656E74735C6C69627261726965735C6222
:10CD80006C6F636B5F6465765C6E72665F626C6F1E
:10CD9000636B5F6465762E6800000000443A5C6E49
:10CDA0006F726469635C73646B31365F305F747299
:10CDB000756E6B5C636F6D706F6E656E74735C6CBB
:10CDC00069627261726965735C757362645C636CDD
:10CDD0006173735C6D73635C6170705F75736264C3
:10CDE0005F6D73632E630000202052303A202030A4
:10CDF0007825303858202052313A2020307825309C
:10CE00003858202052323A202030782530385820A7
:10CE10002052333A20203078253038580000000066
:10CE200020205231323A2030782530385820204C9A
:10CE3000523A202030782530385820205053523A2A
:10CE40002030782530385800537461636B20766940
:10CE50006F6C6174696F6E3A20737461636B2070DC
:10CE60006F696E746572206F757473696465207381
:10CE70007461636B20617265612E0000436175739C
:10CE8000653A204275734661756C74206F6E20613F
:10CE900020766563746F72207461626C65207265C0
:10CEA000616420647572696E67206578636570746B
:10CEB000696F6E2070726F63657373696E672E00A1
:10CEC000443A5C6E6F726469635C73646B31365FA5
:10CED000305F7472756E6B5C6578616D706C6573D4
:10CEE0005C7065726970686572616C5C75736264B0
:10CEF0005F6D73635C70636131303035365C626CDA
:10CF0000616E6B5C6961725C2E2E5C2E2E5C2E2E27
:10CF10005C2E2E5C2E2E5C2E2E5C636F6D706F6E01
:10CF2000656E74735C6C69627261726965735C6270
:10CF30006C6F636B5F6465765C6E72665F626C6F6C
:10CF4000636B5F6465762E6800000000443A5C6E97
:10CF50006F726469635C73646B31365F305F7472E7
:10CF6000756E6B5C65787465726E616C5C6661741D
:10CF700066735C706F72745C6469736B696F5F6217
:10CF80006C6B6465762E6300443A5C6E6F72646904
:10CF9000635C73646B31365F305F7472756E6B5CAB
:10CFA0006578616D706C65735C70657269706865D9
:10CFB00072616C5C757362645F6D73635C706361F6
:10CFC00031303035365C626C616E6B5C6961725C0D
:10CFD0002E2E5C2E2E5C2E2E5C2E2E5C2E2E5C2E8B
:10CFE0002E5C696E746567726174696F6E5C6E72D7
:10CFF00066785C6E7266785F676C75652E68000097
:10D00000443A5C6E6F726469635C73646B31365F63
:10D01000305F7472756E6B5C6D6F64756C65735C9C
:10D020006E7266785C647269766572735C73726343
:10D030005C6E7266785F717370692E630000000029
:10D04000443A5C6E6F726469635C73646B31365F23
:10D05000305F7472756E6B5C6578616D706C657352
:10D060005C7065726970686572616C5C757362642E
:10D070005F6D73635C70636131303035365C626C58
:10D08000616E6B5C6961725C2E2E5C2E2E5C2E2EA6
:10D090005C2E2E5C2E2E5C2E2E5C696E7465677283
:10D0A0006174696F6E5C6E7266785C6E7266785FD2
:10D0B000676C75652E680000443A5C6E6F72646937
:10D0C000635C73646B31365F305F7472756E6B5C7A
:10D0D0006D6F64756C65735C6E7266785C647269A2
:10D0E000766572735C7372635C6E7266785F737080
:10D0F000696D2E6300000000443A5C6E6F726469D3
:10D10000635C73646B31365F305F7472756E6B5C39
:10D110006578616D706C65735C7065726970686567
:10D1200072616C5C757362645F6D73635C70636184
:10D1300031303035365C626C616E6B5C6961725C9B
:10D140002E2E5C2E2E5C2E2E5C2E2E5C2E2E5C2E19
:10D150002E5C696E746567726174696F6E5C6E7265
:10D1600066785C6E7266785F676C75652E68000025
:10D17000443A5C6E6F726469635C73646B31365FF2
:10D18000305F7472756E6B5C6D6F64756C65735C2B
:10D190006E7266785C647269766572735C737263D2
:10D1A0005C6E7266785F756172742E6300000000B9
:10D1B000443A5C6E6F726469635C73646B31365FB2
:10D1C000305F7472756E6B5C6578616D706C6573E1
:10D1D0005C7065726970686572616C5C75736264BD
:10D1E0005F6D73635C70636131303035365C626CE7
:10D1F000616E6B5C6961725C2E2E5C2E2E5C2E2E35
:10D200005C2E2E5C2E2E5C2E2E5C696E7465677211
:10D210006174696F6E5C6E7266785C6E7266785F60
:10D22000676C75652E680000443A5C6E6F726469C5
:10D23000635C73646B31365F305F7472756E6B5C08
:10D240006D6F64756C65735C6E7266785C64726930
:10D25000766572735C7372635C6E7266785F75611B
:10D260007274652E63000000443A5C6E6F726469EC
:10D27000635C73646B31365F305F7472756E6B5CC8
:10D280006578616D706C65735C70657269706865F6
:10D2900072616C5C757362645F6D73635C70636113
:10D2A00031303035365C626C616E6B5C6961725C2A
:10D2B0002E2E5C2E2E5C2E2E5C2E2E5C2E2E5C2EA8
:10D2C0002E5C6D6F64756C65735C6E7266785C68FD
:10D2D000616C2F6E72665F757362642E6800000069
:10D2E000443A5C6E6F726469635C73646B31365F81
:10D2F000305F7472756E6B5C6D6F64756C65735CBA
:10D300006E7266785C647269766572735C73726360
:10D310005C6E7266785F757362642E630000000055
:10D32000443A5C6E6F726469635C73646B31365F40
:10D33000305F7472756E6B5C6578616D706C65736F
:10D340005C7065726970686572616C5C757362644B
:10D350005F6D73635C6D61696E2E6300352E2043D3
:10D360006F6E6E65637420746F20504320616E642D
:10D37000206F70656E2054455354312E747874209C
:10D38000746F20636865636B2069662066696C65ED
:10D3900020636F72727570746564206F72206E6F97
:10D3A000742E00004027002024E900000100020341
:10D3B000810100005018002000040000020000005D
:10D3C000E802002001000000219200000650000049
:10D3D0005468652070726F636573736F7220686143
:10D3E0007320617474656D7074656420616E20696A
:10D3F0006C6C6567616C206C6F6164206F662045A2
:10D4000058435F52455455524E20746F20746865DE
:10D410002050432C206173206120726573756C74F9
:10D42000206F6620616E20696E76616C696420638E
:10D430006F6E746578742C206F7220616E20696E37
:10D4400076616C6964204558435F52455455524E8D
:10D450002076616C756500005CEA00000000000049
:10D4600068EA00000000000074EA0000000000000C
:10D47000ECE900000000000080EA0000000000006D
:10D480008CEA000000000303F0EA00000000000046
:10D4900080EB000000000303A4EA0000000000008D
:10D4A00050EB00000000000058EB000000000000FE
:10D4B00084EB00000000000060EB000000000000B2
:10D4C00068EB00000000000070EB000000000000AE
:10D4D00078EB000000000000443A5C6E6F726469F3
:10D4E000635C73646B31365F305F7472756E6B5C56
:10D4F0006578616D706C65735C7065726970686584
:10D5000072616C5C757362645F6D73635C706361A0
:10D5100031303035365C626C616E6B5C6961725CB7
:10D520002E2E5C2E2E5C2E2E5C2E2E5C2E2E5C2E35
:10D530002E5C6D6F64756C65735C6E7266785C688A
:10D54000616C5C6E72665F6770696F2E68000000C8
:10D55000443A5C6E6F726469635C73646B31365F0E
:10D56000305F7472756E6B5C6578616D706C65733D
:10D570005C7065726970686572616C5C7573626419
:10D580005F6D73635C70636131303035365C626C43
:10D59000616E6B5C6961725C2E2E5C2E2E5C2E2E91
:10D5A0005C2E2E5C2E2E5C2E2E5C6D6F64756C6571
:10D5B000735C6E7266785C68616C2F6E72665F6712
:10D5C00070696F2E68000000443A5C6E6F72646987
:10D5D000635C73646B31365F305F7472756E6B5C65
:10D5E0006578616D706C65735C7065726970686593
:10D5F00072616C5C757362645F6D73635C706361B0
:10D6000031303035365C626C616E6B5C6961725CC6
:10D610002E2E5C2E2E5C2E2E5C2E2E5C2E2E5C2E44
:10D620002E5C6D6F64756C65735C6E7266785C6899
:10D63000616C2F6E72665F6770696F2E6800000004
:10D64000443A5C6E6F726469635C73646B31365F1D
:10D65000305F7472756E6B5C6578616D706C65734C
:10D660005C7065726970686572616C5C7573626428
:10D670005F6D73635C70636131303035365C626C52
:10D68000616E6B5C6961725C2E2E5C2E2E5C2E2EA0
:10D690005C2E2E5C2E2E5C2E2E5C6D6F64756C6580
:10D6A000735C6E7266785C68616C2F6E72665F6721
:10D6B00070696F2E68000000443A5C6E6F72646996
:10D6C000635C73646B31365F305F7472756E6B5C74
:10D6D0006578616D706C65735C70657269706865A2
:10D6E00072616C5C757362645F6D73635C706361BF
:10D6F00031303035365C626C616E6B5C6961725CD6
:10D700002E2E5C2E2E5C2E2E5C2E2E5C2E2E5C2E53
:10D710002E5C6D6F64756C65735C6E7266785C68A8
:10D72000616C2F6E72665F6770696F2E6800000013
:10D73000F0B40246106895681318506803EB500463
:10D74000C0071CD54D441AE013F8017B05F8017B96
:10D75000491EF9D198B113F8011BC6F38106032EB7
:10D7600008BF13F8016B01EB06214942801C2944D4
:10D7700005D011F8016B05F8016B401EF9D1A342E9
:10D780000ED013F8016B16F0030104BF13F8011B50
:10D79000C91C30090F28DBD113F8010B0F30D7E774
:10D7A000F0BC02F10C007047446174612062757333
:10D7B000206572726F72202850432076616C756507
:10D7C00020737461636B656420666F722074686592
:10D7D00020657863657074696F6E20726574757208
:10D7E0006E20706F696E747320746F20746865208A
:10D7F000696E737472756374696F6E207468617496
:10D800002063617573656420746865206661756C5A
:10D81000742900004461746120627573206572721E
:10D820006F72202872657475726E2061646472650F
:10D83000737320696E2074686520737461636B2054
:10D840006672616D65206973206E6F742072656CFD
:10D850006174656420746F2074686520696E7374E8
:10D8600072756374696F6E2074686174206361758A
:10D8700073656420746865206572726F7229000098
:10D88000A1070000C107000005090000070900000A
:10D890000B0900000F090000130900001709000020
:10D8A0001B0900001F090000DD0A00002509000017
:10D8B00069090000C9090000CD090000D109000074
:10D8C000D5090000D9090000DD090000E1090000C8
:10D8D000E5090000290A0000650B0000F50A0000B8
:10D8E000E50B00005468652070726F636573736F99
:10D8F0007220617474656D707465642061206C6F52
:10D900006164206F722073746F726520617420618E
:10D91000206C6F636174696F6E2074686174206439
:10D920006F6573206E6F74207065726D69742074FA
:10D930006865206F7065726174696F6E0000000029
:10D940005468652070726F636573736F72206861CD
:10D950007320617474656D7074656420746F2065E4
:10D9600078656375746520616E20696E7374727575
:10D970006374696F6E2074686174206D616B657388
:10D9800020696C6C6567616C20757365206F66201B
:10D99000746865204550535200000000556E616266
:10D9A0006C6520746F206F706572617465206F6E96
:10D9B0002066696C6573797374656D207768696C2E
:10D9C000652055534220697320636F6E6E656374E2
:10D9D000656400000D0A556E61626C6520746F20ED
:10D9E0006F70656E206F722063726561746520666A
:10D9F000696C653A20257500443A5C6E6F72646903
:10DA0000635C73646B31365F305F7472756E6B5C30
:10DA1000636F6D706F6E656E74735C6C696272615A
:10DA2000726965735C626C6F636B5F6465765C7171
:10DA30007370695C6E72665F626C6F636B5F646566
:10DA4000765F717370692E6300000000443A5C6E6B
:10DA50006F726469635C73646B31365F305F7472DC
:10DA6000756E6B5C636F6D706F6E656E74735C6CFE
:10DA700069627261726965735C6C6F675C73726313
:10DA80005C6E72665F6C6F675F64656661756C740F
:10DA90005F6261636B656E64732E6300443A5C6E13
:10DAA0006F726469635C73646B31365F305F74728C
:10DAB000756E6B5C636F6D706F6E656E74735C6CAE
:10DAC00069627261726965735C757362645C6170CE
:10DAD000705F757362645F737472696E675F6465AB
:10DAE00073632E6300000000556E737461636B20D6
:10DAF000666F7220616E20657863657074696F6E01
:10DB00002072657475726E2068617320636175732D
:10DB10006564206F6E65206F72206D6F7265206185
:10DB200063636573732076696F6C6174696F6E737C
:10DB300000000000537461636B696E6720666F724A
:10DB400020616E20657863657074696F6E20656E04
:10DB50007472792068617320636175736564206FE6
:10DB60006E65206F72206D6F7265206163636573EF
:10DB7000732076696F6C6174696F6E7300000000CA
:10DB800041204D656D4D616E616765206661756C04
:10DB900074206F6363757272656420647572696E58
:10DBA0006720666C6F6174696E672D706F696E7443
:10DBB000206C617A7920737461746520707265736A
:10DBC0006572766174696F6E0000000054686520AC
:10DBD00070726F636573736F72206861732065780C
:10DBE00065637574656420616E2053444956206FE7
:10DBF00072205544495620696E7374727563746956
:10DC00006F6E207769746820612064697669736F2C
:10DC100072206F6620300000443A5C6E6F72646957
:10DC2000635C73646B31365F305F7472756E6B5C0E
:10DC3000636F6D706F6E656E74735C6C6962726138
:10DC4000726965735C6C6F675C7372635C6E72663D
:10DC50005F6C6F675F6261636B656E645F75617255
:10DC6000742E6300415353455254494F4E20464150
:10DC7000494C45442061742025733A257500000005
:10DC8000456E64206F66206572726F7220726570D7
:10DC90006F727400554E4B4E4F574E204641554CB7
:10DCA000542061742030782530385800443A5C6E36
:10DCB0006F726469635C73646B31365F305F74727A
:10DCC000756E6B5C636F6D706F6E656E74735C6C9C
:10DCD00069627261726965735C757362645C6170BC
:10DCE000705F757362645F636C6173735F626173AD
:10DCF000652E6800443A5C6E6F726469635C73649D
:10DD00006B31365F305F7472756E6B5C636F6D7014
:10DD10006F6E656E74735C6C696272617269657353
:10DD20005C757362645C6170705F757362645F637D
:10DD30006C6173735F626173652E6800443A5C6E58
:10DD40006F726469635C73646B31365F305F7472E9
:10DD5000756E6B5C636F6D706F6E656E74735C6C0B
:10DD600069627261726965735C7574696C5C61701B
:10DD7000705F7574696C5F706C6174666F726D2E24
:10DD800063000000443A5C6E6F726469635C7364A4
:10DD90006B31365F305F7472756E6B5C636F6D7084
:10DDA0006F6E656E74735C6C6962726172696573C3
:10DDB0005C6C6F675C7372635C6E72665F6C6F67DE
:10DDC0005F66726F6E74656E642E6300443A5C6EBB
:10DDD0006F726469635C73646B31365F305F747259
:10DDE000756E6B5C636F6D706F6E656E74735C6C7B
:10DDF00069627261726965735C736F72746C697366
:10DE0000745C6E72665F736F72746C6973742E6388
:10DE100000000000443A5C6E6F726469635C736476
:10DE20006B31365F305F7472756E6B5C636F6D70F3
:10DE30006F6E656E74735C6C696272617269657332
:10DE40005C627574746F6E5C6170705F627574741F
:10DE50006F6E2E6300000000443A5C6E6F7264695E
:10DE6000635C73646B31365F305F7472756E6B5CCC
:10DE7000636F6D706F6E656E74735C6C69627261F6
:10DE8000726965735C757362645C6170705F7573F1
:10DE900062645F636F72652E63000000556E737479
:10DEA00061636B20666F7220616E206578636570B8
:10DEB00074696F6E2072657475726E20686173206C
:10DEC000636175736564206F6E65206F72206D6F7E
:10DED0007265204275734661756C747300000000B2
:10DEE000537461636B696E6720666F7220616E2088
:10DEF000657863657074696F6E20656E74727920E1
:10DF000068617320636175736564206F6E65206F4F
:10DF100072206D6F7265204275734661756C747303
:10DF2000000000004120627573206661756C7420EA
:10DF30006F6363757272656420647572696E6720C1
:10DF4000666C6F6174696E672D706F696E74206C9A
:10DF5000617A79207374617465207072657365727B
:10DF6000766174696F6E0000443A5C6E6F7264692A
:10DF7000635C73646B31365F305F7472756E6B5CBB
:10DF8000636F6D706F6E656E74735C6C69627261E5
:10DF9000726965735C62616C6C6F635C6E72665F04
:10DFA00062616C6C6F632E6300000000443A5C6E2B
:10DFB0006F726469635C73646B31365F305F747277
:10DFC000756E6B5C636F6D706F6E656E74735C6C99
:10DFD00069627261726965735C6D656D6F626A5CBE
:10DFE0006E72665F6D656D6F626A2E630000000081
:10DFF000443A5C6E6F726469635C73646B31365F64
:10E00000305F7472756E6B5C636F6D706F6E656E92
:10E0100074735C6C69627261726965735C74696D5A
:10E0200065725C6170705F74696D6572322E630039
:10E03000443A5C6E6F726469635C73646B31365F23
:10E04000305F7472756E6B5C636F6D706F6E656E52
:10E0500074735C6C69627261726965735C7573621A
:10E06000645C6170705F757362642E68000000000C
:10E07000443A5C6E6F726469635C73646B31365FE3
:10E08000305F7472756E6B5C636F6D706F6E656E12
:10E0900074735C6C69627261726965735C757362DA
:10E0A000645C6170705F757362642E6300000000D1
:10E0B000443A5C6E6F726469635C73646B31365FA3
:10E0C000305F7472756E6B5C636F6D706F6E656ED2
:10E0D00074735C6C69627261726965735C7573629A
:10E0E000645C6170705F757362642E68000000008C
:10E0F0005468652070726F636573736F7220686116
:10E100007320617474656D7074656420746F20652C
:10E1100078656375746520616E20756E64656669E7
:10E120006E656420696E737472756374696F6E00D6
:10E13000443A5C6E6F726469635C73646B31365F22
:10E14000305F7472756E6B5C696E74656772617452
:10E15000696F6E5C6E7266785C6C65676163795C32
:10E160006E72665F6472765F636C6F636B2E6300C2
:10E17000443A5C6E6F726469635C73646B31365FE2
:10E18000305F7472756E6B5C696E74656772617412
:10E19000696F6E5C6E7266785C6C65676163795CF2
:10E1A0006E72665F6472765F756172742E630000D2
:10E1B000443A5C6E6F726469635C73646B31365FA2
:10E1C000305F7472756E6B5C65787465726E616CCD
:10E1D0005C667072696E74665C6E72665F667072A1
:10E1E000696E74665F666F726D61742E6300000005
:10E1F000443A5C6E6F726469635C73646B31365F62
:10E20000305F7472756E6B5C6D6F64756C65735C9A
:10E210006E7266785C647269766572735C73726341
:10E220005C6E7266785F636C6F636B2E63000000D8
:10E23000443A5C6E6F726469635C73646B31365F21
:10E24000305F7472756E6B5C6D6F64756C65735C5A
:10E250006E7266785C647269766572735C73726301
:10E260005C6E7266785F6770696F74652E6300001C
:10E27000443A5C6E6F726469635C73646B31365FE1
:10E28000305F7472756E6B5C6D6F64756C65735C1A
:10E290006E7266785C647269766572735C737263C1
:10E2A0005C6E7266785F706F7765722E6300000037
:10E2B000443A5C6E6F726469635C73646B31365FA1
:10E2C000305F7472756E6B5C6D6F64756C65735CDA
:10E2D0006E7266785C647269766572735C73726381
:10E2E0005C7072735C6E7266785F7072732E63001E
:10E2F000443A5C6E6F726469635C73646B31365F61
:10E30000305F7472756E6B5C6D6F64756C65735C99
:10E310006E7266785C647269766572735C73726340
:10E320005C6E7266785F7379737469636B2E6300D9
:10E330004D6F756E74206661696C65642E20466948
:10E340006C6573797374656D206E6F7420666F757C
:10E350006E642E20506C6561736520666F726D610E
:10E3600074206465766963652E000000443A5C6E33
:10E370006F726469635C73646B31365F305F7472B3
:10E38000756E6B5C65787465726E616C5C667072DC
:10E39000696E74665C6E72665F667072696E7466D2
:10E3A0002E6300000B4B1EF0040F1CBFEFF309801F
:10E3B0001847EFF308800549054A884201D8904282
:10E3C00002D88D464FF00000184700BF584C00207F
:10E3D000582C0020ADC900007047FEE7443A5C6E3F
:10E3E0006F726469635C73646B31365F305F747243
:10E3F000756E6B5C636F6D706F6E656E74735C626F
:10E400006F617264735C626F617264732E6300008B
:10E410005468652070726F636573736F72206861F2
:10E420007320617474656D7074656420746F20610D
:10E430006363657373206120636F70726F636573CC
:10E44000736F72005468652070726F636573736FC9
:10E450007220686173206D61646520616E20756E45
:10E46000616C69676E6564206D656D6F727920619E
:10E47000636365737300000038E80000D8EA0000A9
:10E48000E0EA0000E8EA00000002000001000000ED
:10E490000000000013111415161700000000010001
:10E4A000000F0600180800204E52465F4552524F9A
:10E4B000525F424C455F495053505F4348414E4E76
:10E4C000454C5F414C52454144595F45584953546E
:10E4D000530000004552524F52202575205B257392
:10E4E0005D2061742025733A25750D0A5043206123
:10E4F000743A203078253038780000004E52465F5C
:10E500004552524F525F4D4F44554C455F414C521E
:10E51000454144595F494E495449414C495A454443
:10E52000000000004E52465F4552524F525F424C2F
:10E53000455F495053505F4C494E4B5F44495343EC
:10E540004F4E4E45435445440000000010B5074966
:10E5500079441831064C7C44163404E00A68081DDE
:10E56000114488470146A142F8D110BD04010000C2
:10E5700020010000556E2D696E697469616C697ABD
:10E58000696E67206469736B2030202851535049AD
:10E59000292E2E2E000000004E52465F4552524F4B
:10E5A000525F534F46544445564943455F4E4F547E
:10E5B0005F454E41424C4544000000004E52465FCC
:10E5C0004552524F525F4D4F44554C455F4E4F544C
:10E5D0005F494E495449414C495A454400000000A6
:10E5E0004E52465F4552524F525F4D555445585F0B
:10E5F000434F4E445F494E49545F4641494C454460
:10E60000000000004E52465F4552524F525F424C4E
:10E61000455F495053505F52585F504B545F5452BE
:10E62000554E4341544544004E52465F4552524F69
:10E63000525F424C455F495053505F504545525FD1
:10E6400052454A4543544544000000004EF6885167
:10E65000CEF20001086840F470000860BFF34F8FED
:10E66000BFF36F8F4FF00070E1EE100A70470000AB
:10E67000AF32FFFF3C24000018080020000000001B
:10E68000B1F0FFFF2D050000EE01000000000020AA
:10E69000FEE700004E52465F4552524F525F5356BE
:10E6A000435F48414E444C45525F4D495353494E98
:10E6B000470000004E52465F4552524F525F4D5543
:10E6C0005445585F554E4C4F434B5F4641494C456E
:10E6D000440000004E52465F4552524F525F415037
:10E6E000495F4E4F545F494D504C454D454E544542
:10E6F000440000004E52465F4552524F525F46451D
:10E7000041545552455F4E4F545F454E41424C4532
:10E71000440000004E52465F4552524F525F4452F1
:10E72000565F5457495F4552525F4F5645525255B6
:10E730004E0000000120C046002801D0FFF706FF70
:10E74000AFF300800020AFF30080FAF70FFE00F077
:10E7500000F800F001B8FEE707463846FAF722FC59
:10E76000FBE7FEE74E52465F4552524F525F494E1D
:10E7700056414C49445F4C454E4754480000000008
:10E780004E52465F4552524F525F4D555445585F69
:10E79000494E49545F4641494C4544004E52465FFC
:10E7A0004552524F525F4D555445585F4C4F434B65
:10E7B0005F4641494C4544004E52465F4552524FD8
:10E7C000525F4452565F5457495F4552525F414E23
:10E7D00041434B004E52465F4552524F525F4452A6
:10E7E000565F5457495F4552525F444E41434B0078
:10E7F0004E6F726469632053656D69636F6E6475F3
:10E8000063746F720000000044656661756C74206B
:10E81000636F6E66696775726174696F6E00000080
:10E82000496E737472756374696F6E2062757320BC
:10E830006572726F720000006FBD00007DBE000047
:10E84000E9BE0000CBC000008DC10000F3C1000094
:10E850004E52465F4552524F525F4E4F545F535592
:10E8600050504F52544544004E52465F4552524F0D
:10E87000525F494E56414C49445F504152414D0010
:10E880004E52465F4552524F525F494E56414C4997
:10E89000445F5354415445004E52465F4552524FD7
:10E8A000525F494E56414C49445F464C41475300E4
:10E8B0004E52465F4552524F525F494E56414C4967
:10E8C000445F4441544100004E52465F4552524F0E
:10E8D000525F494E56414C49445F41444452000006
:10E8E0004E52465F4552524F525F53544F5241472A
:10E8F000455F46554C4C00004E52465F4552524FC4
:10E90000525F494F5F50454E44494E47000000005A
:10E91000FD66000000000000000000000000000094
:10E9200000000000214F0000CF5600000000000052
:10E9300000000000000000006E52463532205553A2
:10E9400042204D53432044656D6F00007561727421
:10E950005F6C6F675F6261636B656E6400000000EF
:10E960004E52465F4552524F525F494E5445524EA9
:10E97000414C00004E52465F4552524F525F4E4F3F
:10E980005F4D454D000000004E52465F4552524FCC
:10E99000525F4E4F545F464F554E44004E52465FB5
:10E9A0004552524F525F444154415F53495A4500CA
:10E9B0004E52465F4552524F525F54494D454F5556
:10E9C000540000004E52465F4552524F525F464F30
:10E9D0005242494444454E00302C0020282C00204F
:10E9E000302C002080260020180000006170705F2D
:10E9F000757362645F636F7265000000E02B002036
:10EA000010E90000010002030080000030303030C7
:10EA10003030303030303031000000004E52465F30
:10EA20004552524F525F4E554C4C00004E52465F7D
:10EA30004552524F525F425553590000014880479A
:10EA400001480047E1C60000BDEA000098EA000066
:10EA5000000000004CE90000440700206170705F76
:10EA6000627574746F6E00006170705F74696D65BB
:10EA7000720000006170705F7573626400000000D6
:10EA8000757362645F6D7363000000006861726497
:10EA90006661756C7400000015A2000027A20000DA
:10EAA00025A20000736F72746C697374000000001B
:10EAB0004E52465F5355434345535300AFF30080D6
:10EAC000FFF7C4FDFFF736FE000004030904000051
:10EAD00055736572203100004E6F726469630000E7
:10EAE0005153504900000000312E3030000000002A
:10EAF000636C6F636B0000006572726F72000000E0
:10EB00007761726E696E6700696E666F0000000063
:10EB100064656275670000001B5B313B33306D003C
:10EB20001B5B313B33326D001B5B313B33336D007C
:10EB30001B5B313B33346D001B5B313B33356D0068
:10EB40001B5B313B33366D001B5B313B33376D0054
:10EB5000434C4F434B0000004750494F5445000081
:10EB60005350494D00000000554152540000000030
:10EB700055415254450000005553424400000000E6
:10EB80006170700050525300FEE7FEE7FEE7FEE7BB
:10EB9000FEE7FEE7FEE7FEE7FEE7FEE7FEE7FEE74D
:10EBA000FEE7FEE7FEE7FEE7FEE7FEE7FEE7FEE73D
:10EBB00000F20B0001F005FF1001401100040001FC
:10EBC000F1FF01F10B014B1D5D3F100BC8EA000086
:10EBD000F0E7000038E900000C0C200308E8000012
:10EBE000D0144003E00000E4D8248808E8DA0000EC
:10EBF00034DB000080DB731220281003A8D700004C
:10EC0000142410039CDE0000E0048324DF20214054
:10EC10001340D94C1AD3AFFA01E4AB12441412CC0E
:10EC200050F001FF78E40001F1FF01F104017938AF
:10EC3000F3FF010001F1E90138012000400E6108F5
:10EC4000110152FF091EF8D4041F00EBE004110467
:10EC50001210041003D8240000180812E008122033
:10EC6000081228041230041238041240049B48EBA6
:10EC700058200190D0030E296BF309B0EB0452FF2A
:10EC800001E3DA2614400200009265401398079EC3
:10EC9000110143B32C6012AD0852C90CCBB12CCC7E
:08ECA00043B11A108B9F1AE723
:040000050000EABD50
:00000001FF
